:020000040800F2
:10000000B057012439040008EF8A0008EF7F000888
:10001000ED8A0008A10B000861B50008000000008F
:10002000000000000000000000000000790300084C
:10003000851D000800000000D50300085993000842
:100040005304000853040008530400085304000834
:100050005304000853040008530400085304000824
:100060005304000853040008530400085304000814
:100070005304000853040008530400085304000804
:10008000DD18000853040008530400085304000856
:1000900053040008530400085304000853040008E4
:1000A00053040008530400085304000853040008D4
:1000B00053040008530400085304000853040008C4
:1000C00053040008530400085304000853040008B4
:1000D00053040008A9A200085304000853040008B0
:1000E00053040008530400080000000053040008F3
:1000F0005304000853040008530400085304000884
:100100005304000853040008530400085304000873
:10011000530400085304000853040008F99400082D
:100120005304000853040008530400085304000853
:100130005304000853040008530400085304000843
:1001400000000000000000000000000000000000AF
:100150005304000853040008530400085304000823
:100160005304000853040008530400085304000813
:100170005304000853040008530400085304000803
:1001800053040008530400085304000853040008F3
:1001900053040008530400085304000853040008E3
:1001A00053040008530400085304000853040008D3
:1001B00053040008530400085304000853040008C3
:1001C00053040008530400085304000853040008B3
:1001D00053040008F18A000853040008530400087F
:1001E0005304000853040008530400085304000893
:1001F0005304000853040008530400085304000883
:100200005304000853040008530400085304000872
:100210005304000853040008530400085304000862
:1002200053040008530400085304000800000000B1
:1002300053040008530400080000000053040008A1
:10024000E9180008950B000853040008530400083F
:100250005304000853040008530400085304000822
:100260005304000853040008530400085304000812
:100270005304000853040008530400080000000061
:100280005304000853040008530400080000000051
:10029000000000005304000800F002F800F05CF8D1
:1002A0000AA090E8000C82448344AAF10107DA45D1
:1002B00001D100F051F8AFF2090EBAE80F0013F0C7
:1002C000010F18BFFB1A43F00103184714E50000A3
:1002D00034E500000A444FF0000C10F8013B13F025
:1002E000070408BF10F8014B1D1108BF10F8015B8F
:1002F000641E05D010F8016B641E01F8016BF9D182
:1003000013F0080F1EBF10F8014BAD1C0C1B09D1D8
:100310006D1E58BF01F801CBFAD505E014F8016B4A
:1003200001F8016B6D1EF9D59142D6D370470000DC
:100330000023002400250026103A28BF78C1FBD8EE
:10034000520728BF30C148BF0B6070471FB50DF082
:1003500079FE1FBD10B510BD00F0E4F91146FFF79E
:10036000F5FF0BF055FE00F002FA03B4FFF7F2FFC1
:1003700003BC00F005FA00002C4B19680868B0E8CF
:10038000F04F80F30988BFF36F8F4FF0000080F3C8
:10039000118870470000000008480068006880F37A
:1003A00008884FF0000080F3148862B661B6BFF38E
:1003B0004F8FBFF36F8F00DF00BF00BF08ED00E07D
:1003C000DFF80C00016841F470010160704700BF64
:1003D00088ED00E0EFF30980BFF36F8F134B1A68CD
:1003E0001EF0100F08BF20ED108A20E9F04F1060BA
:1003F00009B44FF0500080F31188BFF34F8FBFF363
:100400006F8F0CF0CBFE4FF0000080F3118809BC19
:1004100019680868B0E8F04F1EF0100F08BFB0EC84
:10042000108A80F30988BFF36F8F7047F8000024AB
:10043000EFF30580704700000948804709480047EE
:10044000FEE7FEE7FEE7FEE7FEE7FEE7FEE7FEE784
:10045000FEE7FEE704480549054A064B70470000E1
:100460001D94000899020008B0510124B0570124DE
:10047000B0530124B053012453EA020C00F0698008
:100480002DE9F04B4FF00006002B1FBFB3FA83F5A8
:1004900003FA05F424FA05F65E4012BF1643B2FAD9
:1004A00082F502FA05F4C5F120051EBF22FA05FC0B
:1004B00044EA0C04203556EA044C4FEA144418BFB1
:1004C000641C4FF000084FF00009904271EB030CE0
:1004D00039D3002919BFB1FA81F701FA07F6B0FA4A
:1004E00080F700FA07F6C7F120071EBF20FA07FCC5
:1004F00046EA0C062037B6FBF4FCA7EB0507103FD5
:1005000007F01F0BCBF120060CFA0BFB2CFA06F6BA
:1005100044BFB3460026202FA4BF5E464FF0000B19
:100520005BEA060C08BF4FF0010B19EB0B09ABFBA4
:10053000027C48EB0608C01B06FB02CC0BFB03CC7D
:1005400071EB0C01C1E70B46024641464846BDE847
:10055000F08B13B54FF000004FF00001AFF30080B7
:10056000BDE81C407047032A40F2308010F0030CB5
:1005700000F0158011F8013BBCF1020F624498BFF6
:1005800011F801CB00F8013B38BF11F8013BA2F193
:10059000040298BF00F801CB38BF00F8013B11F00E
:1005A000030300F02580083AC0F0088051F8043BAE
:1005B000083A51F804CBA0E80810F5E7121D5CBF1B
:1005C00051F8043B40F8043BAFF30080D20724BF4E
:1005D00011F8013B11F801CB48BF11F8012B24BFE2
:1005E00000F8013B00F801CB48BF00F8012B704731
:1005F00010B5203AC0F00B80B1E81850203AA0E8BE
:100600001850B1E81850A0E81850BFF4F5AF5FEAF1
:10061000027C24BFB1E81850A0E8185044BF18C9A4
:1006200018C0BDE810405FEA827C24BF51F8043B4B
:1006300040F8043B08BF7047D20728BF31F8023B9F
:1006400048BF11F8012B28BF20F8023B48BF00F833
:10065000012B704702F0FF0343EA032242EA024201
:1006600000F002B84FF000020429C0F0128010F030
:10067000030C00F01B80CCF1040CBCF1020F18BF7E
:1006800000F8012BA8BF20F8022BA1EB0C0100F011
:100690000DB85FEAC17C24BF00F8012B00F8012BE4
:1006A00048BF00F8012B70474FF0000200B5134619
:1006B00094469646203922BFA0E80C50A0E80C5082
:1006C000B1F12001BFF4F7AF090728BFA0E80C5033
:1006D00048BF0CC05DF804EB890028BF40F8042B2C
:1006E00008BF704748BF20F8022B11F0804F18BF99
:1006F00000F8012B704770477047704710B500F045
:1007000009F8006810BD10B5044600F003F8046055
:1007100010BD0000004870474C510124004870474C
:100720004C5101247546FFF7F9FFAE4605006946B6
:10073000534620F00700854618B020B5FFF78AFE23
:10074000BDE820404FF000064FF000074FF00008D2
:100750004FF0000B21F00701AC46ACE8C009ACE853
:10076000C009ACE8C009ACE8C0098D46704710B5B7
:100770000446AFF300802046BDE81040FFF7F5BD0A
:1007800001491820ABBEFEE72600020070470000BA
:1007900070B5054641492868884202D0404A9042D7
:1007A00005D1D1F8080310F4403F05D118E03D48C9
:1007B000006810F4403F13D005F0DAFF0446686883
:1007C000B0F5803F06D0B0F5003F03D0B0F5403F14
:1007D00029D103E0000CB4FBF0F424E0A40822E0EB
:1007E00000214FF4002004F05BFE0446686881039A
:1007F000890B18D181140C2915D2DFE801F01406F9
:1008000006060606060B0D0F1113800C4000B4FB04
:10081000F0F408E0240906E0640904E0A40902E019
:10082000E40900E0240A03F095FE41F20301884246
:100830000ED81D48844205D92868816841F480712A
:10084000816070BD2868816821F48071816070BD0D
:1008500060081649884205D82868816821F44071EB
:10086000816070BD1249884207D82868816821F4E8
:10087000407141F48071816070BD0E49884207D893
:100880002868816821F4407141F40071816070BD75
:100890002868816841F44071816070BD0020024089
:1008A0000021024008630258002D3101105E5F00F4
:1008B00020BCBE0040787D012DE9F04104460E4683
:1008C0000025206807F09CFB0746206807F090FB96
:1008D000074365D02068C16889011CD5617D012965
:1008E00019D1217D012916D101262E490DE08D4215
:1008F0000AD3606D40F010006065A06D40F001000B
:10090000A0650120BDE8F0816D1C0268D24352064B
:10091000EDD440210160244D022E0DD0206807F057
:100920006FFB48B120688168C1F3400121B981683B
:10093000294041F010018160012E0DD0206807F0A0
:1009400057FB48B120688168C1F3400121B9816833
:10095000294041F020018160022E08D0032E04D0EE
:10096000042503F0FDFD064616E00C25F9E70825F1
:10097000F7E703F0F5FD801B05280DD92068806896
:10098000284209D0606D40F010006065A06D40F015
:100990000100A0650120B5E7206880682842E8D101
:1009A0000020AFE700DC0C00C0FFFF7F10B5846BB8
:1009B000616D11F0500F06D0616DC90630D520462B
:1009C00001F052FE10BD606D40F40070606520685B
:1009D0000168090712D507F017FBE8B12068C06865
:1009E000800419D4606D20F480706065606DC0046F
:1009F00012D4606D40F0010060650DE0C0688007B2
:100A00000AD1606D20F480706065606DC00403D40D
:100A1000606D40F001006065204601F09DFC10BD56
:100A2000E16CC96CBDE81040084710B5806B416DA2
:100A300041F040014165816D41F00401816501F0A3
:100A400013FE10BD10B5806B01F056FD10BD000007
:100A500070B5044620688168C1F3400507F0CCFA00
:100A600078B375BB2068816801F00D01012909D0B8
:100A7000606D40F010006065A06D40F00100A06561
:100A8000012070BD8168124A1140891C8160216873
:100A90000320086003F064FD054613E003F060FDE9
:100AA000401B02280ED920688068C0070AD0606DFC
:100AB00040F010006065A06D40F00100A0650120CD
:100AC00070BD03E020688068C007E7D10020F7E729
:100AD000C0FFFF7F70B50446206807F08DFA50BB59
:100AE00020688168264A114209D0606D40F01000EC
:100AF0006065A06D40F00100A065012070BD8168B7
:100B00001F4E7F3E3140491C816003F029FD0546A0
:100B10001C4920681C4B884201D0984201D11B4AD5
:100B200000E01B4A926802F01F02984200D0014682
:100B300081421DD0E2B120E007F05EFA20B92068C2
:100B400081683140491C816003F00AFD401B022886
:100B50000ED920680068C043C00709D0606D40F01E
:100B600010006065A06D40F00100A065012070BD1F
:100B700020680168C943C907DED1002070BD0000AC
:100B80003F0000800020024000210240002302407C
:100B900000630258014802F0ABBB0000B0EA002439
:100BA000FEE7000010B5B2B03D4CB0F5966F4AD0EC
:100BB00008DC96281CD0B0F5167F27D0B0F5487F0A
:100BC00007D132E0A0F5A060DC384BD0B0F5FA7F59
:100BD00056D0C422334901A8FFF70AFD6220607194
:100BE0002F48C42201A91830FFF7BDFC32B010BD58
:100BF000C4222D4901A8FFF7FBFC2948C42201A902
:100C00001830FFF7B0FC24206071EFE7C4222649BA
:100C1000C43101A8FFF7ECFC3C2060712048C422DD
:100C200001A91830FFF79FFCE0E7C4221F4901A883
:100C3000FFF7DEFC402060711948C42201A918307A
:100C4000FFF791FCD2E7C4221849C43101A8FFF78D
:100C5000CFFC442060711248C42201A91830FFF76C
:100C600082FCC3E7C422124901A8FFF7C1FC4E2051
:100C700060710B48C42201A91830FFF774FCB5E776
:100C8000C4220849C43901A8FFF7B2FC582060719A
:100C90000348C42201A91830FFF765FCA6E700004D
:100CA0000800002420E6000888E1000810E300089E
:100CB00098E4000870B54FF48051454C4D108E10EB
:100CC000082805D2DFE800F0041424344454647486
:100CD0000022204603F036FC00222946204603F07D
:100CE00031FC31462046BDE87040002203F02ABCAA
:100CF0000122204603F026FC00222946204603F06C
:100D000021FC31462046BDE87040002203F01ABCA9
:100D10000022204603F016FC01222946204603F05B
:100D200011FC31462046BDE87040002203F00ABCA9
:100D30000122204603F006FC01222946204603F04A
:100D400001FC31462046BDE87040002203F0FABBAA
:100D50000022204603F0F6FB00222946204603F03D
:100D6000F1FB31462046BDE87040012203F0EABBAA
:100D70000122204603F0E6FB00222946204603F02C
:100D8000E1FB31462046BDE87040012203F0DABBAA
:100D90000022204603F0D6FB01222946204603F01C
:100DA000D1FB31462046BDE87040012203F0CABBAA
:100DB0000122204603F0C6FB01222946204603F00B
:100DC000C1FB31462046BDE87040012203F0BABBAA
:100DD0000018025870B58EB0044600250A950B9590
:100DE0000C950D950795089509951C216846FFF708
:100DF0005BFC30484FF08041016064B12E49052C06
:100E00000FD242F210726243B1FBF2F1491E41600F
:100E10006321C1600EE02748002106F0FFFC0EB000
:100E200070BD4FF47A726243B1FBF2F1491E41602A
:100E30000921C16085600561802686611D4806F034
:100E40009BF908B100F09FFF4FF480500A901948B9
:100E50000AA906F033FA08B100F095FF154806F02C
:100E60001FFC08B100F08FFF20200790099607A90A
:100E7000104806F031F908B100F085FF052C02D2C8
:100E80003220019001E00520019060200090029541
:100E9000049500220748694606F067FB08B100F098
:100EA00072FF044806F038FB0248002106F022FCDD
:100EB000B5E7000074030024001C4E0E054A1178AB
:100EC0000844C0B27921B0FBF1F301FB13001070AC
:100ED00070470000000000242DE9F04F9FB0E74864
:100EE0004FF0FF3100680BF0FFF8DFF894B33221C8
:100EF000E3481830FFF7D8FBE148183000F0DAF982
:100F0000E049486000287DD0DD48183081780C2900
:100F10001BD2DFE801F01A061B212A2E323984A9E0
:100F2000F3F2D94C00228021204603F00BFB322043
:100F30000BF09CF801222046802103F003FB0020E7
:100F40008BF8040001208BF80C008EE100208BF858
:100F500004008BF80C0088E18179407941EA002097
:100F6000ABF80000FFF71EFE7FE140798BF802002E
:100F70007BE140798BF8030077E101208BF80D00CD
:100F800000208BF8040070E19BF804006428DCD199
:100F9000BB484025BD4B0122072100954A3000F097
:100FA00013FFC4B2BA4F012238461602314603F08D
:100FB000C9FAB3494FF0FF38B64843464A31224692
:100FC00006F0B8FFB34806F037FD2128FAD03220EA
:100FD0000BF04CF8AD4BFF22A94807214033009598
:100FE0004A3000F0F1FEC2B2A549AA4843464A3150
:100FF00006F0A0FFA74806F01FFD2128FAD0002226
:10100000314600E036E1384603F09CFA64200BF0EC
:101010002DF8A14980229F4806F082FC25E101209D
:1010200000909748FF2208214A300BF1040300F09A
:10103000CBFEC4B2964E012230461502294603F07B
:1010400081FA8F494FF0FF33924822464A3106F029
:1010500071FF904806F0F0FC2128FAD000222946C2
:10106000304603F06FFA00E19BF8040064288AD14F
:101070009BF8038000210020884A32F810302BB101
:10108000491CC9B2401CC0B26228F6D308FB01F06B
:101090004FEA80094FF0010A00258BE0A9EB05001B
:1010A000782800D97820C7B20026AC0878480122F9
:1010B000110203F047FA734880780AF0D7FF002244
:1010C00057E0B4FBF8F008FB1040C0B2B4FBF8F1F5
:1010D000C9B29FED730A8DED000A08280FD200EB0C
:1010E000001303EB40106F4B03EB401000EB81004B
:1010F00090ED000A8DED000A33E092E06CE01028DC
:101100000ED2083800EB001303EB4010664B03EBE4
:10111000401000EB810090ED000A8DED000A20E008
:1011200018280ED2103800EB001303EB40105F4B71
:1011300003EB401000EB810090ED000A8DED000AFA
:101140000FE020280DD2183800EB001303EB4010FD
:10115000574B03EB401000EB810090ED000A8DED42
:10116000000A01A8009930440160361D641C521C1D
:10117000D2B2B2EB970FA4D33D444D4501D3FF2229
:1011800000E052463E48092100974A3001AB00F08A
:101190001BFEC2B23A493F484FF0FF334A3106F0D6
:1011A000C9FE3C4806F048FC2128FAD00AF1010AA1
:1011B0000AF0FF0A4D45FFF471AF354800224FF4A5
:1011C000807103F0BFF964200AF050FF3249802299
:1011D000304806F0A5FB48E0294B0420012200908E
:1011E00010330A2103F13A0000F0EEFDC4B2284E9C
:1011F000012230461502294603F0A4F920494FF098
:10120000FF33244822464A3106F094FE214806F076
:1012100013FC2128FAD000222946304603F092F927
:1012200023E0174B04200122009014330B2103F11B
:10123000360000F0C9FDC4B2154E01223046150239
:10124000294603F07FF90E494FF0FF33114822463B
:101250004A3106F06FFE0F4806F0EEFB2128FAD067
:1012600000222946304603F06DF906484068002800
:101270007FF43DAE1FB0BDE8F08F000014000024E5
:10128000F8010024000000240020025830EA002465
:10129000000002580C0400249025002420000024A3
:1012A000000000001026002410570024108800249D
:1012B00010B900242DE9F04107462D4E42E00020F0
:1012C000BDE8F081307800F06BF8AA2806D13078BC
:1012D000401CC0B200F064F8552803D00120FFF78D
:1012E000EDFD2FE03078C01CC0B200F059F8044684
:1012F00000F040F8A04201D20020E1E700250023E1
:10130000A4F1020808E030781844C0B200F048F8B0
:10131000284485B25B1CDBB24345F4DB30782044C3
:10132000401EC0B200F03CF8034630782044801ED6
:10133000C0B200F035F843EA0020A84207D00120EF
:10134000FFF7BCFD00F016F80428BBD2B7E7002376
:1013500007E030781844C0B200F022F8F8545B1C63
:10136000DBB2A342F5D32046FFF7A8FD2046A7E74E
:1013700000000024054841780078081A7930792166
:1013800090FBF1F201FB1200C0B270470000002494
:1013900000B5FFF7EFFFC0F17900C0B200BD00005B
:1013A0007921B0FBF1F201FB12000149085C7047A2
:1013B0007C0100242DE9F04180460C46FFF7E8FF50
:1013C000A04202D20020BDE8F081104E1048717892
:1013D0000A19792A08D2084422464146FFF7C3F881
:1013E0007078204470700FE0C1F17902D5B20844E2
:1013F0002A464146FFF7B7F8621B054808EB05018E
:101400001746FFF7B0F87770E0B2DCE70000002481
:101410007C0100242DED048B84B09FEDFE8AFE4DEF
:101420004FF0FF3128690AF05FFEFC48007B00287E
:101430007ED0FA48002404714FF4005007F06CFD90
:10144000F748002106F056F9F54800214C3006F027
:10145000E5F9F348B03801F04DFBF1484FF4205264
:10146000F049B03801F0C0FA0020FFF723FC05F185
:1014700018000088FFF7AEFC4FF47A700AF0F6FD12
:10148000022007F0A1FDAC70EC700021E4484C3064
:1014900006F030F95BE1E14D2A7B002A7DD000EEB9
:1014A000100AB8EE401B9FEDE02B82EE010B01EE1F
:1014B000104AB8EE411B20EE010BBCEEC00B10EE43
:1014C000100A28710A200AF0D1FD0026D348017BBA
:1014D00000297CD00025D148007B002878D05A2CE8
:1014E00004D34FF4FA600AF0C1FD02E0C8200AF00C
:1014F000BDFDC94F4FF0000887F8008001207870CB
:101500001E200AF0B3FD38780028F9D0C448002125
:101510004C3006F083F9C248B03801F0EBFAC0480D
:101520004FF42052BF49B03801F05EFA022D00E0BE
:10153000BDE109D2E81CC0B207F046FDB848002161
:101540004C3006F0D7F824E0072E08D1612C06D2E3
:10155000B148611C183030F81100FFF73BFC701CDB
:10156000C0B2FFF7A7FB022007F02EFD87F802802C
:1015700087F803805A2C07D34FF4006007F0CCFCA7
:1015800040F2DC500AF072FDA54800214C3006F014
:10159000B1F80020DFF898A200E0DDE0DFF894B2B7
:1015A0004FF4805200EB8001C91C3AF821102BF84F
:1015B0001010401C9042F5DB9E484FF480510AF019
:1015C000E7FCB7EEC09AAF1C00EE107A01E0BCE079
:1015D000B6E0B8EE401BB2EE040B09F0EDFF89EE69
:1015E000001B06EB061000EB4618934805EB0511AF
:1015F00001EB451900EB481000EBC90000EB84003B
:10160000B7EEC10B80ED000AB5EEC00AF1EE10FA9C
:1016100001D280ED008A00204FF4805100EB80025F
:10162000D21C5AF82220120C2BF81020401C8842A1
:10163000F4DB80484FF480510AF0AAFCB7EEC09A60
:1016400000EE107AB8EE401BB2EE040B09F0B4FFC6
:1016500089EE001B794800EB481000EBC90000EB55
:101660008400B7EEC10B80ED000AB5EEC00AF1EEC2
:1016700010FA01D280ED008A00204FF4805100EB77
:101680008002121D3AF822202BF81020401C8842BC
:10169000F5DB68484FF480510AF07AFCB7EEC09A47
:1016A00000EE107AB8EE401BB2EE040B09F084FF96
:1016B00089EE001B624800EB481000EBC90000EB0C
:1016C0008400B7EEC10B80ED000AB5EEC00AF1EE62
:1016D00010FA01D280ED008A00204FF4805100EB17
:1016E0008002121D5AF82220120C2BF81020401CE8
:1016F0008842F4DB4F480AF04BFCB7EEC09A00EE8C
:10170000107AB8EE401BB2EE040B09F055FF89EEDB
:10171000001B4C4800EB481000EBC90000EB8400B4
:10172000B7EEC10B80ED000AB5EEC00AF1EE10FA7B
:1017300001D280ED008A6D1CEDB2032DFFF4CBAE1B
:10174000761CF6B2082EFFF4C1AE641CE4B2324936
:1017500048798442FFF49FAE002485E00025DFF83D
:10176000D880DFF8D890DFF8D8A0DFF8D8B005EB44
:10177000051000EB451608EB461000EB840797EDCB
:10178000000A8DED000A97ED620A8DED010A97EDD2
:10179000C40A8DED020A0321684600F0F7FA87EDCE
:1017A000000A09EB461000EB840797ED000A8DED67
:1017B000000A97ED620A8DED010A97EDC40A8DEDDE
:1017C000020A0321684600F0E1FA87ED000A0AEBFD
:1017D000461000EB840797ED000A8DED000A97EDA7
:1017E000620A8DED010A97EDC40A8DED020A03210C
:1017F000684600F0CBFA87ED000A0BEB461000EBD1
:10180000840696ED000A8DED000A96ED620A8DEDD4
:10181000010A19E00000000008000024F80100247B
:10182000740300240010003800000000000059403C
:1018300000000524900500241026002410570024E1
:101840001088002410B9002496EDC40A8DED020A18
:101850000321684600F09AFA86ED000A6D1CEDB28D
:10186000082D84D3641CE4B2184840798442FFF404
:1018700075AF1748002105F0D1FF1548FC3801F07D
:1018800039F9144C00228021204602F05BFE40F220
:10189000DC500AF0EBFB01222046802102F052FED0
:1018A0000D48017B69B164210171002101730A4C6B
:1018B000607B00283FF4B3AD06F0AEFB0020607300
:1018C000ADE5002101710173F1E70000080000247B
:1018D000C003002400200258F8010024014801F050
:1018E00007BD0000A0040024014801F0B9B90000C0
:1018F000B0EA002410B52C4A016891423AD02A4A35
:101900001832914236D0284A3032914232D0264A9B
:10191000483291422ED0244A603291422AD0224A43
:101920007832914226D0204A9032914222D01E4AEB
:10193000A83291421ED01D4A91421BD01B4A183238
:10194000914217D0194A3032914213D0174A483287
:1019500091420FD0154A603291420BD0134A78322F
:10196000914207D0114A9032914203D00F4AA832D7
:10197000914214D1CAB2103A1823B2FBF3F20C4CC4
:1019800002F00703E35CC365032A04D96FF309017E
:10199000091D816506E06FF30901816502E021F010
:1019A000FF018165806D10BD1000024010040240EF
:1019B000F4E6000810B501680123224CCAB2A14226
:1019C0001BD0204C1434A14217D01E4C2834A14205
:1019D00013D01C4C3C34A1420FD01A4C5034A142BD
:1019E0000BD0184C6434A14207D0164C7834A14275
:1019F00003D0144C8C34A1420FD1083A1421B2FB0D
:101A0000F1F1114A02EB810202660F4A803242660E
:101A100001F01F018B40836610BD103A1824B2FB01
:101A2000F4F20A4C2144A82900D80832084901EBF5
:101A30008201016606498031416602F01F018B4038
:101A4000836610BD0854025800580258F0FBFDBFD1
:101A5000000802400279521E072A31D8194B01684A
:101A600099421BD0174B1433994217D0154B28338A
:101A7000994213D0134B3C3399420FD0114B503342
:101A800099420BD00F4B6433994207D00D4B7833FA
:101A9000994203D00B4B8C33994207D10A4901EB91
:101AA0008201C16608494031016706E0074901EB40
:101AB0008201C166054940310167012191404167BA
:101AC00070470000085402580059025800090240AB
:101AD000014610B500208B694FF0C0748A6A002B54
:101AE0000ED0B3F5005F1AD062B3012A2AD0022AC1
:101AF00028D0032A03D1C96AC90100D5012010BD2D
:101B00001AB1012A06D0022AF9D1C96AC901F6D54B
:101B1000012010BDC96AA142FBD1012010BD52B104
:101B2000012A0AD0022A06D0032AF7D1C96AA142A3
:101B3000F4D1012010BD012010BDC96AC901FBD537
:101B4000012010BD012010BD2DE9F04F856D8A4E9A
:101B5000894FDFF824C2A836DFF81C82DFF818921C
:101B60000CF1180CDFF810A208F13008DFF808B209
:101B700009F1480904680AF1600A0BF1780BBC42CC
:101B80006DD064456BD0444569D04C4567D0544511
:101B900065D05C4563D0DFF8E0E10EF1900E74454E
:101BA0005DD0B4425BD0DFF8D4E1744557D0DFF8A4
:101BB000CCE10EF1180E744551D0DFF8C0E10EF102
:101BC000300E74454BD0DFF8B4E10EF1480E744589
:101BD00045D0DFF8A8E10EF1600E74453FD0DFF884
:101BE0009CE10EF1780E744539D0DFF890E10EF1EA
:101BF000900E744533D0DFF884E10EF1A80E7445E1
:101C00002DD0DFF87CE1744529D0DFF874E10EF1C6
:101C1000140E744523D0DFF868E10EF1280E7445E8
:101C20001DD0DFF85CE10EF13C0E744517D0DFF8F3
:101C300050E10EF1500E744511D0DFF844E10EF181
:101C4000640E74450BD0DFF838E10EF1780E744560
:101C500005D0DFF82CE10EF18C0E744509D1D0E9E6
:101C600019E4CEF80440C46E1CB1D0E91CE4CEF8EF
:101C700004400468BC422ED064452CD044452AD090
:101C80004C4528D0544526D05C4524D03A4F903757
:101C9000BC4220D0B4421ED0384EB4421BD0374E86
:101CA0001836B44217D0354E3036B44213D0334EC6
:101CB0004836B4420FD0314E6036B4420BD02F4E6E
:101CC0007836B44207D02D4E9036B44203D02B4E16
:101CD000A836B4421BD190F85C4004F01F063F24A4
:101CE000B440AC600468256825F48025256004684C
:101CF00063608368402B05D0036899600068C26008
:101D0000BDE8F08F03689A600068C160F8E71C4E78
:101D1000B4421BD01A4E1436B44217D0184E28368F
:101D2000B44213D0164E3C36B4420FD0144E503647
:101D3000B4420BD0124E6436B44207D0104E7836FF
:101D4000B44203D00E4E8C36B442D9D190F85C40E8
:101D500004F01F060124B4406C600468636083686B
:101D6000402B04D0036899600068C260C8E703682C
:101D70009A600068C160C3E710000240100402408E
:101D800008540258704772B6FEE7000090ED000A52
:101D900001220CE000EB8203D3ED000AF4EEC00A4E
:101DA000F1EE10FA01DDB0EE600A521C92B28A42E6
:101DB000F0D310EE101A034A914201DA90ED020AB4
:101DC00070470000CDCC4C3D2DE9F04704468846D5
:101DD00091461E46089F002580212046FEF742FCC2
:101DE000AA2020705520607084F802800020E070E6
:101DF00084F8049007200021625C2A4495B2491CB3
:101E0000C9B20529F8D3002109E06318725C5A7140
:101E1000725C2A4495B2401CC0B2491CC9B2B94296
:101E2000F3D3E07029180B0A221802F8023D517012
:101E3000BDE8F087F8B504460E4617460025009524
:101E400094F85000012810D0012084F8500020465A
:101E5000FEF7FEFD0346180009D0606D40F010004B
:101E6000606584F850501846F8BD0220F8BD606DDA
:101E700020F4885040F002006065206806F480314C
:101E800007F0804211438268114E3240114341F005
:101E9000004181600F4920680FE0009A521C0092B7
:101EA000009A8A4209D3606D20F0020040F01000D1
:101EB000606584F850500120F8BD8268D20F002A76
:101EC000EBD1606D20F0020040F001006065C8E7D2
:101ED000C0FFFE3F00F8C3252DE9FC5F04460D4618
:101EE0004FF0000800200190DFF8D8B3DFF8D8A346
:101EF000F64EF74F94F85000012813D04FF0010927
:101F000084F85090206806F07BF868B1606D40F06E
:101F1000200060654FF00108002084F85000404622
:101F2000BDE8FC9F0220FBE7286800280DDB216844
:101F3000CA69030329D090FAA0F0B0FA80F000F04B
:101F40001F0009FA00F00243CA61A98820682A68C4
:101F500001F4407300EB9310036B01F01F014FF08D
:101F60001F0CC2F384620CFA01FC8A4023EA0C03C2
:101F700013430363206806F043F80090206806F0DE
:101F800037F80099014303D094E0C0F38460D6E7AA
:101F90002168AA68286800F0007301EBD3514B69EF
:101FA0004FF0070CC0F304500CFA00FC824023EA07
:101FB0000C0313434B61C7480068B9EB107F07D18E
:101FC00021686869C968C1F382014900884010E04E
:101FD0002168C868C00606D46869C968C1F382016F
:101FE0004900884005E06869C96801F010014908A6
:101FF0008840296904292DD023682A6803EB8101D0
:102000000B6E02F0F842024303F0004313430B66E9
:10201000697E20682A69012916D0002100EB820020
:10202000026E22F000420A430266297E20682A6975
:1020300001290CD00021036902F01F0223F4F043B0
:1020400091400B43036135E04FF00041E6E74FF468
:102050000061F0E72068016E2A7801F0F841B1EBE9
:10206000826F03D1016E21F0004101662068416E4C
:102070002A7801F0F841B1EB826F03D1416E21F073
:10208000004141662068816E2A7801F0F841B1EB89
:10209000826F03D1816E21F0004181662068C16E9C
:1020A0002A7801F0F841B1EB826F03D1C16E21F0C3
:1020B0000041C166206805F09FFF00287FF42CAF27
:1020C00020682A7B296850F8C03FC1F3130C23EA2B
:1020D0000C0302F0180C804A22FA0CF20A40134357
:1020E0000360E868584570D12168DFF8F0B1DFF887
:1020F000F0C15145DFF8ECE17B4A7C4B37D12868D1
:10210000584501D1012269E0A0F1066BBBF1040B37
:102110000FD0A0F1496CBCF1080C0CD0A0F1865C8A
:10212000BCF1100C09D0DFF8C8C1604507D1714A75
:1021300054E0624652E0724650E06F4A4EE0DFF8EB
:10214000BCC160454AD0904201D11A4646E098424F
:1021500001D16B4A42E06B4A904201D16A4A3DE0AC
:102160006A4A904201D16A4A38E0002236E0B14220
:1021700033D12868584501D101222FE0A0F1066B28
:10218000BBF1040B0FD0A0F1496CBCF1080C0CD0D2
:10219000A0F1865CBCF1100C09D0DFF854C1604599
:1021A00007D1544A1AE0624618E0724616E0524AD5
:1021B00014E0DFF848C1604510D0904201D11A46C2
:1021C0000CE0984202D14E4A08E015E04F4A904296
:1021D00001D14F4A02E0002200E00022CB69100347
:1021E00018D092FAA2F0B0FA80F000F01F0009FABD
:1021F00000F943EA0903CB612A68002ABFF68CAED6
:102200002068444BDFF810C1504501D0B04204D1E2
:10221000194603E0C2F38460E7E76146896801F08C
:10222000E071504501D0B0420AD1DAF80850C5F348
:102230000005D6F80890C9F3000945EA090502E04F
:10224000BD68C5F3000535B1606D40F020006065E4
:102250004FF0010860E6314DAA421FD10D021DD496
:10226000B842F7D1504502D0B04200D0634641F4A5
:102270000000996821F0E0710143996028482949DC
:102280000068B0FBF1F0401C4000019002E00198B2
:10229000401E019001980028F9D13DE6224DAA4246
:1022A00044D1CD0142D4B842D4D1504502D0B0423D
:1022B00000D0634641F08070996821F0E0710143DD
:1022C000996029E60000FF470020024000210240FB
:1022D000006002580010005CFFFF0F000200300495
:1022E000400020198000501D0008302E0010603280
:1022F0002000F0140002B025000180210004002A13
:102300000020903600002143000052470000844B1B
:102310000000B84F0023024000630258000084CB45
:10232000E4000024400D0300000052C7094DAA42FA
:1023300090D14A028ED4B8428CD1504502D0B042DE
:1023400000D0634641F48000996821F0E0710143B8
:102350009960E1E50000B8CF2DE9F05F5E49022207
:102360005E4F5E4CDFF874B1AC3FC96C603C5C4EB4
:10237000A7F104085B4D0968594501D9326011E0A5
:10238000A14201D93A600DE0564BB833994202D9C7
:10239000C8F8002006E0534B5833994201D9EA604F
:1023A00000E0AA604FF00009DFF83CA19AF80110A4
:1023B00000296ED000684D4988427FD19AF8030009
:1023C00004287DD29AF80210814277D9484801F05A
:1023D00063FB08B1FFF7D7FC9AF803004FF42053D2
:1023E000444900EB800001EB003241484FF03821B6
:1023F00001F050FD3E483A4BDFF8E0C0394A1B1F60
:10240000DFF8E0E0ACF1B80C0068B8320EF1580E1D
:10241000584503D9196801F0200117E0A04205D9F9
:102420002E49B439096801F020010FE0904204D927
:10243000DCF8001001F0200108E0704503D969685C
:1024400001F0200102E0296801F020010029DFD01D
:102450001021584501D931600DE0A04201D9396001
:1024600009E0904202D9C8F8001004E0704501D993
:10247000E96000E0A9602021584501D9316010E0F1
:10248000A04201D939600CE0904205D9C8F800108B
:1024900007E01EE012E013E0704501D9E96000E0BA
:1024A000A9609AF80300401CC0B28AF8030004280F
:1024B00004D101208AF800008AF80190BDE8F09F5D
:1024C00004208AF8030001208AF800008AF80190AD
:1024D000F4E78AF80390F1E7C4020024B80402404C
:1024E0000454025800000240080000240060025812
:1024F00018050024002805242DE9F05F5149042225
:10250000514F514C524DAC3FC96C603CDFF838A183
:10251000B83D4E4EA7F10408DFF834B109685145C3
:1025200001D932600FE0A14201D93A600BE0594570
:1025300002D9C8F8002006E0454B603B994201D91A
:10254000EA6000E0AA60DFF80C9199F8011091B3FD
:102550000068414988426CD199F8020004286AD287
:102560003E4801F099FA08B1FFF70DFC99F8020016
:102570004FF420533A4900EB800001EB0032394917
:10258000364801F087FC3548304A2F4BDFF8C0E071
:10259000121F0068B43BA3F1040CAEF1600E50456D
:1025A00003D9116801F0100116E0A04204D919689E
:1025B00001F0100110E041E0584504D9DCF80010AA
:1025C00001F0100108E0704503D9696801F01001BD
:1025D00002E0296801F010010029E0D010215045E7
:1025E00001D931600DE0A04201D9396009E05845B8
:1025F00002D9C8F8001004E0704501D9E96000E094
:10260000A9602021504501D931600DE0A04201D9D7
:10261000396009E0584502D9C8F8001004E0704557
:1026200001D9E96000E0A96099F80200401C89F82E
:102630000200BDE8F09F89F80220FAE7002089F83F
:102640000200F6E7C4020024B80402400454025811
:10265000B800024008000024006002581805002459
:10266000000005240010003870470000F8B504464B
:10267000002500260096002C02D0606D10B107E006
:102680000120F8BD204600F007F9A66584F85060E7
:1026900020688168C1F3407119B18168734A1140A3
:1026A000816020688168C1F3007199B98168704ABE
:1026B000114041F0805181606E486F490068B0FB65
:1026C000F1F0401C009002E00098401E009000983D
:1026D0000028F9D120688168C1F3007141B9616DAA
:1026E00041F010016165A16D41F00101A165012575
:1026F00005F086FC616DC90600D430B1606D40F014
:102700001000606501252846F8BD606D20F48070DA
:1027100040F002006065206805F06EFC00BB574A7F
:102720002068574B904201D0984207D19168C1F37D
:1027300000019E68C6F30006314303E051498968F1
:10274000C1F3000161B9904201D0984201D14E48D5
:1027500000E04E486168826822F47C120A4382607D
:1027600001F0F8FE41F20301884202D9A068102866
:102770000CD0A168206B227F0843617D490341EAA8
:1027800002410843217F01290CD00FE0617D227FA7
:10279000206B490340F0100041EA0241084340F039
:1027A0000C00EFE7218C491E40EA4140616A29B1E3
:1027B000A26A01F47871014342EA01002168CA6803
:1027C000334B1A400243CA60206805F019FC0646E4
:1027D000206805F00DFC06431DD1217DE06A40EA2A
:1027E00081312068C26844F203039A430A43C260FD
:1027F00094F8380001281DD02068016921F00101FA
:10280000016120680169626B21F07041114301612F
:102810002046FDF7BDFFE06801281DD02068016B50
:1028200021F00F010163606D20F0020040F0010013
:10283000606568E7A28F0123D4E91010521E01439E
:10284000A06C03EB02421043014320680269114B64
:102850001A4011430161D4E72068016BA26921F09D
:102860000F01521E11430163DDE70000C0FFFF5F4F
:10287000C0FFFF7FE4000024400D03000020024061
:102880000021024000600258002302400063025809
:1028900003C0F0FF1EF800FC70B5BCB00646142162
:1028A00036A8FDF701FFC02102A8FDF7FDFE47494C
:1028B000306888427ED100204FF40021CDE902101B
:1028C00005200490902005900A2006900220079091
:1028D00008908020099000250A950B952B9502A859
:1028E00003F0D6F808B1FFF74EFA3948016841F015
:1028F00080710160016801F080710191016841F00F
:1029000020010160016801F020010191016841F09E
:1029100004010160016801F004010191016841F0C6
:1029200080010160006800F080000190082036906E
:1029300003243794389536A9264801F0F1FC3694E3
:102940003794389536A9244801F0EAFC3C203690AB
:102950003794389536A9214801F0E2FC4FF08060A9
:10296000014604F067FB4FF00060014604F062FB93
:102970001C4C1B48206011206060A560E5604FF48E
:1029800080602061400060618000A0614011E061D2
:102990002562204601F080F808B1FFF7F4F90E2017
:1029A000329033958DF8D05001208DF8D1003590BC
:1029B00032A900E007E00B4800F0DCF808B1FFF7AF
:1029C000E2F9F464A6633CB070BD000000600258F8
:1029D000E04402580014025800080258001C025833
:1029E00008540258B0EA00242DE9F047044689460D
:1029F0009246384FDFF8E0802068B84201D0404569
:102A000001D1364900E03649896801F01F0505F01B
:102A1000F7FA10B10220BDE8F08794F850000128C1
:102A20000BD0012084F85000002645B1052D06D0BA
:102A3000092D04D084F85060EDE70220EBE7204632
:102A4000FEF748F810B184F85060E4E7606D40F696
:102A50000161884340F4807060652068404500D083
:102A60000746874200D01DB9606D20F48010606574
:102A7000606DC00404D5A06D20F00600A06500E0E4
:102A8000A665E16C1748C863E16C17480864E16CFF
:102A90001648C8641C202168086084F850602068CB
:102AA000416841F010014160E16A2068C26822F08B
:102AB00003020A43C26021685346E06C4A46403133
:102AC00001F0B8FA21688A68094B1A40121D8A6021
:102AD000A1E7000000200240002102400023024044
:102AE00000630258AD090008450A00082B0A0008D7
:102AF000C0FFFF7F70B5044694F85000012809D04C
:102B0000012084F8500003212046FDF7D5FE05463C
:102B100015B129E0022070BD2068C16821F00301D1
:102B2000C160E06C90F83510022907D100F0CAF8B6
:102B300005461DB1606D40F0400060652068416849
:102B400021F01001416025B12046FDF781FF2DB134
:102B50000AE02046FDF77CFF0546F8E7606D20F4AB
:102B6000885040F001006065002084F8500028463D
:102B700070BD000030B5002200230C7A012C3ED13C
:102B8000354B02689A4238D0334B18339A4234D0CE
:102B9000314B30339A4230D02F4B48339A422CD0AD
:102BA0002D4B60339A4228D02B4B78339A4224D055
:102BB000294B90339A4220D0274BA8339A421CD0FD
:102BC000264B9A4219D0254B18339A4215D0234BE5
:102BD00030339A4211D0214B48339A420DD01F4BCB
:102BE00060339A4209D01D4B78339A4205D01B4B73
:102BF00090339A4201D0194BA8330A684B6890F879
:102C00003540012C04D04FF400614165012030BDF6
:102C100090F83440012C1CD0012400F8344FC46AD1
:102C2000256825F48135256014068A89521E44EAF8
:102C3000C2421A430B7A497A42EA034242EA4122EB
:102C4000C16A0B68DBB21A430A60002101700020E0
:102C500030BD022030BD00001000024010040240D0
:102C600010B50446606E0068A16E08420FD0206E59
:102C7000016821F480710160D4E919104860606D29
:102C800040F400706065E16C09B120468847E06E51
:102C9000002816D0216F0968626F114211D00168B7
:102CA00021F480710160D4E91C104860606D40F42B
:102CB00080606065E16C002903D02046BDE81040CB
:102CC000084710BD2DE9F84F044601F049FC00907B
:102CD0005CB194F83500022809D08020606500209E
:102CE00084F834000120BDE8F88F0120FBE7D14EC5
:102CF000D04FD0491836DFF83C833037DFF83493B3
:102D0000DFF830A308F14808DFF828B309F16009BB
:102D100020680AF1780A0BF1900B88422ED0B0425D
:102D20002CD0B8422AD0404528D0484526D050451E
:102D300024D0584522D0BF4AA83290421ED0BE4A65
:102D400090421BD0BC4A1832904217D0BA4A303257
:102D5000904213D0B84A483290420FD0B64A6032FF
:102D600090420BD0B44A7832904207D0B24A9032A7
:102D7000904203D0B04AA83290420AD1026822F0B1
:102D80001E0202602068426922F0800242612568CA
:102D900004E0026822F00E02026025682068884282
:102DA0004DD0B0424BD0B84249D0404547D04845BD
:102DB00045D0504543D0584541D09E4AA832904214
:102DC0003DD09D4A90423AD09B4A1832904236D02C
:102DD000994A3032904232D0974A483290422ED0AF
:102DE000954A603290422AD0934A7832904226D057
:102DF000914A9032904222D08F4AA83290421ED0FF
:102E00008E4A90421BD08D4A1432904217D08B4A82
:102E10002832904213D0894A3C3290420FD0874AE0
:102E2000503290420BD0854A6432904207D0834A98
:102E30007832904203D0814A8C32904204D1206E85
:102E4000026822F4807202607A49206888422ED09B
:102E5000B0422CD0B8422AD0404528D0484526D090
:102E6000504524D0584522D07249A83188421ED0FE
:102E7000714988421BD070491831884217D06E4979
:102E80003031884213D06C49483188420FD06A49AA
:102E9000603188420BD068497831884207D0664952
:102EA0009031884203D06449A831884204D1016836
:102EB00021F00101016013E0016821F001010160CE
:102EC0000EE001F04DFB0099401A052808D920209A
:102ED000343420620320607000202070012002E75B
:102EE0002868C007EDD1534A0121206890422ED0B6
:102EF000B0422CD0B8422AD0404528D0484526D0F0
:102F0000504524D0584522D04A4BA83398421ED071
:102F1000494B98421BD0484B1833984217D0464B28
:102F20003033984213D0444B483398420FD0424B31
:102F3000603398420BD0404B7833984207D03E4BD9
:102F40009033984203D03C4BA833984208D1A06DEF
:102F500094F85C3003F01F053F23AB40836007E02B
:102F6000A06D94F85C3003F01F0301FA03F3436093
:102F7000206890424DD0B0424BD0B84249D0404535
:102F800047D0484545D0504543D0584541D0294ABF
:102F9000A83290423DD0284A90423AD0264A183270
:102FA000904236D0244A3032904232D0224A4832BF
:102FB00090422ED0204A603290422AD01E4A783267
:102FC000904226D01C4A9032904222D01A4AA8320F
:102FD00090421ED0194A90421BD0184A1432904297
:102FE00017D0164A2832904213D0144A3C329042ED
:102FF0000FD0124A503290420BD0104A64329042A5
:1030000007D00E4A7832904203D00C4A8C3290425C
:103010000BD1D4E919205060E06E30B1026822F47F
:1030200080720260D4E91C2050603434617000204A
:10303000207058E610000240100402400854025864
:103040002DE9F05F002808D090F83510022906D04D
:10305000802141650120BDE8F09F0120FBE7A14AE6
:10306000A04BA04C18329F4D30339E4E4834DFF8B1
:1030700074B26035DFF870C27836DFF86C82DFF842
:1030800068920CF1300CDFF860A208F1600801686A
:1030900009F17809944F0AF1900A594531D09142CB
:1030A0002FD099422DD0A1422BD0A94229D0B14294
:1030B00027D0DFF830E20EF1900E714521D0DFF815
:1030C00024E20EF1A80E71451BD0DFF81CE2AEF130
:1030D000180E714515D0B94213D0DFF80CE20EF18D
:1030E000180E71450DD061450BD0DFF8FCE10EF1F3
:1030F000480E714505D0414503D0494501D05145A1
:1031000037D14FF0040E80F835E0594527D0914271
:1031100025D0994223D0A14221D0A9421FD0B1424B
:103120001DD070489030814219D06E48A83081423D
:1031300015D06D481838814211D0B9420FD06A4875
:10314000183081420BD0614509D067484830814230
:1031500005D0414503D0494501D0514504D1086807
:1031600020F001000860BAE0086820F00100086063
:10317000B5E0D1F800E02EF00E0EC1F800E00168D5
:10318000DE46594531D091422FD099422DD0A142EF
:103190002BD0A94229D0B14227D0DFF848B10BF19A
:1031A000900B594521D0DFF83CB10BF1A80B5945E4
:1031B0001BD0DFF834B1ABF1180B594515D0B9422B
:1031C00013D0DFF824B10BF1180B59450DD0614530
:1031D0000BD0DFF814B10BF1480B594505D0414530
:1031E00003D0494501D0514506D1D1F800B02BF0AC
:1031F000010BC1F800B005E0D1F800B02BF0010BD5
:10320000C1F800B001684FF0010B714546D0914202
:1032100044D0994242D0A14240D0A9423ED0B142CE
:103220003CD0304A9032914238D02E4AA832914256
:1032300034D02D4A183A914230D0B9422ED02A4A81
:10324000183291422AD0614528D0274A483291420B
:1032500024D0414522D0494520D051451ED0234A93
:1032600091421BD0214A1432914217D01F4A283272
:10327000914213D01D4A3C3291420FD01B4A50322A
:1032800091420BD0194A6432914207D0174A7832E2
:10329000914203D0154A8C32914218D1016E0A68CE
:1032A00022F480720A60816D90F85C2002F01F02A7
:1032B0000BFA02F24A60D0E919215160C16E31B1B6
:1032C0000A6822F480720A60D0E91C21516080F8FB
:1032D00035B0002180F83410016D01B1884700201D
:1032E000B9E60000100002402804024008540258C9
:1032F0002DE9FF5F0446002001904FF41651FD4870
:103300000068B0FBF1F00090A56D2E682968FA4FB7
:10331000DFF8E4B3DFF8E083DFF8DC930BF1180BA0
:10332000DFF8D4A308F13008206809F148090AF150
:10333000600AB8423BD05A46904238D0404536D019
:10334000484534D0504532D0EB4A783290422ED0A6
:10335000E94A903290422AD0E74AA832904226D0D9
:10336000E64A904223D0E54A183290421FD0E34B00
:10337000303398421BD0E14B4833984217D0DFF8E6
:103380007CC30CF1600C604511D0DFF870C30CF108
:10339000780C60450BD0DFF864C30CF1900C6045ED
:1033A00005D0DFF858E30EF1A80E70457ED194F8F1
:1033B0005C10082301F01F0103FA01F232424BD0E6
:1033C000B84232D0584530D040452ED048452CD058
:1033D00050452AD0C8497831884226D0C649903114
:1033E000884222D0C449A83188421ED0C3498842AD
:1033F0001BD0C2491831884217D0C04930318842A9
:1034000013D0BE49483188420FD0BC496031884250
:103410000BD0BA497831884207D0B84990318842F8
:1034200003D0B649A831884203D1016801F00401F4
:1034300002E0016801F0080171B1016821F00401A6
:10344000016094F85C0000F01F0003FA00F2AA602B
:10345000606D40F00100606594F85C00012100F0AF
:103460001F008140314240D02068B84234D05845D6
:1034700032D0404530D048452ED050452CD09E4AC1
:103480007832904228D09C4A9032904224D09A4A76
:10349000A832904220D0994A90421DD0974A1832C3
:1034A000904219D0954A3032904200E0D2E113D0D8
:1034B000924A483290420FD0904A603290420BD0EC
:1034C0008E4A7832904207D08C4A9032904203D094
:1034D0008A4AA83290427DD1406910F0800F04D012
:1034E000A960606D40F00200606594F85C00042102
:1034F00000F01F00814031423ED02068B84232D0F7
:10350000584530D040452ED048452CD050452AD083
:10351000794A7832904226D0774A9032904222D02F
:10352000754AA83290421ED0744A90421BD0734A0A
:103530001832904217D0714A3032904213D06F4AFD
:10354000483290420FD06D4A603290420BD06B4AA5
:103550007832904207D0694A9032904203D0674A4D
:10356000A83290424ED1006810F0020F04D0A9603A
:10357000606D40F00400606594F85C00102100F07C
:103580001F008140314260D02068B84234D0584595
:1035900032D0404530D048452ED050452CD0564AE8
:1035A0007832904228D0544A9032904224D0524AE5
:1035B000A832904220D0514A90421DD04F4A183232
:1035C000904219D04D4A3032904215D04B4A483281
:1035D000904200E014E00FD0484A603290420BD095
:1035E000464A7832904207D0444A9032904203D003
:1035F000424AA832904207D1006800F0080006E075
:10360000006872E70068B7E7006800F0040058B18E
:10361000A9602068016849030CD50068000304D440
:10362000216C09B1204688470FE0A16C69B12046A2
:1036300088470AE00168C90503D4016821F0080140
:103640000160216C09B12046884794F85C00202174
:1036500000F01F00814031427BD02068B84232D058
:10366000584530D040452ED048452CD050452AD022
:10367000214A7832904226D01F4A9032904222D07E
:103680001D4AA83290421ED01C4A90421BD01B4AB1
:103690001832904217D0194A3032904213D0174A4C
:1036A000483290420FD0154A603290420BD0134AF4
:1036B0007832904207D0114A9032904203D00F4A9C
:1036C000A832904203D1006800F0100002E00068C8
:1036D00000F00200E8B3A96094F83500042812D085
:1036E0002068016849033DD50068000335D4616C4A
:1036F00079B305E0E4000024100002401004024009
:10370000204688473FE02068016821F016010160EB
:103710002068416921F080014161206C08B9A06CEA
:1037200020B12068016821F00801016094F85C0074
:1037300000F01F013F208840A860012084F8350078
:10374000002084F83400216D002974D004B0204694
:1037500000E018E0BDE8F05F0847E16B99B1204652
:10376000884710E00168C90509D4016821F01001FB
:103770000160012084F83500002084F83400E16BFA
:1037800009B120468847606D002854D0606DC0079D
:1037900058D0042084F835002068B84231D058450C
:1037A0002FD040452DD048452BD0504529D0B74982
:1037B000884226D0B5491831884222D0B3493031E9
:1037C00088421ED0B24988421BD0B1491831884284
:1037D00017D0AF493031884213D0AD4948318842C3
:1037E0000FD0AB49603188420BD0A949783188426B
:1037F00007D0A7499031884203D0A549A831884213
:1038000004D1016821F00101016003E0016821F0A9
:103810000101016021680198009A401C01909042CA
:1038200002D80868C007F6D10868C00704D0032092
:1038300084F8350003E087E0012084F8350000209B
:1038400084F83400E16C00297ED004B02046BDE845
:10385000F05F08478F4EB0421BD08E4E1436B042F8
:1038600017D08C4E2836B04213D08A4E3C36B04228
:103870000FD0884E5036B0420BD0864E6436B042E0
:1038800007D0844E7836B04203D0824E8C36B04298
:103890005AD106684FF0040E94F85CB00BF01F0B81
:1038A0000EFA0BFE1EEA010FCDF80CE05ED05FEAC7
:1038B000467E5BD503986860300411D5F00307D4C9
:1038C000A16C002940D004B02046BDE8F05F084755
:1038D000216C002938D004B02046BDE8F05F0847CD
:1038E000B0063BD42068B8422DD068496039884280
:1038F00029D0404527D0484525D0504523D063499D
:10390000884220D06149183188421CD05F4930314B
:10391000884218D05E49884215D0904213D05C4945
:10392000303188420FD098420DD0594960318842D9
:1039300009D057497831884205D0604503D05449B1
:10394000A831884206D100E07CE0016821F008013E
:10395000016003E0016821F004010160216C00298D
:1039600070D004B02046BDE8F05F08474FF0020E6B
:103970000EFA0BFE1EEA010FCDF808E063D05FEAF5
:10398000867E60D502986860300411D5F00307D4B4
:10399000616C002978D004B02046BDE8F05F08478C
:1039A000E16B002970D004B02046BDE8F05F084705
:1039B000B0063FD42068B8422DD0344960398842DF
:1039C00029D0404527D0484525D0504523D02F4900
:1039D000884220D02D49183188421CD02B493031E3
:1039E000884218D02A49884215D0904213D02849DD
:1039F000303188420FD098420DD02549603188423D
:103A000009D023497831884205D0604503D0204948
:103A1000A831884204D1016821F01401016003E05B
:103A2000016821F00A010160012084F835000020BE
:103A300084F83400E16B002926D004B02046BDE8AC
:103A4000F05F084720E0082202FA0BF20A421BD07E
:103A5000310719D5016821F00E01016094F85C006E
:103A600000F01F01012000FA01F16960606584F82F
:103A70003500002084F83400E16C002904D004B043
:103A80002046BDE8F05F0847BDE8FF9F8800024080
:103A900010040240085402582DE9F05F044600F07B
:103AA0005FFD0646002C7DD0F44F0222DFF8CC8368
:103AB0000025DFF8C893DFF8C4A308F13008DFF869
:103AC000BCB309F1480920680AF1600A0BF1780BD0
:103AD000B84232D0E949183188422ED040452CD026
:103AE00048452AD0504528D0584526D0E349903142
:103AF000884222D0E149A83188421ED0E04988425C
:103B00001BD0DF491831884217D0DD493031884257
:103B100013D0DB49483188420FD0D94960318842FF
:103B20000BD0D7497831884207D0D54990318842A7
:103B300003D0D349A83188427ED184F8352084F857
:103B40003450B84234D0CD491831884230D0404545
:103B50002ED048452CD050452AD0584528D0C749AA
:103B60009031884224D0C549A831884220D0C44928
:103B700088421DD0C2491831884219D0C04930311D
:103B8000884215D0BE494831884211D0BC496031C5
:103B900088420DD0BA497831884209D0B84990316D
:103BA000884200E009E003D0B549A831884207D136
:103BB000016821F00101016013E00120BDE8F09FE0
:103BC000016821F0010101600BE000F0C9FC801BDD
:103BD000052806D920206065032084F835000120DF
:103BE000ECE720680068C007EFD122681168A5489B
:103BF0000140D4E902031843D4E90436334318439F
:103C0000A3691843E3691843236A18430843616AA8
:103C1000042903D1D4E90B13194308439A490968CD
:103C20006FF30F01B1F1005F11D36168A1F12903B6
:103C3000052B0AD9163B00E02EE0032B05D9083BE3
:103C4000012B02D94F39032901D840F480101060AC
:103C50002068406920F00701606A40EA01060428F4
:103C60000DD1A06A0643E06A48B12046FDF730FF57
:103C700028B140206065012084F835009EE7206867
:103C800046612046FDF736FE94F85C1001F01F02F5
:103C90003F219140816066E07C4988421BD07B4B8C
:103CA0001433984217D0794B2833984213D0774B6E
:103CB0003C3398420FD0754B503398420BD0734B26
:103CC0006433984207D0714B7833984203D06F4BDE
:103CD0008C3398427ED1884211D06C49143188428D
:103CE0000DD06A492831884209D068493C31884260
:103CF00005D066495031884201D06449643184F866
:103D0000352084F83450026861490A40A16840298E
:103D10007ED080297DD00021E36841EAD301236968
:103D200041EAD301636941EAD301A36941EAD301BE
:103D3000E36941EAD301236A41EA131111430160A7
:103D400052492068494208441421B0FBF1F0800038
:103D5000E0652046FDF7CEFD94F85C1001F01F02EF
:103D60000121914041602068B84256D04349183142
:103D7000884252D0404550D048454ED050454CD056
:103D800058454AD03D499031884246D03B49A831F8
:103D9000884242D03A4988423FD039491831884256
:103DA0003BD037493031884237D035494831884295
:103DB00033D03349603188422FD03149783188423D
:103DC0002BD02F499031884227D02D49A8318842E5
:103DD00023D000E02DE02D4988421ED02B4914311C
:103DE00088421AD029492831884216D027493C31C7
:103DF000884212D02549503188420ED0234964317F
:103E000088420AD021497831884206D01F4901E012
:103E10000AE00BE08C31884229D12046FDF7CAFD2B
:103E2000A06880280CD00CE0102175E74FF4804189
:103E300072E740206065032084F835000120BDE66C
:103E40006560216E20790860D4E9191048606068C7
:103E5000401E072808D82046FDF7FCFDE06E0560EF
:103E6000D4E91C10486002E0E56625676567656572
:103E7000012084F835000020A0E600001000024078
:103E8000100402403F8010FE0010005C08540258ED
:103E90000F00FEFF2DE9F05F04460025002C14D032
:103EA00094F83400012812D0012084F8340094F8EA
:103EB00035600020012E0CD04FF40061616584F85C
:103EC000340001252846BDE8F09F0120FBE70220D1
:103ED000F9E7022684F835606065544F534EDFF8E9
:103EE0004C811837DFF84491DFF840A108F1300821
:103EF000DFF838B109F1480920680AF1600A0BF1CE
:103F0000780BB04243D0B84241D040453FD04845FD
:103F10003DD050453BD0584539D0DFF810C10CF1A9
:103F2000900C604533D0DFF804C10CF1A80C60455B
:103F30002DD0DFF8FCC0604529D0DFF8F4C00CF1CB
:103F4000180C604523D0DFF8E8C00CF1300C604558
:103F50001DD0DFF8DCC00CF1480C604517D0DFF84D
:103F6000D0C00CF1600C604511D0DFF8C4C00CF17A
:103F7000780C60450BD0DFF8B8C00CF1900C6045B0
:103F800005D0DFF8ACC00CF1A80C604506D1D0F824
:103F900000C02CF0010CC0F800C005E0D0F800C053
:103FA0002CF0010CC0F800C02046FDF7CDFD2068C4
:103FB000B04230D0B8422ED040452CD048452AD00F
:103FC000504528D0584526D018499031884222D0F3
:103FD0001649A83188421ED0154988421BD0144981
:103FE0001831884217D012493031884213D0104915
:103FF000483188420FD00E49603188420BD00C49BD
:104000007831884207D00A499031884203D0084964
:10401000A831884204D1016841F00101016051E7F3
:10402000016841F0010101604CE70000100002400E
:10403000100402402DE9F84F044600200090002CA7
:1040400015D094F83400012813D0012084F83400EE
:1040500094F835500020012D0DD04FF400616165BA
:1040600084F83400012000900098BDE8F88F01200A
:10407000FBE70220F9E7022584F835506065A54D7D
:10408000A44EA44F1835DFF88CC23036DFF8848296
:104090004837DFF88092DFF87CA208F16008DFF88B
:1040A00074B209F1780920680AF1900A0BF1A80BA3
:1040B00060453BD0A84239D0B04237D0B84235D065
:1040C000404533D0484531D050452FD058452DD0AC
:1040D000DFF844C2604529D0DFF83CC20CF1180C6F
:1040E000604523D0DFF830C20CF1300C60451DD0A4
:1040F000DFF824C20CF1480C604517D0DFF818C275
:104100000CF1600C604511D0DFF80CC20CF1780C9A
:1041100060450BD0DFF800C20CF1900C604505D073
:10412000DFF8F4C10CF1A80C604506D1D0F800C04E
:104130002CF0010CC0F800C005E0D0F800C02CF055
:10414000010CC0F800C02046FDF7FEFC7149206854
:1041500088422CD0A8422AD0B04228D0B84226D0DB
:10416000404524D0484522D0504520D058451ED047
:10417000694A90421BD0684A1832904217D0664A6A
:104180003032904213D0644A483290420FD0624A93
:10419000603290420BD0604A7832904207D05E4A3B
:1041A0009032904203D05C4AA83290420DD102680E
:1041B00022F01E0242F016020260206C90B12068CC
:1041C000026842F0080202600CE0026822F00E026F
:1041D00042F00A020260206C20B12068026842F0BE
:1041E00004020260206888424BD0A84249D0B04205
:1041F00047D0B84245D0404543D0484541D05045CE
:104200003FD058453DD0444A90423AD0424A1832B5
:10421000904236D0404A3032904232D03E4A483204
:1042200090422ED03C4A603290422AD03A4A7832AC
:10423000904226D0384A9032904222D0364AA83254
:1042400090421ED0354A90421BD0344A14329042DC
:1042500017D0324A2832904213D0304A3C32904232
:104260000FD02E4A503290420BD02C4A64329042EA
:1042700007D02A4A7832904203D0284A8C329042A2
:104280000DD1206E0268D20303D5026842F4807219
:104290000260E06E18B1026842F480720260206829
:1042A00088422CD0A8422AD0B04228D0B84226D08A
:1042B000404524D0484522D0504520D058451ED0F6
:1042C000154988421BD014491831884217D0124929
:1042D0003031884213D01049483188420FD00E49FE
:1042E000603188420BD00C497831884207D00A49A6
:1042F0009031884203D00849A831884204D101682E
:1043000041F001010160AFE6016841F00101016087
:10431000AAE60000100002401004024008540258AF
:104320002DE9F84F00227B4D03264FF001080F279F
:104330004FF0B04CE6E008FA02F31C409A46002C1D
:104340007ED00B7903F00303012B01D0022B1BD18C
:10435000D0F80890530006FA03FB29EA0B09D1F8BC
:104360000CB00BFA03FB4BEA090BC0F808B043682A
:1043700023EA0A0391F80490C9F3001909FA02F933
:1043800049EA0309C0F804900B79DB439B070ED080
:10439000D0F80C90530006FA03FA29EA0A09D1F87A
:1043A00008A00AFA03FA4AEA090AC0F80CA00B7935
:1043B00003F00303022B14D1D30800EB8303D3F8DB
:1043C00020A04FEA42794FEAD96907FA09FB2AEAA5
:1043D0000B0AD1F810B00BFA09FB4BEA0A0BC3F831
:1043E00020B0D0F80090530006FA03FA29EA0A092F
:1043F00091F804A00AF0030A0AFA03FA4AEA090A41
:10440000C0F800A04B6813F4403F7AD0424BD3F879
:10441000009049F00209C3F800901B6803F0020302
:10442000009322F0030909F1B049D9F808B49307C1
:104430004FEA137A07FA0AF32BEA030B374B00E033
:104440005FE0984201D100232DE0354B984201D125
:10445000012328E0334B984201D1022323E0324B61
:10446000984201D103231EE0304B984201D104232E
:1044700019E02F4B984201D1052314E02D4B9842AF
:1044800001D106230FE02C4B984201D107230AE00B
:104490002A4B984201D1082305E0294B984201D1CB
:1044A000092300E00A2303FA0AF343EA0B03C9F8DD
:1044B0000834DCF80030A343D1F804905FEAC9293E
:1044C00000D52343CCF80030DCF80430A343D1F806
:1044D00004905FEA892900D52343CCF804306B6847
:1044E000A343D1F804905FEA893900D523436B6078
:1044F0002B68A343D1F804905FEAC93900D5234360
:104500002B60521C0C6834FA02F37FF414AFBDE840
:10451000F88F000080000058F44402580000025850
:104520000004025800080258000C025800100258FB
:104530000014025800180258001C025800200258AB
:1045400000240258002A01D081617047090481616A
:104550007047000001480068000C70470010005CC4
:104560000148806870470000EC0000240248816820
:104570000278114481607047EC00002410B50320DC
:1045800000F0B2F802F03AF90F490A68C2F30323C7
:104590000E4AD35C03F01F03D840096801F00F01F5
:1045A000515C0B4A01F01F0120FA01F11160094929
:1045B00008600F2000F010F808B1012010BD00F0D5
:1045C00053F8002010BD000018440258E4E600082B
:1045D000E8000024E400002410B58AB00446102C42
:1045E0002FD200222146372000F05EF8372000F05D
:1045F0004DF8184804601848016841F02001016036
:10460000006800F02000009001A902A802F080F8E4
:104610000798C0B102F0CEF840001049B0FBF1F1AC
:10462000491E10480E4A026040F2E732C260416003
:1046300000210161816002F09FFD38B101200AB0C4
:1046400010BD0120FBE702F0B5F8E6E7054802F0EF
:10465000EBFDF4E7F0000024E844025840420F006C
:10466000001400402CF2002482B00748016841F099
:1046700002010160006800F00200019000220F2199
:10468000901E02B000F010B8F4440258002809DB74
:10469000012100F01F0291404009800000F1E0205C
:1046A000C0F8001170470000F0B40D460D4B1B68B8
:1046B000C3F30223C3F10704042C00D90424191DF9
:1046C000072901D2002300E0DB1E012606FA04F1CF
:1046D000491E294099409E40761E16403143F0BC49
:1046E00006F057BF0CED00E000F00701054A106826
:1046F0004FF6FF03184040EA0120034908431060C9
:10470000704700000CED00E00000FA057047D0F89B
:10471000E00406F054B801EBC10200EB8202D0F8CD
:10472000E004126A05F078BF01EBC10200EB8202DF
:10473000D0F8E004D2F8602205F0DCBFD0F8E00445
:1047400006F03FB80A0601F00F0101EBC10100EBD2
:10475000810101D5143101E001F51571006806F001
:104760008FBD70B5044601F00F002279904201D947
:10477000012070BD0B064FF0010201F00F014FF058
:10478000000501EBC10104EB810102D514314A702F
:1047900002E001F515714D708D70087094F8940465
:1047A000012808D084F89424206806F0E7FB84F8F8
:1047B0009454002070BD022070BD2DE9F0410446E4
:1047C0004FF0010601F00F004FF000050F0600EB5F
:1047D000C00104EB810102D514314E7002E001F5F5
:1047E00015714D700870C2F30A028A600B714A7825
:1047F00002B14883022B00D14D7194F89404012832
:1048000009D084F89464206806F03EFB284684F8BA
:104810009454BDE8F0810220FBE710B501F00F04CD
:1048200004EBC40100EB810101F51571CA600B6155
:1048300000234B614B700C708379012B00D1CA614E
:104840008279006806F0F2FB002010BD70B50446C6
:104850000D4605F00F002179884201D9012070BD75
:1048600029064FF000064FF0010206D500EBC0010B
:1048700004EB810114314A7006E005EBC50104EB3D
:10488000810101F515714E708A70087094F89404D6
:10489000012807D084F89424206806F09BFB2807A1
:1048A00002D007E0022070BDA17904F29C4220688A
:1048B00006F03AFB84F89464002070BD10B501F056
:1048C0000F0404EBC40100EB81011431CA600B61D9
:1048D00000234B6101234B700C708379012B00D1B5
:1048E000CA618279006806F0A1FB002010BD2DE9A5
:1048F000F84F04462568284606F046FD00287ED17C
:10490000206806F06DFD002879D0D5F80808C0F3BE
:104910000D20C4F8D404206806F062FD800704D599
:104920002068416901F002014161206806F058FDEC
:10493000C10604F29C40009035D52068816921F0C1
:10494000100181612F6A07F00F0000EBC00004EB3B
:10495000800606F51576C7F34340022802D00628E4
:1049600012D01BE047F6F070074217D0C7F30A12C7
:10497000F1681746284606F037FDF0683844F060C5
:1049800070693844706109E000990822284606F0F1
:104990002BFD7069C7F30A110844706120688169B2
:1049A00041F010018161206806F01AFD00034FF00C
:1049B000080B4FF000094FF001085ED50026206873
:1049C00006F0EDFC824655E05FEACA704FD02068E1
:1049D000F1B206F0FDFC0746F80707D005EB4610DC
:1049E000C0F8088B3146204604F0ACF8380709D5EA
:1049F00005EB4610C0F808BB3146204600E015E242
:104A000004F07CF8F80604D505EB46111020C1F837
:104A1000080BB8071CD56869000605D5D5F8040849
:104A200040F48061C5F8041806EBC60004EB800072
:104A300000F51570C178012905D180F80390204652
:104A4000F1B200F0F9F905EB46110220C1F8080BAC
:104A5000B80604D505EB46102021C0F8081BB804A1
:104A600005D505EB46104FF40051C0F8081B761C25
:104A70004FEA5A0ABAF1000FA6D1206806F0B0FC3E
:104A800040036CD5206806F083FC8246002663E074
:104A90005FEACA705DD02068F1B206F087FC074675
:104AA000F80723D006F00F0108FA01F0D5F8341802
:104AB0008143C5F8341805EB4610C0F80889A07981
:104AC00001280FD106EBC60004EB8000D0E90721D6
:104AD0001144016236B9606A20B920680121009A48
:104AE00006F022FA2046F1B2FFF715FE380703D58B
:104AF00005EB4610C0F808B9F80604D505EB4611D9
:104B00001020C1F80809780604D505EB46104021AD
:104B1000C0F80819B80716D53146284606F002FC39
:104B200006EBC60004EB80001430C178012905D1E2
:104B300080F803902046F1B200F07AF905EB4611B7
:104B40000220C1F80809380603D53146204604F092
:104B50006BF8761C4FEA5A0ABAF1000F98D1206818
:104B600006F03EFC002811DAD5F8040820F0010117
:104B7000C5F8041894F8CC04012839D0204600F078
:104B800076F92068416901F000414161206806F032
:104B900027FC00050BD5D5F80808C00702D0204631
:104BA00000F088F92068416901F4006141612068E2
:104BB00006F016FC00010AD52068416901F0006189
:104BC000416194F8CC04D0B1204600F073F920681C
:104BD00006F006FCC0046ED5D5F8040820F00101EB
:104BE000C5F804182068102106F09CFB00212DE078
:104BF00084F8CC9400212046FFF788FDC1E784F8B3
:104C0000CC842068406DC0F38300C4F8D004012137
:104C10002046FFF77BFDDAE705EB41104FF67F32C8
:104C200000F510608260036823F400130360C0F88D
:104C30000822D0F8002222F40012C0F80022D0F896
:104C4000002242F00062C0F80022491C207988420C
:104C5000E2D8D5F81C0840F00111C5F81C18E07B1B
:104C600060B1D5F8840840F00B01C5F88418D5F878
:104C7000440840F00B01C5F844180CE0D5F81408BE
:104C800042F22B010843C5F81408D5F8100840F08B
:104C90000B01C5F81018D5F8000820F4FE61C5F81E
:104CA0000018A1792068009A06F03EF92068416951
:104CB00001F480514161206806F092FB800415D513
:104CC000206806F023F9206806F04EFBE07101F041
:104CD0004FFDE2790146206806F0B4FB204600F063
:104CE000AFF82068416901F400514161206806F085
:104CF00077FB000707D5204600F0BDF82068416922
:104D000001F008014161206806F06AFB000615D534
:104D1000A86920F08001A96101260CE006EBC6001D
:104D200004EB800090F85702012803D12046F1B22D
:104D3000FFF708FD761C2079B042EFD8206806F016
:104D40004FFBC0021FD5012615E005EB4610D0F839
:104D5000001906EBC60004EB8000027E012A09D18F
:104D6000002907DA80F81780F0B240F08001204671
:104D7000FFF7E8FC761C2079B042E6D8206841694C
:104D800001F480114161206806F02AFB800230D5D1
:104D9000012026E005EB4011D1F8001B00EBC0021A
:104DA00004EB820292F85832012B19D1002917DA4C
:104DB00094F8D434C1F3004103F001038B420FD1C6
:104DC00082F85782A96941F08002AA6169690906DF
:104DD00006D4D5F8040840F40070C5F8040803E0D0
:104DE000401C21798142D5D82068416901F4001125
:104DF0004161206806F0F4FA400007D52046FFF72D
:104E000086FC2068416901F080414161206806F01C
:104E1000E7FA40070AD520684568680702D52046AA
:104E2000FFF78CFC2068416829434160BDE8F88F9A
:104E3000D0F8E00405F0E4BCD0F8E00405F0F5BCDF
:104E400070B504460125E07900280ED0022801D073
:104E5000FCF799FFD4F8E004294605F057FDD4F893
:104E6000E004BDE8704005F00ABD0025F2E7D0F887
:104E7000E00405F034BDD0F8E00405F03ABD10B50B
:104E8000044694F8940401280AD0012084F894047C
:104E90006174206806F0C7FA002084F8940410BDFD
:104EA000022010BDD0F8E02400F29C41104605F02D
:104EB00039BD000010B50446D4F8E00405F06BFDE0
:104EC0002068D0F8001E41F00101C0F8001EE07A11
:104ED000002804D00248016841F00601016010BDBD
:104EE00010ED00E070B514490A68D243520708D5A6
:104EF000096801F00701814201D0012070BD002046
:104F000070BD0A6822F0070202430A60FFF728FB1F
:104F10000446094D4FF47A76083D06E0FFF720FB82
:104F2000001BB04201D9012070BD2868C043800435
:104F3000F4D4002070BD00000C48025810B501F0F8
:104F400017FC05490968054AC1F30211515C01F0DB
:104F50001F01C84010BD000020440258E4E60008CC
:104F600010B569490A6802F003020968C1F3051126
:104F7000654B1B1D1B6803F00103634C0C34246854
:104F8000C4F3CC0414FB03F300EE103AB8EE400A6D
:104F9000002971D09FED5D1A9FED5D2A5A4BF7EE07
:104FA000000A0833F2B3012A7DD0022A7AD001EE3A
:104FB000901A1968F8EE611AC2EE212AC1F30801AD
:104FC00001EE901AF8EE611A40EE011A31EEA00AD5
:104FD00022EE800A1968C1F3462101EE101AB8EEDC
:104FE000411A31EE201AC0EE011ABCEEE11A80ED32
:104FF000001A1968C1F3064101EE101AB8EE411A01
:1050000031EE201AC0EE011ABCEEE11A80ED011A51
:105010001968C1F3066101EE101AB8EE411A71EE7B
:10502000200A00E006E080EE201ABCEEC10A80ED06
:10503000020A10BD344A283A1468A4061ED5126824
:10504000C2F3C104334AE24001EE902AF8EE612A2D
:1050500001EE901A1968F8EE611A82EEA12AC1F3E6
:10506000080101EE901AF8EE611A40EE011A31EED5
:10507000A00A22EE000AADE741E014E001EE901A2A
:105080001968F8EE611AC2EE212AC1F3080101EE97
:10509000901AF8EE611A40EE011A31EEA00A22EEE3
:1050A000800A97E715E001EE901ADFED1B2A1968D8
:1050B000F8EE611A82EEA12AC1F3080101EE901AFE
:1050C000F8EE611A40EE011A31EEA00A22EE000A53
:1050D00080E701EE901ADFED112A1968F8EE611AE7
:1050E00082EEA12AC1F3080101EE901AF8EE611ACE
:1050F00040EE011A31EEA00A22EE000A6AE7002112
:1051000001604160816010BD2844025800000039F0
:105110000024744C0090D0030024744A20BCBE4B81
:1051200010B569490A6802F003020968C1F3053144
:10513000654B1B1D1B68C3F30013634C14342468B8
:10514000C4F3CC0414FB03F300EE103AB8EE400AAB
:10515000002971D09FED5D1A5B4BF7EE000A10330A
:10516000F2B39FED5B2A012A7FD0022A7CD001EEA8
:10517000901A1968F8EE611AC2EE212AC1F30801EB
:1051800001EE901AF8EE611A40EE011A31EEA00A13
:1051900022EE800A1968C1F3462101EE101AB8EE1A
:1051A000411A31EE201AC0EE011ABCEEE11A80ED70
:1051B000001A1968C1F3064101EE101AB8EE411A3F
:1051C00031EE201AC0EE011ABCEEE11A80ED011A90
:1051D0001968C1F3066101EE101AB8EE411A00E039
:1051E00008E071EE200A80EE201ABCEEC10A80EDC4
:1051F000020A10BD344A283A1468A4061ED5126863
:10520000C2F3C104334AE24001EE902AF8EE612A6B
:1052100001EE901A1968F8EE611A82EEA12AC1F324
:10522000080101EE901AF8EE611A40EE011A31EE13
:10523000A00A22EE000AADE741E016E001EE901A66
:10524000DFED252A1968F8EE611A82EEA12AC1F372
:10525000080101EE901AF8EE611A40EE011A31EEE3
:10526000A00A22EE000A95E713E001EE901A1968F1
:10527000F8EE611AC2EE212AC1F3080101EE901A7C
:10528000F8EE611A40EE011A31EEA00A22EE800A11
:1052900080E701EE901ADFED112A1968F8EE611A25
:1052A00082EEA12AC1F3080101EE901AF8EE611A0C
:1052B00040EE011A31EEA00A22EE000A6AE7002150
:1052C00001604160816010BD28440258000000392F
:1052D0000024744A0090D0030024744C20BCBE4BC0
:1052E00010B569490A6802F003020968C1F3055163
:1052F000654B1B1D1B68C3F30023634C1C342468DF
:10530000C4F3CC0414FB03F300EE103AB8EE400AE9
:10531000002971D09FED5D1A5B4BF7EE000A183340
:10532000F2B39FED5B2A012A7FD0022A7CD001EEE6
:10533000901A1968F8EE611AC2EE212AC1F3080129
:1053400001EE901AF8EE611A40EE011A31EEA00A51
:1053500022EE800A1968C1F3462101EE101AB8EE58
:10536000411A31EE201AC0EE011ABCEEE11A80EDAE
:10537000001A1968C1F3064101EE101AB8EE411A7D
:1053800031EE201AC0EE011ABCEEE11A80ED011ACE
:105390001968C1F3066101EE101AB8EE411A00E077
:1053A00008E071EE200A80EE201ABCEEC10A80ED02
:1053B000020A10BD344A283A1468A4061ED51268A1
:1053C000C2F3C104334AE24001EE902AF8EE612AAA
:1053D00001EE901A1968F8EE611A82EEA12AC1F363
:1053E000080101EE901AF8EE611A40EE011A31EE52
:1053F000A00A22EE000AADE741E016E001EE901AA5
:10540000DFED252A1968F8EE611A82EEA12AC1F3B0
:10541000080101EE901AF8EE611A40EE011A31EE21
:10542000A00A22EE000A95E713E001EE901A19682F
:10543000F8EE611AC2EE212AC1F3080101EE901ABA
:10544000F8EE611A40EE011A31EEA00A22EE800A4F
:1054500080E701EE901ADFED112A1968F8EE611A63
:1054600082EEA12AC1F3080101EE901AF8EE611A4A
:1054700040EE011A31EEA00A22EE000A6AE700218E
:1054800001604160816010BD28440258000000396D
:105490000024744A0090D0030024744C20BCBE4BFE
:1054A0002DE9F04F89B0FD4CFB4A80F48079DFF89C
:1054B000E8834FF080572511F94BDFF8E8A3503A05
:1054C00059EA0109A8F104064FF0005C36D080F4D7
:1054D000007959EA01097FD0DFF8BC9380F4806B32
:1054E0005BEA010B09F108096FD080F4006B5BEAFD
:1054F000010B6BD080F4805B5BEA010B67D080F41A
:10550000005B5BEA010B4FF4803A4FF4003E6ED033
:1055100080F4002B5BEA010B6AD080F4803B5BEAED
:10552000010B75D080F480460E4372D080F40040A9
:1055300008436FD0002009B0BDE8F08FD8F8000014
:1055400000F00700052845D2DFE800F0030D174200
:1055500021001068800104D506A8FFF701FD079817
:10556000E9E70020E7E71068000104D503A8FFF78A
:10557000D7FD0398DFE70020DDE71068800004D541
:105580006846FFF7ADFE0098D5E70020D3E7306806
:1055900000F040501168490700D530B11168C905C5
:1055A0000AD5B84208D12846C5E71068C0F3C10043
:1055B00024FA00F0BFE70FE01168890303D56045C6
:1055C00001D11846B7E70020B5E759E0AAE0FBE0B3
:1055D0005046B0E70020AEE7D8F8000000F4E070D5
:1055E000802824D005DC58B1402807D115E03DE1E2
:1055F0008AE1C02842D0B0F5807F22D000209AE70F
:105600001068800107D506A8FFF7AAFC079892E763
:10561000B6E1D1E115E200208DE71068000104D564
:1056200003A8FFF77DFD039885E7002083E7106856
:10563000800004D56846FFF753FE00987BE7002002
:1056400079E7306800F040501168490700D530B163
:105650001168C90509D5B84207D128466BE710681B
:10566000C0F3C10024FA00F065E71168890303D58F
:10567000604501D118465EE700205CE750465AE7D6
:10568000D9F8000000F46000B0F5800F21D004DCF0
:1056900058B1B0F5001F06D111E0B0F5C00F3FD0F2
:1056A000B0F5000F1FD0002045E71068800104D539
:1056B00006A8FFF755FC07983DE700203BE7106878
:1056C000000104D503A8FFF72BFD039833E7002062
:1056D00031E71068800004D56846FFF701FE0098A6
:1056E00029E7002027E7306800F04050116849079B
:1056F00000D530B11168C90509D5B84207D128468F
:1057000019E71068C0F3C10024FA00F013E711682C
:10571000890303D5604501D118460CE700200AE74C
:10572000504608E7D9F8000000F0E060B0F1007FD3
:1057300021D004DC58B1B0F1807F06D111E0B0F186
:10574000407F3FD0B0F1806F1FD00020F3E610689B
:10575000800104D506A8FFF703FC0798EBE60020BC
:10576000E9E61068000104D503A8FFF7D9FC039807
:10577000E1E60020DFE61068800004D56846FFF708
:10578000AFFD0098D7E60020D5E6306800F0405025
:105790001168490700D530B11168C90509D5B8426B
:1057A00007D12846C7E61068C0F3C10024FA00F00C
:1057B000C1E61168890303D5604501D11846BAE6F0
:1057C0000020B8E65046B6E6D8F8000000F4E04005
:1057D000B0F5005F21D004DC58B1B0F5805F06D190
:1057E00011E0B0F5405F3FD0B0F5804F1FD00020F2
:1057F000A1E61068800104D506A8FFF7B1FB079861
:1058000099E6002097E61068000104D503A8FFF789
:1058100087FC03988FE600208DE61068800004D591
:105820006846FFF75DFD009885E6002083E6306856
:1058300000F040501168490700D530B11168C90522
:1058400009D5B84207D1284675E61068C0F3C100F3
:1058500024FA00F06FE61168890303D5604501D191
:10586000184668E6002066E6504664E6D8F8000070
:1058700000F4E020B0F5403F2DD015DCE0B15045FC
:105880001DD0704516D11068800022D56846FFF7FC
:1058900027FD01984FE60000504402580090D003C5
:1058A00040787D010080BB00B0F5802F1ED0B0F5A0
:1058B000A02F22D000203EE600F07CFF3BE61068DF
:1058C000000104D503A8FFF72BFC049833E6002061
:1058D00031E600202FE61068400705D51068C0F3B8
:1058E000C10024FA00F026E6002024E61068C00576
:1058F00001D528461FE600201DE61068800301D56B
:10590000184618E6002016E6D9F8000000F44030EA
:1059100088B1504519D0704530D1306800F0405002
:105920001168490700D5D0B11168C9051DD5B84225
:105930001BD12846FFE51068000104D503A8FFF736
:10594000EFFB0398F7E50020F5E51068800004D52B
:105950006846FFF7C5FC0298EDE50020EBE510680E
:10596000C0F3C10024FA00F0E5E51168890303D50E
:10597000604501D11846DEE50020DCE50020DAE5CF
:10598000306800F4803048B1504513D110680001F0
:105990000ED503A8FFF7C4FB0598CCE5106880017D
:1059A00004D506A8FFF7DCFA0798C4E50020C2E595
:1059B0000020C0E50020BEE5D9F8000000F0E0407E
:1059C000B0F1405F24D00CDC98B1B84214D06045EF
:1059D0000DD11068800019D56846FFF781FC019849
:1059E000A9E5B0F1804F1ED0B0F1A04F22D0002029
:1059F000A1E5FFF7A3FA9EE51068000104D503A80E
:105A0000FFF78EFB049896E5002094E5002092E5D0
:105A10001068400705D51068C0F3C10024FA00F0F3
:105A200089E5002087E51068C00501D5284682E594
:105A3000002080E51068800301D518467BE5002032
:105A400079E5D8F8000000F0405058B1B84210D0C5
:105A500060451AD11068000115D503A8FFF760FB57
:105A6000049868E51068800301D5184663E50020B6
:105A700061E51068800104D506A8FFF771FA079860
:105A800059E5002057E5002055E5002053E50000CA
:105A90002DE9FC5F044600250026F94F2068DFF859
:105AA000E483C043010104F10800019004F12800DF
:105AB00000900DD4A06EB8B1B0F5801F19D0B0F52C
:105AC000001F1CD0B0F5401F00D00125EDB12E46BF
:105AD0002088C043C00535D4A06D05282FD2DFE84B
:105AE00000F01D22282F2F00386840F40030386065
:105AF000ECE70198022103F0E5F80546E6E7009897
:105B0000022103F071F90546E0E7D8F80000A16E24
:105B100020F440100843C8F80000D9E7386840F482
:105B2000003038600CE00198002103F0CBF8054606
:105B300006E00098002103F057F9054600E0012532
:105B400065B12E462088C043800518D4E06D8028BA
:105B500031D00CDC20B340280ED126E0D8F800006C
:105B6000A16D20F007000843C8F80000EAE7C0284C
:105B700003D0B0F5807F00D0012515B32E462088D4
:105B8000DFF80493C04340052DD4D4F8A800B0F545
:105B9000800F43D01EDCA8B3B0F5001F20D137E042
:105BA000386840F400303860E7E70198002103F0DE
:105BB00089F80546E1E70098002103F015F905464C
:105BC000DBE7D8F80000E16D20F4E0700843C8F886
:105BD0000000D4E7B0F5C00F03D0B0F5000F00D03F
:105BE00001250DB32E462088C04300052FD4D4F8DC
:105BF000AC00B0F1007F54D020DCE8B3B0F1807F7E
:105C000022D148E0FFE7386840F400303860E8E728
:105C10000198002103F056F80546E2E700980021BC
:105C200003F0E2F80546DCE7D9F80000D4F8A81044
:105C300020F460000843C9F80000D4E7B0F1407FC9
:105C400003D0B0F1806F00D0012585B32E462068C7
:105C5000C04380010AD4E06C30B1102832D0202833
:105C600036D0302800D001258DB32E462088C04381
:105C7000C00446D4206E00E008E0B0F5005F5CD0C0
:105C800036DCA0B3B0F5805F38D150E0386840F41E
:105C900000303860D9E70198002103F013F8054679
:105CA000D3E70098002103F09FF80546CDE7FFE712
:105CB000D9F80000D4F8AC1020F0E0600843C9F82F
:105CC0000000C4E7386840F400303860CCE705E0F5
:105CD0000198022102F0F6FF0546C5E76948001F5A
:105CE0000168E26C21F0300111430160BEE719E068
:105CF000B0F5405F03D0B0F5804F00D0012515B35B
:105D00002E462088C04380042FD4606EB0F5403FFB
:105D100029D021DC38B3B0F5803F38D0B0F5003F52
:105D200020D13AE0386840F400303860E7E7019865
:105D3000002102F0C7FF0546E1E70098002103F0CB
:105D400053F80546DBE7D8F80000216E20F4E04068
:105D50000843C8F80000D4E7B0F5802F03D0B0F5B1
:105D6000A02F00D00125F5B12E462088C043400465
:105D70002BD4D4F8B000B0F1405F24D01CDC10B3B9
:105D8000B0F1805F4ED0B0F1005F1BD151E00198BF
:105D9000012102F097FF0546E5E70098012103F095
:105DA00023F80546DFE7D8F80000616E20F4E02014
:105DB0000843C8F80000D8E7B0F1804F03D0B0F135
:105DC000A04F00D001259DB32E462088C04300047B
:105DD0000AD4206F30B1B0F1805F3CD0B0F1005FE9
:105DE0003ED00125ADB32E462068C043C0010AD481
:105DF000A06C30B101284DD0022850D0032800D02B
:105E000001253DB32E462068DFF880B0C043400234
:105E100061D41F48016841F480710160FEF7A0FB66
:105E2000824652E00198012102F04CFF0546CAE784
:105E300005E00098012102F0D7FF0546C3E7D9F835
:105E40000000D4F8B01020F0E0400843C9F800008A
:105E5000BBE70BE029E0386840F400303860C1E768
:105E60000198012102F02EFF0546BBE7D8F800009B
:105E7000216F20F040500843C8F80000B4E700004C
:105E80002C440258504402585844025810440258B6
:105E900000480258386840F400303860B1E7019893
:105EA000022102F00FFF0546ABE7FE480168A26C35
:105EB00021F0030111430160A5E7FEF751FBA0EBC0
:105EC0000A00642801D9032503E0F7480068C005EB
:105ED000F3D53DB12E462078DFF8D0A3C043C007EC
:105EE00055D065E0F1481C300068B4F8B41000F4F7
:105EF000407001F4407188420DD0EC481C300168BC
:105F000021F44071026842F480320260026822F497
:105F1000803202600160D4F8B400B0F5807F12D105
:105F2000FEF71EFB824609E0FEF71AFBA0EB0A0112
:105F300041F28830814201D9032504E0DB481C305E
:105F400000688007F0D50DB12E46C4E7D4F8B40040
:105F5000C0F3012103290FD0DBF8000020F47C50AE
:105F6000CBF80000D1481C300168B4F8B420C2F36B
:105F70000B0211430160AEE7DBF80010CC4A21F4BC
:105F80007C51104041EA1010CBF80000EAE7E06FC6
:105F900018280BD005DC48B1082815D0102804D1EA
:105FA00018E0202802D0282800D00125C5B12E46AF
:105FB0002078C04380072BD4A06F062825D2DFE8C5
:105FC00000F025181E2525250198012102F07AFEF2
:105FD0000546EBE70098012102F006FF0546E5E7DC
:105FE000DAF80000E16F20F038000843CAF800003A
:105FF000DEE70198012102F065FE054606E0009803
:10600000012102F0F1FE054600E001256DB12E46AA
:106010002078C043400720D4D4F89400062819D231
:10602000DFE800F0190C12191919DAF80000A16F55
:1060300020F007000843CAF80000E9E701980121B1
:1060400002F040FE054606E00098012102F0CCFE79
:10605000054600E0012595B12E462078C043800614
:1060600020D4D4F89000B0F1405F19D011DCB8B161
:10607000B0F1805F28D0B0F1005F10D12AE0D9F8EC
:106080000000D4F8941020F007000843C9F800007D
:10609000E3E7B0F1804F03D0B0F1A04F00D001256D
:1060A000F5B12E462078C04340062CD4D4F89C008D
:1060B000B0F5406F25D01DDC18B3B0F5806F34D03B
:1060C000B0F5006F1CD136E00198002102F0FAFD16
:1060D0000546E5E70098022102F086FE0546DFE767
:1060E000DAF80000D4F8901020F0E0400843CAF835
:1060F0000000D7E7B0F5805F03D0B0F5A05F00D017
:106100000125F5B12E462078C04300062CD4D4F8E2
:10611000A000B0F5C04F25D01DDC18B3B0F5005F6E
:106120002CD0B0F5804F1CD12EE00198002102F058
:10613000C9FD0546E5E70098022102F055FE054637
:10614000DFE7D9F80000D4F89C1020F4E0500843B1
:10615000C9F80000D7E7B0F5004F03D0B0F5204FE5
:1061600000D00125B5B12E462078C04300072AD4BF
:10617000D4F88400B0F5805F16D01BE001980021B0
:1061800002F0A0FD0546EDE70098022102F02CFE8A
:106190000546E7E7D9F80000D4F8A01020F46040E5
:1061A0000843C9F80000DFE70098022102F01CFE56
:1061B00000B10126DAF80000D4F8841020F4405031
:1061C0000843CAF800002078C043C00613D4D4F8AE
:1061D0009800B0F5807F05D10098022102F004FEFE
:1061E00000B10126D9F80000D4F8981020F44070CE
:1061F0000843C9F800002068C04300030BD4D4F85A
:10620000A400E8B3B0F5803F7DD0B0F5003F00D0EA
:106210000125B5B32E462068C04340030DD4D4F801
:106220008800B0F5801F70D0B0F5001F6ED0B0F5BB
:10623000401F00D00125EDB32E462068C043C003A7
:1062400007D4206DB8B3B0F5803F7CD001259DB355
:106250002E462068C043800005D40098022102F039
:10626000C3FD00B101262068C043800311D4D4F8D7
:10627000800060B1B0F5807F66D0B0F5007F01E0AE
:1062800070E07BE003D0B0F5407F00D00125DDB3A6
:106290002E462068C043C00213D4D8F8000020F076
:1062A00000400AE04C440258004802585444025846
:1062B000FFFCFF0F77E080E08AE0616F0843C8F8D9
:1062C00000002068C043C00008D4DBF80000D4F808
:1062D000B81020F480400843CBF800002068C04389
:1062E000800207D4D8F80000E16E20F080700843E7
:1062F000C8F800002068C043400011D4DBF800005B
:1063000020F4004003E033E06FE041E045E0CBF8EB
:106310000000DBF80000D4F8BC100843CBF8000004
:106320002068C04306D45A480168626D21F040518C
:10633000114301602068C04300020BD4DAF800006A
:1063400020F4400001E03DE04AE0D4F88C1008431E
:10635000CAF8000020790025C04300F0010028435E
:106360004DD052E00198002102F0ACFC054650E708
:106370000098022102F038FD05464AE7D9F80000EE
:10638000D4F8A41020F440300843C9F8000042E7D4
:10639000386840F4003038604DE70098012102F081
:1063A00023FD054647E7DAF80000D4F8881020F40A
:1063B00040100843CAF800003FE7386840F4003056
:1063C000386044E70198022102F07CFC05463EE774
:1063D0002F480168226D21F480311143016038E7B4
:1063E000386840F40030386051E7DAF80000D4F83B
:1063F000801020F440700843CAF8000049E7019873
:10640000002102F05FFC00B106462079C04300F095
:106410000200284305D10198012102F053FC00B18C
:1064200006462079C04300F00400284305D10198B6
:10643000022102F047FC00B106462079C04300F07B
:106440000800284305D10098002102F0CDFC00B1DE
:1064500006462079C04300F01000284305D100987B
:10646000012102F0C1FC00B106462079C04300F0D2
:106470002000054305D10098022102F0B5FC00B1CF
:10648000064616B10120BDE8FC9F0020FBE7000096
:106490004C4402582DE9F05F04460D46002C17D0FD
:1064A000DFF84C82D8F8000000F00F00A84211D2AB
:1064B000D8F8000020F00F002843C8F80000D8F8F2
:1064C000000000F00F00A84204D00120BDE8F09FBA
:1064D0000120FBE72078874E40070AD52069316804
:1064E00001F07001884204D9316821F07001014344
:1064F00031602078804F00070AD56069396801F063
:106500007001884204D9396821F070010143396073
:106510002078C0060AD5A069396801F4E061884294
:1065200004D9396821F4E061014339602078DFF84B
:10653000CC9180060DD5E069D9F8001001F070010A
:10654000884206D9D9F8001021F070010143C9F83A
:106550000010207880070AD5E068316801F00F014B
:10656000884204D9316821F00F010143316020785D
:10657000C00743D03068A16820F4706008433060E1
:106580005C4960681839022808D003280BD001281C
:106590000ED00968490710D4012097E709688903DC
:1065A0000BD4012092E70968890106D401208DE708
:1065B0000968C90501D4012088E7DFF838A1AAF1EC
:1065C000080ADAF8001021F007010143CAF80010A8
:1065D000FDF7C6FF834609E0FDF7C2FFA0EB0B0104
:1065E00041F28830814201D903206FE7DAF80000D8
:1065F000616800F03800B0EBC10FEDD12078800762
:106600000AD5E068316801F00F01884204D2316890
:1066100021F00F0101433160D8F8000000F00F00B5
:10662000A8420ED9D8F8000020F00F002843C8F87F
:106630000000D8F8000000F00F00A84201D00120AF
:1066400044E7207840070AD52069316801F07001DD
:10665000884204D2316821F0700101433160207812
:1066600000070AD56069396801F07001884204D2D8
:10667000396821F07001014339602078C0060AD5DD
:10668000A069396801F4E061884204D2396821F4D4
:10669000E06101433960207880060DD5E069D9F8C2
:1066A000001001F07001884206D2D9F8001021F0E4
:1066B00070010143C9F8001000F0A0F83168C1F37F
:1066C00003220F498A5C02F01F02D040326802F0B8
:1066D0000F02895C0B4A01F01F0120FA01F11160E1
:1066E0000949086009480068BDE8F05FFDF774BF1C
:1066F00000200052184402581C44025820440258FA
:10670000E4E60008E8000024E4000024F00000248F
:106710003F220260144A126802F007024260124AE5
:106720000832136803F470638360136803F00F0387
:10673000C360126802F0700202610B4A0C321368E7
:1067400003F070034361126802F4E0628261064A5A
:106750001032126802F07002C2610448006800F052
:106760000F000860704700001044025800200052DB
:1067700000B500F043F80B490A68C2F303230A4A44
:10678000D35C03F01F03D840096801F00F01515C8E
:10679000064A01F01F0120FA01F11160044A10605D
:1067A000084600BD18440258E4E60008E80000244A
:1067B000E400002400B5FFF7DBFF05490968054A3E
:1067C000C1F30211515C01F01F01C84000BD00007F
:1067D0001C440258E4E6000800B5FFF7C9FF05496C
:1067E0000968054AC1F30221515C01F01F01C8404C
:1067F00000BD00001C440258E4E6000830B56448BF
:106800000068654C10F03801624808D00211082970
:106810000DD010290DD018290DD0104630BD21689B
:106820008906FBD52168C1F3C101C84030BD1046BF
:1068300030BD5A4830BD564918310A6802F003028B
:106840000968C1F30511524B1C331B6803F00103A7
:106850004F4D24352D68C5F3CC0515FB03F300EE31
:10686000103AB8EE400A002977D0DFED4D0A484BC8
:10687000B7EE001A20333AB39FED4A2A012A58D0C6
:10688000022A6CD001EE901A1868F8EE611AC2EE76
:10689000212AC0F3080001EE900AF8EE611A40EEDA
:1068A000201A31EE810A22EE800A1868C0F34620D1
:1068B000401C00EE900AF8EE600A80EE201ABCEE52
:1068C000C10A10EE100A30BD226892061BD522685C
:1068D000C2F3C102D04001EE900A1868F8EE612AB6
:1068E00001EE901AF8EE611A82EEA12AC0F30800B8
:1068F00001EE900AF8EE611A40EE201A31EE810A9C
:1069000022EE000AD1E701EE901ADFED272A18687F
:10691000F8EE611A82EEA12AC0F3080001EE900A97
:10692000F8EE611A40EE201A31EE810A22EE000ADA
:10693000BBE701EE901A1868F8EE611AC2EE212A40
:10694000C0F3080001EE900AF8EE611A40EE201A3A
:1069500031EE810A22EE800AA7E716E0FFE701EE9A
:10696000901ADFED122A1868F8EE611A82EEA12A59
:10697000C0F3080001EE900AF8EE611A40EE201A0A
:1069800031EE810A22EE000A8FE7002030BD0000C0
:10699000104402580090D0030044025840787D0112
:1069A000000000390024744A0024744C20BCBE4B03
:1069B0002DE9F05F0446002C10D02078DFF8F88332
:1069C000FE4EFF4DC0075DD0D8F8000000F0380043
:1069D000316810281FD0182803D006E00120BDE838
:1069E000F09F01F00300022815D06068B0F5803FE9
:1069F00018D0E0B1B0F5A02F22D0286820F4803064
:106A00002860286820F480202860606860B3FDF763
:106A1000A7FD074624E02868800333D5606810BBD3
:106A20000120DCE7286840F480302860EDE7286822
:106A300020F480302860286820F480202860E4E773
:106A4000286840F480202860286840F4803028605E
:106A5000DBE7FDF785FDC01B642801D90320BEE7F5
:106A600028688003F5D50DE0FDF77AFD074606E0BE
:106A7000FDF776FDC01B642801D90320AFE7286825
:106A80008003F5D4207841F2030ACE4F80073DD52C
:106A9000D8F8000000F03800316870B1182801D132
:106AA00088070AD0E06890B3296821F019010143F2
:106AB0002960FDF755FD814641E02868400701D572
:106AC000E06848B12868E16820F0190008432860B0
:106AD000FDF746FD814609E0012080E7FDF740FD16
:106AE000A0EB0900022801D9032078E728684007B5
:106AF000F4D5FDF72FFD504511D82069402807D067
:106B0000396821F47C3141EA003038604AE036E0EF
:106B1000386820F47C3040F40030386042E0386857
:106B2000217C20F0FE4040EA016038603AE0FDF749
:106B300017FDA0EB0900022801D903204FE72868C0
:106B40004007F4D5FDF706FD504510D820694028D0
:106B500006D0396821F47C3141EA0030386021E008
:106B6000386820F47C3040F4003038601AE038682F
:106B7000217C20F0FE4040EA0160386012E0286885
:106B800020F001002860FDF7EBFC814607E0FDF7EF
:106B9000E7FCA0EB0900022801D903201FE72868C1
:106BA0004007F4D42078C0062FD5D8F8000000F0B4
:106BB00038003168DFF800B20828ABF1040B0FD0C1
:106BC000182803D101F00300012809D0E06978B347
:106BD000286840F080002860FDF7C2FC814630E064
:106BE0002868C00504D5E069802801D00120F6E6B8
:106BF000FDF7B0FC504510D8206A202806D039682F
:106C000021F0F84141EA806038604FE0386820F0B8
:106C1000F84040F08040386048E0DBF8000094F82D
:106C2000201020F07C5040EA0160CBF800003DE0ED
:106C30002AE0FDF795FCA0EB0900022801D903200A
:106C4000CDE62868C005F4D5FDF784FC504510D882
:106C5000206A202806D0396821F0F84141EA806096
:106C6000386023E0386820F0F84040F08040386019
:106C70001CE0DBF8000094F8201020F07C5040EA83
:106C80000160CBF8000011E0286820F08000286047
:106C9000FDF766FC074606E0FDF762FCC01B022814
:106CA00001D903209BE62868C005F5D420780007A9
:106CB00030D5DFF80891606909F14C09A8B1D9F81D
:106CC000000040F00100C9F80000FDF749FC07464C
:106CD00006E0FDF745FCC01B022801D903207EE633
:106CE000D9F800008007F4D514E0D9F8000020F0AE
:106CF0000100C9F80000FDF733FC074606E0FDF788
:106D00002FFCC01B022801D9032068E6D9F8000037
:106D10008007F4D42078800626D5A06990B1286831
:106D200040F480502860FDF71BFC074606E0FDF7A5
:106D300017FCC01B022801D9032050E628688004F4
:106D4000F5D511E0286820F480502860FDF708FC94
:106D5000074606E0FDF704FCC01B022801D903200A
:106D60003DE628688004F5D42078400768D5164FA2
:106D7000386840F480703860FDF7F2FB814607E028
:106D8000FDF7EEFBA0EB0900642801D9032026E6FD
:106D90003868C005F4D5094FA068483701281DD0D0
:106DA00008B3052828D0386820F00100386038681A
:106DB00020F00400386009E01044025828440258CA
:106DC000004402580444025800480258A06841F2A6
:106DD000883A30B3FDF7C4FB81461EE0386840F0C6
:106DE00001003860E7E7386820F001003860386853
:106DF00020F004003860DEE7386840F004003860B6
:106E0000386840F001003860D5E7FDF7A9FBA0EB3A
:106E10000900504501D90320E1E538688007F4D521
:106E20000EE0FDF79DFB814607E0FDF799FBA0EB27
:106E30000900504501D90320D1E538688007F4D412
:106E4000616AE1B3D8F800004FF6F87BDFF8E0A103
:106E5000C0F3C20003280AF10409AAF104087DD096
:106E6000022907D0286820F080702860FDF778FBA1
:106E700004468BE0286820F080702860FDF770FBE6
:106E8000074606E0FDF76CFBC01B022801D9032072
:106E9000A5E528688001F5D4306840F2F3318843D5
:106EA000E16A40EA0110A16A08433060208E4FF683
:106EB000FF72616B401E491EC0F3080000E0B5E0A0
:106EC00002EA41210843218F4FF4FE02491E02EAE3
:106ED0000141084394F83C10491E120202EA016184
:106EE0000843CAF80000D8F8000020F00100C8F8F4
:106EF0000000D9F80000A16C20EA0B0040EAC100B4
:106F0000C9F80000D8F80000216C20F00C000843FC
:106F1000C8F80000D8F80000616C20F002000843B7
:106F2000C8F80000D8F8000040F48030C8F800002D
:106F3000D8F8000040F40030C8F80000D8F800008D
:106F400040F48020C8F80000D8F8000040F00100AC
:106F5000C8F80000286840F0807000E01AE028605F
:106F6000FDF7FEFA044606E0FDF7FAFA001B0228D8
:106F700001D9032033E528688001F5D556E0FDF7F7
:106F8000EFFA001B022801D9032028E528688001B8
:106F9000F5D44BE03268DAF80000012921D0A36A69
:106FA00002F0030199421CD1E16AC2F30512914239
:106FB00017D1216BC0F30802491E8A4211D1616BBF
:106FC000C0F34622491E91420BD1A16BC0F3064289
:106FD000491E914205D1E16BC0F30660491E814212
:106FE00001D00120FBE4D9F80000C0F3CC00A16C73
:106FF00081421BD0D8F8000020F00100C8F8000042
:10700000FDF7AEFA0546FDF7ABFAA842FBD0D9F87A
:107010000000A16C20EA0B0040EAC100C9F80000A2
:10702000D8F8000040F00100C8F800000020D6E4C5
:1070300030440258024A136883430B43136070477D
:1070400004040058704770477047000030B590F84E
:107050003C20012A3AD0012280F83C20CA68002452
:107060008B6822F440721A434B6822F480621A4300
:107070000B6822F400621A430B6922F480521A430F
:107080004B6922F400521A438B6A22F480421A435D
:107090000B8B22F4702242EA03420D4D0368AB428F
:1070A00002D00C4DAB420CD18D8C22F4700242EA1E
:1070B0000552CD6922F080722A43096A22F00072DB
:1070C0000A435A6480F83C40002030BD022030BDA5
:1070D0000000014000040140F0B590F83C20012A76
:1070E0003AD0012680F83C60022280F83D200368F7
:1070F0005A689C68194FDFF868C0BB4201D06345ED
:1071000003D122F470054A682A4322F070020D6808
:1071100015435D600268BA4213D0B2F1804F10D0BF
:10712000104B9A420DD0104B9A420AD00F4B9A4204
:1071300007D0624505D00E4B9A4202D00D4B9A42C1
:1071400004D124F080038968194391603C30467073
:10715000002101700020F0BD0220F0BD00000140C0
:10716000000401400004004000080040000C004002
:10717000001800400040014010B50446002C03D028
:1071800094F83D0010B107E0012010BD002084F804
:107190003C00204600F018F8022084F83D002068EA
:1071A000211D02F0AFF901203D34E0726070A07043
:1071B000E07020716071A071E07120726072A07245
:1071C0002070002010BD000008B5006813498842F7
:1071D00009D11348016841F001010160006800F025
:1071E0000100009008BD0E490839B0F1804F0BD066
:1071F0000C4A9042F6D1086840F004000860086824
:1072000000F00400009008BD086840F0010008602C
:10721000086800F00100009008BD00000000014077
:10722000F04402580008004090F83D10012901D0B8
:1072300001207047022180F83D100168CA6842F0C1
:107240000102CA6000681549884214D0B0F1804F2D
:1072500011D0134988420ED0124988420BD01249EE
:10726000884208D01149884205D01149884202D08D
:10727000104988420CD181680F4A114006290BD071
:10728000B1F5803F08D0016841F00101016003E0E1
:10729000016841F0010101600020704700000140D9
:1072A0000004004000080040000C004000040140C1
:1072B00000180040004001400700010070B504467E
:1072C000002594F83C00012815D0012684F83C6084
:1072D000022084F83D0020688268394B1A4022F46D
:1072E0007F4282600868702802462ED010DC10F0C1
:1072F0000F0F03D022E04FF0020070BD4FEA2010C4
:1073000007281BD2DFE800F0575757574D39430085
:10731000B0F1101F4FD009DCB0F5805F0FD0B0F591
:10732000005F1ED0B0F5801F08D144E0A0F58010AA
:10733000203840D010283ED020283CD001253C34B5
:10734000667000202070284670BDCB682068D1E9A7
:10735000012102F048F92068816841F077018160DD
:10736000EDE7CB682068D1E9012102F03CF9206803
:10737000816841F480418160E1E7CA68496820681A
:1073800002F0D4FA2068502102F038F9D7E7CA6831
:107390004968206802F0DBFA2068602102F02EF9CB
:1073A000CDE7CA684968206802F0C0FA2068402129
:1073B00002F024F9C3E72068114602F01FF9BEE786
:1073C00088FFCEFF70472DE9F04104462068C6686B
:1073D00005694FF00007A90714D5B10712D5F91EAA
:1073E00001610120207720688069800703D0204652
:1073F000FFF7E8FF05E0204600F0B6F8204600F071
:1074000077F92777680717D5700715D521686FF0CA
:1074100004000861022020772068806910F4407F12
:1074200003D02046FFF7CEFF05E0204600F09CF891
:10743000204600F05DF92777280716D5300714D5C8
:1074400021686FF008000861042020772068C06977
:10745000800703D02046FFF7B5FF05E0204600F087
:1074600083F8204600F044F92777E80617D5F006A0
:1074700015D521686FF0100008610820207720687A
:10748000C06910F4407F03D02046FFF79BFF05E062
:10749000204600F069F8204600F02AF92777E8072F
:1074A00008D0F00706D021686FF00100086120467F
:1074B00000F00CFA280601D4A80408D5300606D539
:1074C00021686FF4025008612046FFF7BCFDE80513
:1074D00008D5300606D521686FF480700861204613
:1074E000FFF7B0FD680608D5700606D521686FF075
:1074F00040000861204600F0F3F9A8060AD5B0065E
:1075000008D521686FF0200008612046BDE8F041F1
:10751000FFF79ABDBDE8F08110B586B0044614218E
:1075200001A8F9F7C1F82068B0F1804F16D10C48D6
:10753000016841F001010160006800F00100009065
:107540004FF400400190122002900020039004901C
:107550000120059001A90348FCF7E2FE06B010BD2A
:10756000E044025800000258704770B504460D46CA
:10757000002694F83C0001280BD0012084F83C0040
:107580000C2A4FD007DC82B1042A22D0082A06D167
:1075900034E0022070BD102A59D0142A6BD0012685
:1075A000002084F83C00304670BD2068294602F077
:1075B0002FF82068816941F00801816120688169A4
:1075C00021F004018161206881692A691143816188
:1075D000E6E72068294602F06BF82068816941F4EB
:1075E000006181612068816921F480618161206886
:1075F00081692A6941EA02218161D1E7206829462F
:1076000002F0A0F82068C16941F00801C16120685A
:10761000C16921F00401C1612068C1692A6911436F
:10762000C161BDE72068294602F0D6F82068C1692B
:1076300041F40061C1612068C16921F48061C161C8
:107640002068C1692A6941EA0221C161A8E720686E
:10765000294602F0FBF82068416D41F008014165C0
:107660002068416D21F0040141652068416D2A695F
:107670001143416594E72068294602F01FF920680C
:10768000416D41F4006141652068416D21F48061E4
:1076900041652068416D2A6941EA022141657FE721
:1076A00010B50446002C03D094F83D0010B107E05B
:1076B000012010BD002084F83C00204600F017F89F
:1076C000022084F83D002068211D01F01BFF0120ED
:1076D0003D34E0726070A070E07020716071A07144
:1076E000E07120726072A0722070002010BD70479F
:1076F0007047000030B5044600290DD004290ED093
:1077000008290FD00C2910D0102911D094F843006B
:10771000012810D0012030BD94F83E00F8E794F81D
:107720003F00F5E794F84000F2E794F84100EFE7F6
:1077300094F84200ECE70220E9B3042947D0082975
:1077400048D00C2949D010294AD084F8430001229E
:10775000206801F03BFF27492068274A274B8842D1
:1077600009D0904207D0984205D0254DA84202D0BA
:10777000244DA84203D1456C45F40045456420687A
:10778000884212D0B0F1804F0FD01F4988420CD0F0
:107790001E49884209D01E49884206D0904204D032
:1077A0001C49884201D098421DD181681A4A114073
:1077B00006291CD000E007E0B1F5803F17D0016832
:1077C00041F00101016012E084F83E00BFE784F857
:1077D0003F00BCE784F84000B9E784F84100B6E711
:1077E00084F84200B3E7016841F001010160002024
:1077F00030BD000000000140000401400040014095
:1078000000440140004801400004004000080040DE
:10781000000C0040001800400700010030B504468D
:107820000D4600222946206801F0D0FE41F21112D7
:1078300021492068931088420BD02049884208D003
:107840001F49884205D01F49884202D01E498842FC
:1078500009D1016A114206D1016A194203D1416C72
:1078600021F4004141642068016A114206D1016A95
:10787000194203D1016821F00101016001205DB1CD
:10788000042D0CD0082D0DD00C2D0ED0102D0FD0A6
:1078900084F84300002030BD84F83E00FAE784F805
:1078A0003F00F7E784F84000F4E784F84100F1E78F
:1078B00084F84200EEE700000000014000040140AF
:1078C0000040014000440140004801400068034975
:1078D000884201D1FCF74ABE704700000014004006
:1078E000704790F88410012918D0012180F8841085
:1078F0002421C0F8881001680A680B6823F001038E
:107900000B6022F0005100224266036819602021BA
:10791000C0F8881080F8842000207047022070474B
:1079200010B50446D4F88C00202801D0022010BDE8
:1079300051B14AB10120E06600202067204602F0E4
:1079400015FC014611B105E0012010BDE06E0128D3
:1079500002D00121084610BD226810201062206864
:1079600050E8002F42F0100240E80023002BF6D12F
:10797000F0E7000010B50648F9F71CFD042805D310
:107980000448C068BDE8104004F03ABC10BD0000D7
:107990009025002408000024704770B5044694F830
:1079A000840001281DD0012084F884002420C4F81C
:1079B000880020680568026822F0010202602068E1
:1079C000826822F060620A438260204601F0D2FFA2
:1079D000206805602020C4F88800002084F8840016
:1079E00070BD022070BD70B5044694F88400012873
:1079F0001DD0012084F884002420C4F88800206869
:107A00000568026822F0010202602068826822F0A4
:107A100060420A438260204601F0ACFF20680560A6
:107A20002020C4F88800002084F8840070BD022063
:107A300070BD704770477047014651F8880F49681C
:107A4000084370472DE9F04104462368D869196856
:107A50009A6840F60F0500EA0507002F0ED185064B
:107A60000CD501F0200502F08056354306D0616F39
:107A700000297DD02046BDE8F041084700260225B8
:107A8000002F76D0D54FDFF858C3174001EA0C0C11
:107A900057EA0C0C6DD05FEAC07C0CD05FEAC15C89
:107AA00009D54FF0010CC3F820C0D4F8903043F052
:107AB0000103C4F89030830709D5D30707D02368A2
:107AC0001D62D4F8903043F00403C4F890304307AB
:107AD0000AD5D30708D0256804232B62D4F8903048
:107AE00043F00203C4F8903003070CD501F02003E3
:107AF0003B4308D0256808232B62D4F8903043F02C
:107B00000803C4F8903003050BD54B0109D525684F
:107B10004FF400632B62D4F8903043F02003C4F894
:107B20009030D4F89030002B3CD0800609D501F07D
:107B3000200002F08051084303D0616F09B1204654
:107B40008847D4F8900021688968490602D410F06B
:107B5000280F2DD0204602F06DF82068806840067E
:107B600022D52068083050E8001F21F0400101E0D4
:107B700018E023E040E80012002AF2D1D4F8800097
:107B800068B198490165D4F88000FBF759FA0028DC
:107B900008D0D4F88000016DBDE8F04108472046C8
:107BA000FFF749FFBDE8F0812046FFF744FFF9E702
:107BB0002046FFF740FFC4F89060F3E7E76E012F1F
:107BC0007ED1C7067CD5CF067AD5102018622068F2
:107BD00080684FF02003400673D5D4F88020824996
:107BE000106888423AD080491831884236D07E49A0
:107BF0003031884232D07C49483188422ED07A498F
:107C0000603188422AD078497831884226D0764936
:107C10009031884222D07449A83188421ED07349DD
:107C200088421BD071491831884217D06F493031D2
:107C3000884213D06D49483188420FD06B4960317A
:107C400088420BD069497831884207D06749903122
:107C5000884203D06549A831884201D1406800E0DC
:107C6000406880B24FF4807760B3B4F85C10814212
:107C700040D9A4F85E00D069B84230D0206850E8FE
:107C8000001F21F4807140E80012002AF6D120681C
:107C9000083050E8001F21F0010140E80012002ADE
:107CA000F5D12068083050E8001F21F0400140E87D
:107CB0000012002AF5D1C4F88C30E666206802E094
:107CC00056E023E016E050E8001F21F0100140E8E4
:107CD0000012002AF2D1D4F88000FAF7F3FF2567EA
:107CE000B4F85C00B4F85E10401A81B22046FFF789
:107CF00041FE57E7B4F85C108142FAD1D069B8422E
:107D0000F7D125672046FFF735FE4BE734F85C0FC7
:107D10006188401A81B260885C3C0028E9D0002963
:107D2000E7D0206850E8002F22F4907240E8002746
:107D3000002FF6D1294FFF432068083050E8002F6C
:107D40003A4040E8002CBCF1000FF5D1C4F88C306B
:107D5000E6666667206850E8002F22F0100240E8CF
:107D60000023002BF6D125672046FFF703FE19E715
:107D7000C50209D5550207D54FF480101862204678
:107D8000BDE8F041FFF756BE03060CD501F08003B5
:107D900002F40002134306D0A16F0029A9D02046A7
:107DA000BDE8F0410847420606D54A0604D52046FC
:107DB000BDE8F04101F068BF020206D54A0004D5D3
:107DC0002046BDE8F041FFF734BEC00191D500293F
:107DD0008FDA2046BDE8F041FFF7DEBD010000105C
:107DE000200100042F9B00081000024010040240F4
:107DF00010B50446002C03D0D4F8880010B107E079
:107E0000012010BD002084F88400204600F028F8EE
:107E10002420C4F888002068016821F00101016075
:107E2000A06A10B1204601F0C9FD204601F056FFBE
:107E3000012813D02068416821F4904141602068F6
:107E4000816821F02A0181602068016841F0010108
:107E500001602046BDE8104001F014BE012010BDB5
:107E600070B5B8B00646142132A8F8F71DFCC02141
:107E700002A8F8F719FC2949306888424BD1012142
:107E80000020CDE902100025219502A8FDF700FE93
:107E900008B1F9F778FF2248016841F0100101604C
:107EA000006800F0100001901D481038016841F092
:107EB00001010160006800F0010001904FF4C06012
:107EC000329002203390349535950720369032A9B0
:107ED0001448FCF725FA154C1348206029206060EF
:107EE000A560E5604FF4806020616561A561E56192
:107EF000256265622046FBF7CFFD08B1F9F743FF25
:107F0000C6F88040A663002205212520FCF7CCFBA3
:107F10002520FCF7BBFB38B070BD0000001001400D
:107F2000F04402580000025888000240A0040024D7
:107F3000704770472DE9F84304460E4615461F4624
:107F4000D4F88800202802D00220BDE8F8838EB142
:107F500085B100201834A06721202067FCF700FBC2
:107F60008146A587E58754F8100C183CB0F5805F72
:107F700002D003E00120E8E7206920B13546002661
:107F80004FF0200817E00025FAE700224B46802139
:107F90002046009702F03CF918B1C4F8888003200D
:107FA000D3E7C5B1216815F8010B8862B4F8560013
:107FB000401EA4F85600B4F856000028E5D100226F
:107FC0004B4640212046009702F022F950B1C4F8F8
:107FD00088800320B9E7216836F8020BC0F3080057
:107FE0008862E3E7C4F888800020AEE77047FEE7C8
:107FF0008068C0F3C00070478068C0F3000070471D
:108000008068C0F380007047C06810F4406F01D0F2
:1080100000207047012070472DE9F05F2DED028BA5
:108020004FF00008DFF8049489F804804FF40054FE
:10803000204600F071FFFE480021FFF75BFBFD4882
:1080400000228021FCF77EFAFB4D002221112846F8
:10805000FCF778FA002221462846FCF773FA002242
:1080600028466100FCF76EFA0024F44DF44F4FF4FB
:10807000205AF44E4FF4806BA00089F80400EC48BD
:10808000B038FAF737FDEA4852462946B038FAF7D1
:10809000ABFCE0B2F8F70EFEC5F800800021E44822
:1080A0004C30FFF727FB4FF4FA7003F0DFFFE04896
:1080B00000214C30FFF7B2FB002000EB8001891C4F
:1080C00035F8211027F81010401C80B25845F4D321
:1080D000DB48594603F05CFF06EB840080ED000AA4
:1080E000002000EB8001891C55F82110090C27F8AD
:1080F0001010401C80B25845F3D3D148594603F0C4
:1081000047FF04F1080006EB800080ED000A002024
:1081100000EB800155F82110090C27F81010401CC5
:1081200080B25845F4D3C648594603F031FF04F1F4
:10813000100006EB800080ED000A002000EB8001BB
:1081400035F8211027F81010401C80B25845F5D39F
:10815000BB484FF4806103F01BFFBA4904F11800DB
:1081600001EB800080ED000A641CA4B2082C83D3CC
:10817000B14E00224FF400713046FCF7E3F9AD48F0
:1081800001228021FCF7DEF9012230465103FCF781
:10819000D9F9012230469103FCF7D4F900249FED70
:1081A000AA8AA84E4FF00109203EA0491E2000EBEC
:1081B000840008719E48B038FAF79CFC9F4D4FF43C
:1081C00020529B482946B038FAF70EFCE0B2F8F787
:1081D00071FDC5F80080002195484C30FFF78AFA00
:1081E0000025DFF854B24FF4804A00225146584629
:1081F000FCF7A8F9052003F039FF01225146584643
:10820000FCF7A0F9052003F031FF6D1CADB2322D53
:10821000EBD3874800214C30FFF700FB0020874D4F
:108220004FF4806B00EB8001891C35F8211027F892
:108230001010401C80B25845F4D38148594603F0D1
:10824000A7FE804901EB8400D0ED000AF4EEC00ADD
:10825000F1EE10FA02D230EE600A01E0B0EE480A08
:1082600080ED000A10EE100ADFF8E0A1504502DDB3
:1082700006F8049001E006F80480002000EB80017D
:1082800055F82110090C27F81010401C80B25845F1
:10829000F4D36B484FF4806103F07AFE694904F12E
:1082A000100001EB8000D0ED000AF4EEC00AF1EE00
:1082B00010FA02D230EE600A01E0B0EE480A80ED1A
:1082C000000A10EE100A6149884203DD301980F877
:1082D000109002E0301980F81080641CA4B2082CC1
:1082E000FFF463AF544C012251022046FCF72AF9F7
:1082F000504801228021FCF725F9002220464FF446
:108300000051FCF71FF9012220469103FCF71AF9EE
:10831000002446493C2000EB840008714448B038F2
:10832000FAF7E8FB42484FF420522946B038FAF7F2
:108330005BFBE0B2F8F7BEFCC5F8008000213C48CA
:108340004C30FFF7D7F94FF0000ADFF8E8B0012210
:1083500080215846FCF7F6F8052003F087FE00223E
:1083600058468021FCF7EEF8052003F07FFE0AF165
:10837000010A1FFA8AFABAF1320FE8D32C48002119
:108380004C30FFF74BFA00204FF4806100EB800285
:10839000921C55F82220120C27F81020401C80B2A5
:1083A0008842F3D326484FF4806103F0F1FDDFF8F3
:1083B00094B004F108000BEB8000D0ED000AF4EE5D
:1083C000C00AF1EE10FA02D230EE600A01E0B0EE1F
:1083D000480A80ED000A10EE100ADFF870A0504540
:1083E00003DD301980F8089002E0301980F8088029
:1083F00000204FF4806100EB800235F8222027F83E
:108400001020401C80B28842F5D30D4803F0C0FD17
:1084100004F118000BEB8000D0ED000AF4EEC00A66
:10842000F1EE10FA14D230EE600A13E0F8010024E5
:1084300074030024000C0258001802580010003881
:108440009005002430EA0024000000000000C8422B
:10845000B0EE480A80ED000A10EE100A504503DD28
:10846000301980F8189002E0301980F81880641CE8
:10847000A4B2082CFFF44DAF1A480021FFF7CEF943
:10848000194880F804900022184C80212046FCF7FF
:1084900059F84FF47A7003F0E9FD0122204680215B
:1084A000FCF750F8124800228021FCF74BF8114CE1
:1084B00000224FF400712046FCF744F800222046C9
:1084C0004FF40051FCF73EF8002220464FF4804163
:1084D000FCF738F8084864210171BDEC028BBDE857
:1084E000F09F0000740300240800002400200258BC
:1084F000000C025800180258F801002430B587B06B
:108500001C216846F8F7D0F850484F4901604FF4F5
:1085100000214160002484600125C56008210161BB
:10852000047544750A21816104774FF4B06141629A
:10853000A90281620321C16229030163446380F8B7
:108540003840C563FAF792F808B1F9F71CFC0095BA
:1085500006200190029440F2FF70039004200490E2
:1085600005948DF8194069463848F9F7B5FC08B10B
:10857000F9F709FC364800900C2001906946334811
:10858000F9F7AAFC08B1F9F7FEFB32480090122077
:10859000019069462D48F9F79FFC08B1F9F7F3FB04
:1085A0001820019029486946F9F796FC08B1F9F7B7
:1085B000EAFB294800904FF48070019069462348F7
:1085C000F9F78AFC08B1F9F7DEFB244800904FF474
:1085D0008370019069461D48F9F77EFC08B1F9F7F0
:1085E000D2FB1F4800904FF48670019069461748EF
:1085F000F9F772FC08B1F9F7C6FB1A4800904FF47E
:108600008970019069461148F9F766FC08B1F9F7DD
:10861000BAFB154800904FF48C70019069460B48E6
:10862000F9F75AFC08B1F9F7AEFB104800904FF487
:108630000070019069460548F9F74EFC002801D00A
:10864000F9F7A1FB07B030BD00600258C402002456
:10865000020030042000F0140004002A0008302E2C
:10866000002090360040C03A0080F03E00002143D8
:1086700008B50D48016841F400110160006800F47C
:1086800000100090002205218020FCF70DF88020CA
:10869000FBF7FCFF002205218120FCF705F8BDE86F
:1086A00008408120FBF7F2BFE044025808B51A48A1
:1086B000016841F002010160016801F002010091CE
:1086C000016841F001010160006800F001000090C4
:1086D00013481249016000214160802282609200AB
:1086E000C2605200026141618161C1610162042284
:1086F000426203228262C1620163FBF7CDF908B1D5
:10870000F9F741FB002205211020FBF7CDFFBDE862
:1087100008401020FBF7BABFD844025810040240AA
:10872000180500242DE9F04F87B0142102A8F7F7AF
:10873000BBFF4B48016841F020010160016801F076
:1087400020010191016841F080010160016801F0A0
:1087500080010191016841F004010160016801F0AC
:1087600004010191016841F001010160016801F01B
:1087700001010191016841F008010160016801F007
:1087800008010191016841F040010160016801F0B8
:1087900040010191016841F480710160006800F4BA
:1087A000807001900122DFF8BC801402404621460F
:1087B000FBF7C8FEDFF8B090E600002231464846DD
:1087C000FBF7C0FEDFF8A4A00022BF215046FBF754
:1087D000B9FEDFF89CB04FF4FC47002239465846FA
:1087E000FBF7B0FE234801228021FBF7ABFE029489
:1087F0000125039500240494059402A94046FBF743
:108800008FFD0296112603960494059402A948460A
:10881000FBF786FD3B20029003960494059402A981
:108820005046FBF77DFD8420029003950494059447
:1088300002A95046FBF774FD029703950494059432
:1088400002A95846FBF76CFD802002900395049422
:10885000059402A90748FBF763FD07B0BDE8F08F58
:10886000E04402580000025800080258000C025868
:10887000001802580020025830B599B00024159411
:108880001694179418941294139414941C210BA802
:10889000F7F70AFF2C216846F7F706FF2B482A490D
:1088A0000160EF21416084606321C1600461446123
:1088B00080258561FEF760FC08B1F9F764FA4FF492
:1088C00080501590214815A9FEF7F8FC08B1F9F77A
:1088D0005AFA1E48FEF7E4FE08B1F9F754FA2020D0
:1088E00012901394149512A91848FEF7F5FB08B1DD
:1088F000F9F749FA60200B9005200C900D940E9426
:108900000F9410941194002210480BA9FEF72DFE2D
:1089100008B1F9F738FA009401940294039404948E
:108920004FF40050059006940794000308900994B2
:108930000A9469460548FEF789FB002801D0F9F73B
:1089400022FA19B030BD00000000014028030024C5
:1089500030B58FB000240B940C940D940E940894B1
:1089600009940A941C2101A8F7F79EFE1E484FF0B7
:1089700080410160EF21416084606321C160046136
:1089800080258561FEF7F8FB08B1F9F7FCF94FF493
:1089900080500B9014480BA9FEF790FC08B1F9F732
:1089A000F2F91148FEF77CFE08B1F9F7ECF9202046
:1089B00008900A9508A90C48FEF78EFB08B1F9F754
:1089C000E2F9602001900294039405940022064885
:1089D00001A9FEF7CAFD08B1F9F7D5F90248FEF77B
:1089E0009BFD0FB030BD00007403002430B58FB084
:1089F00000240B940C940D940E94089409940A94FA
:108A00001C2101A8F7F750FE1E481D490160EF2107
:108A1000416084606321C160046180258561FEF747
:108A2000ABFB08B1F9F7AFF94FF480500B90154844
:108A30000BA9FEF743FC08B1F9F7A5F91148FEF7B9
:108A40002FFE08B1F9F79FF9202008900A9508A990
:108A50000C48FEF741FB08B1F9F795F96020019049
:108A600005200290039405940022064801A9FEF710
:108A70007CFD002801D0F9F786F90FB030BD000069
:108A800000080040C003002410B5174815490160D4
:108A90004FF4E131416000218160C16001610C222D
:108AA00042618161C161016241628162FFF7A0F9A7
:108AB00008B1F9F768F90C480021FEF794FF08B1F6
:108AC000F9F761F908480021FEF767FF08B1F9F7E7
:108AD0005AF90548FEF705FF002801D0F9F753F9C8
:108AE00010BD0000001001400C040024FEE7FEE76A
:108AF0000148FBF7FCBE000048ED002470B50446B9
:108B00002068056C00EB4110D0F8081B0C4EB542F4
:108B100005D9090403D54FF40041C0F8081B2046CD
:108B2000FCF7C0F9B54208D9A079012805D1206821
:108B3000012104F29C4202F0F7F9002070BD000010
:108B40000A30544F2DE9F04105460C462E68306C32
:108B500006EB4411D1F8083B4FF4004795F8068026
:108B600005F29C424FF0200CB8F1010F08D0DFF85D
:108B7000B080404545D118043AD5C1F8087B4CE097
:108B8000284E5FEA037806D5B04246D9180444D58A
:108B9000C1F8087B41E05FEA836802D5C1F808CBE1
:108BA0003BE013F0280F38D1B04204D9180402D5A5
:108BB000C1F8087B31E004EBC40005EB800000F550
:108BC0001570D1F8101B036AC1F31201591A4161E3
:108BD00024B903693BB1C2681144C1602846E1B2BF
:108BE000FBF7A2FD19E02868012102F09DF9F5E7E5
:108BF000980601D5C1F808CB2846E1B2FBF794FDF1
:108C00000BE034B9D5F8640218B90021304602F0FF
:108C10008BF92846E1B2FBF787FD0020BDE8F08123
:108C20000A31544F0A30544F2DE9F84F80460E4612
:108C3000D8F8007006EBC60008EB80041434D4E9C1
:108C40000410884202D90120BDE8F88F081AA168F3
:108C5000814200D20846C01C4FEA900A07EB461931
:108C600016E0151AA268AA4200D21546E81C4FEA7F
:108C7000900A98F806000090ABB2E1683846F2B26C
:108C800002F05AFCE0682844E060606928446061B2
:108C9000D9F8180980B2504505D3D4E90420904290
:108CA00001D2002ADDD1D4E90401884208D801208C
:108CB00006F00F018840D7F834188143C7F83418FC
:108CC0000020C1E72DE9F047044688460027DFF879
:108CD0001491D9F80000C043800709D0414D283DC8
:108CE000286820F080602860FBF73AFC064609E01F
:108CF0000120BDE8F087FBF733FC801B022801D977
:108D00000320F6E728680001F5D4D9F800002168AF
:108D100020F47C3040EA0130C9F80000A0884FF60A
:108D2000FF72A168401E491EC0F3080002EA4121FB
:108D30000843A1894FF4FE02491E02EA014108439B
:108D4000217C1202491E02EA0161084325491031C3
:108D500008602448001D0168626921F0C0011143C8
:108D600001600168A26921F02001114301600168DE
:108D700021F0100101601B4914310A684FF6F873A5
:108D80009A43E36942EAC3020A60016841F01001B4
:108D90000160B8F1000F0ED0B8F1010F10D00168DA
:108DA00041F400110160286840F080602860FBF702
:108DB000D7FB044610E0016841F400210160F2E7AE
:108DC000016841F480110160EDE7FBF7C9FB001B6E
:108DD000022801D903208CE728680001F5D5384620
:108DE00087E70000284402582DE9F04704468846EA
:108DF0000027DFF81491D9F80000C043800709D09C
:108E0000414D283D286820F080502860FBF7A8FBE2
:108E1000064609E00120BDE8F087FBF7A1FB801BB7
:108E2000022801D90320F6E728688000F5D4D9F894
:108E30000000218820F07C7040EA0150C9F8000051
:108E4000A0884FF6FF72A168401E491EC0F30800BB
:108E500002EA41210843A1894FF4FE02491E02EAB9
:108E600001410843217C1202491E02EA01610843C4
:108E70002549183108602448001D0168626921F401
:108E80004061114301600168A26921F4007111433E
:108E90000160016821F4807101601B491C310A687E
:108EA0004FF6F8739A43E36942EAC3020A60016825
:108EB00041F480710160B8F1000F0ED0B8F1010FDC
:108EC00010D0016841F080710160286840F0805046
:108ED0002860FBF745FB044610E0016841F480017F
:108EE0000160F2E7016841F400010160EDE7FBF782
:108EF00037FB001B022801D903208CE7286880007B
:108F0000F5D5384687E700002844025801784078B4
:108F100041EA00207047000030B58FB005460024BC
:108F20000B940C940D940E94089409940A941C21AB
:108F300001A8F7F7B9FB2249204A0A6064222148B8
:108F4000B0FBF5F0B0FBF2F0401E48608C6063208F
:108F5000C8600C6180258D610846FEF70DF908B1E7
:108F6000F8F711FF4FF480500B9015480BA9FEF74E
:108F7000A5F908B1F8F707FF1148FEF791FB08B112
:108F8000F8F701FF202008900A9508A90C48FEF781
:108F9000A3F808B1F8F7F7FE6020019005200290D1
:108FA000039405940022064801A9FEF7DEFA002882
:108FB00001D0F8F7E8FE0FB030BD00000008004017
:108FC000C0030024001C4E0E70B50546642003F05B
:108FD0004DF8694C062D04D2DFE805F0032241600C
:108FE0007F9E002220462021FBF7ACFA002220467B
:108FF0001021FBF7A7FA002220460821FBF7A2FA6E
:10900000002220460421FBF79DFA0022204602217F
:10901000FBF798FA002220460121FBF793FA99E02A
:10902000012220462021FBF78DFA00222046102144
:10903000FBF788FA002220460821FBF783FA00227A
:1090400020460421FBF77EFA002220460221FBF78E
:1090500079FA002220460121FBF774FA7AE0012216
:1090600020462021FBF76EFA002220461021FBF754
:1090700069FA012220460821FBF764FA0022204603
:109080000421FBF75FFA002220460221FBF75AFA7F
:10909000002220460121FBF755FA5BE00122204621
:1090A0002021FBF74FFA002220461021FBF74AFA55
:1090B000012220460821FBF745FA00222046042120
:1090C000FBF740FA012220460221FBF73BFA00227F
:1090D00020460121FBF736FA3CE001222046202100
:1090E000FBF730FA002220461021FBF72BFA002272
:1090F00020460821FBF726FA012220460421FBF72F
:1091000021FA012220460221FBF71CFA0022204608
:109110000121FBF717FA1DE0012220462021FBF771
:1091200011FA002220461021FBF70CFA00222046FB
:109130000821FBF707FA012220460421FBF702FA77
:10914000002220460221FBF7FDF9012220461146AC
:10915000FBF7F8F90122094DD40228462146FBF716
:10916000F1F9642002F082FF21462846BDE87040F4
:109170000022FBF7E7B90000000C02580008025873
:109180006748962101800821C1700022654880212E
:10919000FBF7D8F9644C00224FF400712046FBF72E
:1091A000D1F9002220464FF40051FBF7CBF9002201
:1091B00020464FF48041FBF7C5F95C480021FEF7DB
:1091C0002DFB0020FFF700FF59480088F7F702FE4B
:1091D00056480021FEF722FB41F2883002F046FF9C
:1091E000524840F2FF7400212246B038F8F722FEC0
:1091F0004E4822464FF00111B038F8F71BFE4B489D
:109200004FF420524B49B038F9F7EEFB4748802223
:1092100049499830FEF784FB44489830006801685B
:1092200041F01001016045484549006888423AD044
:1092300043491831884236D041493031884232D0D2
:109240003F49483188422ED03D49603188422AD07A
:109250003B497831884226D039499031884222D022
:109260003749A83188421ED0364988421BD035493B
:109270001831884217D033493031884213D03149F0
:10928000483188420FD02F49603188420BD02D4998
:109290007831884207D02B499031884203D0294940
:1092A000A831884204D1016821F00801016003E07F
:1092B000016821F00401016000220120114602F042
:1092C00045FF1B4C183C206100220120114602F092
:1092D0003DFFE06000211C4A1C4802F0BDFF1C4815
:1092E00000224FF48071FBF72DF91A4D00228021E6
:1092F0002846FBF727F94FF4FA7002F0B7FE012277
:1093000028468021FBF71EF94FF49675F7F7E4FD28
:10931000206902F075FF284602F0A8FEF6E700007B
:10932000F8010024000C02580018025874030024AD
:10933000200000240010003890250024A004002400
:10934000100002401004024064E1000815140008F7
:10935000000002580020025810B54FF0E0200069CC
:1093600004F068FC012803D0BDE8104003F0C4BF3E
:1093700010BD000030B59DB04C210AA8F7F794F954
:10938000202102A8F7F790F90220FBF7ABFD00249B
:109390002048016841F44041016001681E490A68A3
:1093A00042F001020A60096801F0010101910168BF
:1093B0008904FCD501200A9000040B900220139030
:1093C000149005211591C021169117900F21189125
:1093D000199008251A951B941C940AA8FDF7E8FA21
:1093E00008B1F8F7D0FC3F200290032003900494CA
:1093F00005954020069007900101089109900421ED
:1094000002A8FDF747F8002801D0F8F7BCFC1DB012
:1094100030BD0000184802582C04005810B52C48E4
:10942000016841F4700101602A4A106800F00F00E1
:10943000072804D2106820F00F00C01D10602649D4
:10944000086840F001000860234B002010331860CA
:109450000B68224C23400B60136803F00F03072BAB
:1094600004D9136823F00F03DB1D13601A4A183266
:109470001060121D1060121D1060174B184A28331F
:109480001A601B1D174A1A601B1D174A1A601B1D04
:1094900018601B1D1A601B1D18601B1D1A601A1D09
:1094A00010600A6822F480220A600B49603108606B
:1094B0000E4800686FF30F00B0F1005F02D20C4954
:1094C0000120086043F2D2000A49086010BD000084
:1094D00088ED00E000200052004402587FEDF6EADB
:1094E000000202020000FF01800201010010005C86
:1094F00008810051004000520148FDF764BF0000A0
:109500002CF200242DE9F04F02684FF0804A274DDD
:10951000274E284FA842DFF8A0C0284B09D050455D
:1095200007D0B04205D0B84203D0604501D0984280
:1095300003D122F070044A682243DFF88480DFF808
:109540008490A842DFF880B00FD050450DD0B042D3
:109550000BD0B84209D0604507D0984205D04045AD
:1095600003D0484501D0584503D122F44074CA685D
:1095700022434C6922F0800222438C68C4620C684A
:109580008462A84207D0984205D0404503D04845A0
:1095900001D0584501D109690163016841F0040116
:1095A0000160012141610260BDE8F08F00000140CF
:1095B0000004004000080040000C0040000401408E
:1095C00000400140004401400048014010B5012323
:1095D00001F01F018B40046A9C430462036A8A40C5
:1095E0001343036210BD10B5846824F47F4442EA3B
:1095F00003220A432243826010BD00008268034BAD
:109600001A400A4342F00701816070478FFFCFFF85
:109610002DE9F043046A026A22F001020262426804
:1096200083691D4D2B4023F003030D681D4324F077
:1096300002048B682343194E194FDFF868C0B0420B
:10964000DFF86480DFF8649007D0B84205D0604549
:1096500003D0404501D0484505D123F00804CB682C
:10966000234323F00403B04207D0B84205D060453D
:1096700003D0404501D0484507D122F4807222F43E
:1096800000724C6914438A692243426085614968CB
:1096900041630362BDE8F0838FFFFEFF00000140DD
:1096A00000040140004001400044014000480140E6
:1096B000F0B5056A026A22F010020262426883690C
:1096C0001A4C234023F440730C6843EA042425F029
:1096D00020038D6843EA0513154D164EA84201D0AC
:1096E000B04206D123F08003CF6843EA071323F08A
:1096F0004003A8420AD0B04208D00F4DA84205D07E
:109700000E4DA84202D00E4DA84209D122F480622B
:1097100022F400624D6942EA85028D6942EA8502BF
:1097200042608461496881630362F0BDFF8FFFFE80
:10973000000001400004014000400140004401409D
:1097400000480140F0B5056A026A22F480720262A4
:109750004268C3691A4C234023F003030C681C437E
:1097600025F400738D6843EA0523164D164EA84272
:1097700001D0B04206D123F40063CF6843EA072347
:1097800023F48063A8420AD0B04208D00F4DA8420B
:1097900005D00F4DA84202D00E4DA84209D122F4A7
:1097A000805222F400524D6942EA05128D6942EA64
:1097B00005124260C4614968C1630362F0BD0000E4
:1097C0008FFFFEFF00000140000401400040014007
:1097D000004401400048014030B5046A026A22F4A6
:1097E000805202624268C369124D2B4023F44073D9
:1097F0000D6843EA052324F400548D6844EA0534D7
:109800000D4DA8420BD00D4DA84208D00C4DA842DA
:1098100005D00C4DA84202D00B4DA84204D122F431
:1098200080424D6942EA85124260C3614968016421
:10983000046230BDFF8FFFFE0000014000040140C4
:1098400000400140004401400048014030B5056A35
:10985000026A22F4803202624268436D114C234056
:109860000C681C4325F400330D8943EA05430E4D73
:10987000A8420BD00D4DA84208D00D4DA84205D0EE
:109880000C4DA84202D00C4DA84204D122F48032E3
:109890004D6942EA05224260446549688165036278
:1098A00030BD00008FFFFEFF0000014000040140BA
:1098B00000400140004401400048014030B5056AC5
:1098C000026A22F4801202624268436D114C234006
:1098D0000C6843EA042425F400130D8943EA055378
:1098E0000D4DA8420BD00D4DA84208D00C4DA842FA
:1098F00005D00C4DA84202D00B4DA84204D122F451
:1099000080224D6942EA8522426044654968C1650A
:10991000036230BDFF8FFFFE0000014000040140E4
:1099200000400140004401400048014010B5036A76
:10993000046A24F001040462846924F0F00444EA17
:10994000021423F00A020A438461026210BD10B5BA
:10995000036A046A24F010040462846924F47044E5
:1099600044EA023223F0A00343EA0111826101625A
:1099700010BD000030B5416E002917D00268916813
:10998000C1F342619268520F0B4B9C5C250103F1BD
:109990000804A25CB5FBF2F2A0F86A205A5C615C94
:1099A0001201B2FBF1F1A0F8681030BD012168305E
:1099B0004180018030BD000014E7000890F82810B5
:1099C000090706D501684A68836B22F400421A43EE
:1099D0004A6090F82810C90706D001684A68C36A2F
:1099E00022F400321A434A6090F82810890706D5FD
:1099F00001684A68036B22F480321A434A6090F887
:109A00002810490706D501684A68436B22F4802272
:109A10001A434A6090F82810C90606D501688A687A
:109A2000C36B22F480521A438A6090F8281089068A
:109A300006D501688A68036C22F400521A438A60D2
:109A400090F82810490611D501684A68436C22F441
:109A500080121A434A60416CB1F5801F06D101683B
:109A60004A68836C22F4C0021A434A6090F82810B6
:109A7000090606D501684A68C06C22F40022024338
:109A80004A6070472DE9F84304460025C4F8905019
:109A9000FAF766FD8046206800686FF07E474FF059
:109AA0002006000716D500224346310420460097C1
:109AB00000F0AEFB70B1206850E8001F21F080017B
:109AC00040E80012002AF6D1843466602570032035
:109AD000BDE8F88320680068400720D5002243468F
:109AE0004FF480012046009700F092FBB8B1206847
:109AF00050E8001F21F4907140E80012002AF6D1CE
:109B00002068083050E8001F21F0010140E80012F1
:109B1000002AF5D18434A66025700320D8E76C3480
:109B2000E66126622560656025760020D0E710B5E5
:109B3000806B0021A0F85E10FDF77DFF10BD70B5B1
:109B4000846BD4F88800D4F88C50216889684FF071
:109B50000006090606D5212804D1A4F8566020463F
:109B600000F0A4F820688068400606D5222D04D1B4
:109B7000A4F85E60204600F05DF8D4F8900040F054
:109B80001000C4F890002046FDF755FF70BD014657
:109B900010B5886B0023C969B1F5807F2DD0A0F87E
:109BA0005E30016851E8002F22F4807241E8002401
:109BB000002CF6D10168083151E8002F22F0010293
:109BC00041E80024002CF5D10168083151E8002F4C
:109BD00022F0400241E80024002CF5D12021C0F8F9
:109BE0008C10C16E012908D1016851E8002F22F0C4
:109BF000100241E80024002CF6D10367C16E012950
:109C000002D0FEF795F910BDB0F85C10FDF7B2FE7A
:109C100010BD10B5806B01210167C16E012902D012
:109C2000FEF787F910BDB0F85C104908FDF7A2FEF9
:109C300010BD000010B5016851E8002F22F49072A9
:109C400041E80023002BF6D10E4B0168083151E8A2
:109C5000002F1A4041E80024002CF6D1C16E0129E2
:109C600008D1016851E8002F22F0100241E80023DA
:109C7000002BF6D12021C0F88C100021C16641676D
:109C800010BD0000FEFFFFEF10B5016851E8002F86
:109C900022F0400241E80023002BF6D12021C0F839
:109CA000881000218167FEF7A1F910BD016851E815
:109CB000002F22F0C00241E80023002BF6D10168FA
:109CC000083151E8002F22F4000241E80023002B64
:109CD000F5D12021C0F88810704700002DE9F0432D
:109CE00087B004460025DFF8F88320682269A16860
:109CF000E369114362691A4311430268F94B1A4040
:109D00000A43026020684168E26821F4405111432F
:109D10004160A0692168414501D0226A10438A68E8
:109D2000F14B1A4002438A602068C16A626A21F0DE
:109D30000F011143C162ED492268ED488A421DD1ED
:109D4000006800F03800182812D005DC50B108284F
:109D50000AD0102804D109E020280BD028280BD0E5
:109D60008021EBE00121E9E00421E7E00821E5E0C2
:109D70001021E3E02021E1E04021DFE0DD498A42DB
:109D800017D1006800F00700062810D2DFE800F0C5
:109D9000030507090B0D0021D0E00421CEE00821C6
:109DA000CCE01021CAE02021C8E04021C6E080219B
:109DB000C4E0D1498A4217D1006800F007000628A4
:109DC00010D2DFE800F0030507090B0D0021B5E014
:109DD0000421B3E00821B1E01021AFE02021ADE083
:109DE0004021ABE08021A9E0C4498A4217D1006834
:109DF00000F00700062810D2DFE800F0030507098D
:109E00000B0D00219AE0042198E0082196E0102132
:109E100094E0202192E0402190E080218EE0B8493A
:109E20008A4217D1006800F00700062810D2DFE848
:109E300000F0030507090B0D00217FE004217DE000
:109E400008217BE0102179E0202177E0402175E0B6
:109E5000802173E0AB498A421DD1006800F03800D0
:109E6000182812D005DC50B108280AD0102804D1D7
:109E700009E020280BD028280BD080215EE00121AA
:109E80005CE004215AE0082158E0102156E020212E
:109E900054E0402152E09C498A4217D1006800F00A
:109EA0000700062810D2DFE800F0030507090B0DB4
:109EB000002143E0042141E008213FE010213DE082
:109EC00020213BE0402139E0802137E08F498A4260
:109ED00017D1006800F00700062810D2DFE800F074
:109EE000030507090B0D002128E0042126E00821C5
:109EF00024E0102122E0202120E040211EE08021EA
:109F00001CE0424519D17A48001D006800F00700A6
:109F1000062810D2DFE800F0030507090B0D022127
:109F20000CE004210AE0082108E0102106E02021CD
:109F300004E0402102E0802100E0802174486C4B65
:109F40000027744E4FF40049543B42454FEA201C11
:109F500053D110292AD006DC02291AD004291BD09B
:109F6000082904D11DE0202928D0402928D000202C
:109F70000125E8B3616A36F81120B0FBF2F166689A
:109F800006EB46038B4202D8B1EB063F1AD90125F6
:109F9000E2E0FAF7D3FFECE704A8FBF7C1F8059875
:109FA000E7E701A8FBF79CF90298E2E71968890640
:109FB000DFD51968C1F3C101C840DAE76046D8E7C8
:109FC0004846D6E700231946F6F756FA0902020278
:109FD00041EA106170081018324679410023F6F703
:109FE0004BFA4D4AA0F54071914204D8216800E037
:109FF0004AE0C860B0E00125AEE0E2694FF6EF78D4
:10A000004A4548D1082932D005DC29B3012926D098
:10A01000042906D126E010292ED0202935D0402948
:10A0200035D00020012578B3616A36F81110B0FBF5
:10A03000F1F04100606801EB5001B1FBF0F0A0F1DC
:10A040001001414525D84FF6F0710140C0F34200A0
:10A0500001432068C1607FE0FCF7ACFBE3E7FCF75D
:10A06000BBFBE0E704A8FBF75BF80598DBE701A87A
:10A07000FBF736F90298D6E719688906D3D519682F
:10A08000C1F3C101C840CEE748E06046CBE748468F
:10A09000C9E7012560E008294CD005DCF9B10129A8
:10A0A00040D0042906D140E0102948D020294ED0C4
:10A0B00040294ED00020012580B3616A36F8111086
:10A0C000B0FBF1F1606801EB5001B1FBF0F0A0F1E1
:10A0D000100141453FD8216880B2C8603CE01EE0D5
:10A0E000000C0058F369FFCFFFF4FF11001001408E
:10A0F000544402580044004000480040004C0040D6
:10A10000005000400014014000780040007C0040F6
:10A110000090D003FCE60008FFFC0F001CE0FCF7F9
:10A1200049FBC9E7FCF758FBC6E704A8FAF7F8FFB4
:10A130000598C1E701A8FBF7D3F80298BCE71968B6
:10A140008906B9D51968C1F3C101C840B4E76046B2
:10A15000B2E74846B0E701250120683460802080DE
:10A16000E760276107B02846BDE8F08370B5044674
:10A1700044F8581FA2800021A16322206063A06AD6
:10A18000583C00281DD01F4BC363241D1E48E36F9D
:10A190001864E36F1D48D864E06F0165134654F8F6
:10A1A000041CE56F606D2431241F02462846F9F730
:10A1B00041FF30B110208C346060202020600120ED
:10A1C00070BD206940B1206850E8001F41F48071E3
:10A1D00040E80012002AF6D12068083050E8001F3D
:10A1E00041F0010140E80012002AF5D12068083052
:10A1F00050E8001F41F0400140E80012002AF5D16C
:10A20000002070BD8F9B0008139C00083F9B000836
:10A210002DE9F04704460D4617469846089E4FF034
:10A22000000935E0701C33D0FAF79AF9A0EB08006A
:10A23000B04219D8C6B120680168490728D5802DD9
:10A2400026D0402D24D0C169C94309070ED4206807
:10A25000082505622046FFF7EDFCC4F8905084F80D
:10A2600084900120BDE8F0870320FBE7C069C0436C
:10A2700000050DD421684FF4006008622046FFF706
:10A28000D9FC2020C4F8900084F884900320E9E7EA
:10A290002068C06935EA000004D00020B842C1D06F
:10A2A0000020DFE70120F9E710B50548FDF7CAFBFC
:10A2B000BDE81040034980220148FDF731BB000092
:10A2C0000C0400249025002410B50024D0F8B822F6
:10A2D0005268904700B10324204610BD90F89C229C
:10A2E000012A05D0022A03D0032A01D000F01DB8AC
:10A2F0004988012904D10021C0F8A41200F039B81E
:10A300007047002070470020704710B513460A467A
:10A31000002100F0ABFA002010BD10B513460A462C
:10A32000002100F045FB002010BD10B5044680213F
:10A33000204600F027FB2046BDE81040002100F039
:10A3400021BB10B50521C0F8941200231A46194606
:10A3500000F08CFA002010BD10B50223C0F8943232
:10A360008261C26113460A46002100F021FB0020F1
:10A3700010BD10B50421C0F8941200231A461946E6
:10A3800000F016FB002010BD0A46D188012902D03A
:10A390001146FFF7CABF90F89C12012906D0022986
:10A3A00004D0032909D01146FFF7BFBF0021816007
:10A3B000012200F10801FFF7CFBF0122011DFFF7C5
:10A3C000CBBF2DE9F84304460F460020009000263D
:10A3D00000257988080A062870D006DC01282FD0CD
:10A3E000022835D0032804D148E0072867D00F2879
:10A3F00017D039462046FFF798FF0125002D0ED1D2
:10A40000FA88002A71D0BDF8000000286ED0824280
:10A4100000D90246009231462046FFF79DFFBDE875
:10A42000F883D4F8B402C26922B1207C694690470F
:10A430000646E3E739462046FFF777FF0125DDE7CB
:10A44000D4F8B412207C0A68694690470646D5E7DE
:10A45000207C4FF0020840B1D4F8B802C16A6846C7
:10A460008847064686F80180C8E7D4F8B802816AB2
:10A4700068468847064686F80180BFE7C8B20628C6
:10A4800062D2DFE800F0031223344352D4F8B4025E
:10A49000426822B1207C694690470646AEE73946BD
:10A4A0002046FFF742FF0125A8E7D4F8B4028268EE
:10A4B00032B1207C6946904706469FE74AE058E063
:10A4C00039462046FFF731FF012597E7D4F8B4025B
:10A4D000C26822B1207C6946904706468EE739461D
:10A4E0002046FFF722FF012588E758E052E0D4F824
:10A4F000B402026922B1207C6946904706467DE796
:10A5000039462046FFF711FF012577E7D4F8B4025A
:10A51000426922B1207C6946904706466EE739467B
:10A520002046FFF702FF012568E7D4F8B4028269EC
:10A5300022B1207C6946904706465FE739462046AF
:10A54000FFF7F3FE012559E739462046FFF7EDFEF8
:10A55000012553E7207C28B139462046FFF7E5FE68
:10A5600001254BE7D4F8B802416B68468847064698
:10A5700044E7207C28B139462046FFF7D6FE012566
:10A580003CE7D4F8B802016B6846884706460721C5
:10A59000717033E739462046FFF7C7FE3FE7204694
:10A5A000FFF7E7FE3BE70A4690F89C12012906D028
:10A5B000022904D0032902D01146FFF7B6BED18884
:10A5C000022902D01146FFF7B0BE0121C160D0F8C8
:10A5D000A41209B10321C160022200F10C01FFF7AE
:10A5E000BBBE01460020002906D0012905D0022962
:10A5F00005D0032905D003207047032070470120B0
:10A6000070470320704710B5D0F8C802FAF7A9F8D0
:10A61000BDE81040FFF7E5BF70B504460B4616468F
:10A62000002B08D043F080012046FFF76AFEFF2888
:10A630005ED078B35CE004F11400D4F894120025E5
:10A6400002293CD1D0E902218A420CD9521A8260F7
:10A6500031462046FFF761FE002320461A46194680
:10A6600000F004F92BE0914215D14068884212D3E2
:10A67000D4F8981288420ED2002220461146FFF7E5
:10A680004CFEC4F8985200231A461946204600F0A2
:10A69000EDF814E01CE094F89C02032808D1D4F8EB
:10A6A000B802C16821B1C4F8D452C16820468847B5
:10A6B0008021204600F066F92046FFF742FE94F81C
:10A6C000A002A8B1204600F095F984F8A0520FE04E
:10A6D00094F89C1203290BD1D4F8B8124A693AB104
:10A6E000C4F8D40220464A6919469047002800D190
:10A6F000002070BD70B504460B4615460022002BA5
:10A7000008D003F07F012046FFF7FBFDFF2854D05F
:10A7100078B352E004F5AA70D4F8941203294CD10E
:10A72000D0E902218A420AD9521A8260C068824264
:10A7300000D3024629462046FFF7E7FD3DE094F8A6
:10A74000AA0210F01F0006D0012806D002280AD065
:10A75000002078B11BE00020FBE794F8AE12204601
:10A76000FFF7D1FDF5E794F8AE122046FFF7C9FDDB
:10A77000EFE710E094F89C12032908D1D4F8B8123E
:10A780000A6922B1C4F8D4022046096988472046E4
:10A79000FFF7EFFD11E094F89C1203290AD1D4F8D9
:10A7A000B8128D6935B1C4F8D40220468A691946B9
:10A7B000904702460AB1104670BD002070BD0020CF
:10A7C000704710B50024012180F89C12D0F8B822FF
:10A7D000002A04D052680179904700B10324204632
:10A7E00010BD0A06D0F8C80201F07F0101EBC101DB
:10A7F00000EB810001D5807D704790F856027047CC
:10A8000010B5D0F8D42200EB8202D2F8B822002A88
:10A8100004D090F89C32032B02D004E0032010BD3A
:10A82000126A02B19047002010BD10B5D0F8D422B2
:10A8300000EB8202D2F8B822002A04D090F89C32B1
:10A84000032B02D004E0032010BD526A02B19047EE
:10A85000002010BD10B514461A46D0F8C802234691
:10A86000F9F7ABFFBDE81040FFF7BBBE10B5D0F85D
:10A87000C802F9F7D2FFBDE81040FFF7B2BE2DE9DC
:10A88000F04104460025012684F89C620020C4F8AB
:10A8900094026060C4F8A40284F8A002D4F8B8025C
:10A8A000002806D0426822B100212046904700B11E
:10A8B00003252046002240231146FFF7CBFFA4F8D2
:10A8C00064614027C4F86071402300222046802143
:10A8D000FFF7C0FFA68427622846BDE8F08190F804
:10A8E0009C12042903D190F89D1280F89C1200203C
:10A8F000704710B590F89C12032905D1D0F8B81212
:10A9000011B1C96901B18847002010BD0174002050
:10A91000704710B5D0F8C802FAF7B1FABDE8104098
:10A92000FFF75FBE70B5044604F2AA20054600F0AA
:10A9300048F80120C4F89402B4F8B002C4F89802B0
:10A9400094F8AA2212F01F000AD001280ED0022883
:10A9500012D02046BDE8704002F0800100F012B82D
:10A9600029462046BDE8704000F0FCB82946204644
:10A97000BDE8704000F041BA29462046BDE870406D
:10A9800000F02BB910B5D0F8C802F9F75FFFBDE8A9
:10A990001040FFF726BE90F89C12042903D090F8CF
:10A9A0009C1280F89D12042180F89C1200207047B0
:10A9B00010B5D0F8C802F9F781FFBDE81040FFF7E5
:10A9C00010BE70B504460846017821704178801C9D
:10A9D000617005462846FEF799FA60802846851C76
:10A9E0002846FEF793FAA0802846801CFEF78EFAD0
:10A9F000E08070BD0020704770B50446888800284C
:10AA000021D1C888F8B9488880281CD200F07F0579
:10AA100094F89C0203280DD084F89E5229462046C3
:10AA2000FFF777FF2046FFF7A4FC45B1022084F82A
:10AA30009C0270BD2046BDE87040FFF776BC012047
:10AA400084F89C0270BD2046BDE87040FFF76DBCE5
:10AA500003460020D3F8B822002A02D01268184614
:10AA6000104770472DE9F04104460F460025334E4C
:10AA7000B9783170012906D939462046FFF755FCCF
:10AA80000320BDE8F08194F89C024FF002080228F0
:10AA90000CD0032824D039462046FFF746FC3178F5
:10AAA0002046FFF711FC03252846EAE7A1B16160C3
:10AAB0002046FFF7CDFF0546280006D03946204640
:10AAC000FFF733FC84F89C82EEE72046FFF751FC49
:10AAD000032084F89C02E7E72046FFF74AFCE3E7FF
:10AAE000C9B16068884224D0C1B22046FFF7ECFBB0
:10AAF000317861602046FFF7ABFF0546280014D08F
:10AB000039462046FFF711FC21792046FFF7DCFB90
:10AB100084F89C82C8E784F89C8261602046FFF735
:10AB2000D3FB2046FFF725FCBEE72046FFF721FCBC
:10AB3000BAE72046FFF71DFCB6E7000078010024C5
:10AB40004A88012A03D0022A06D0FFF7EEBB012172
:10AB5000C0F8A412FFF70DBC8988090A80F8A0127A
:10AB6000FFF707BC10B500240A7812F0600211D07C
:10AB7000202A05D0402A03D0FFF7D7FB204610BD7E
:10AB8000D0F8D42200EB8202D2F8B8229268904723
:10AB90000446F3E74A780A2A1CD2DFE802F01218CA
:10ABA0001B151B08051B0F0BFFF70BFCE6E7FFF758
:10ABB00023FFE3E7FFF756FF0446DFE7FFF7E4FB79
:10ABC000DCE7FFF7F0FCD9E7FFF7BAFFD6E7FFF7BE
:10ABD00085FBD3E7FFF7A9FBD0E72DE9F041054658
:10ABE0000E4600273479307810F060001ED02028FF
:10ABF00008D0402806D031462846FFF796FB384655
:10AC0000BDE8F08121462846FFF77BFBFF28F6D000
:10AC10000028F4D1C5F8D402D5F8B8028268002A19
:10AC2000EDD03146284690470746E8E7707800287F
:10AC300070D0012831D0032804D031462846FFF7D0
:10AC400074FBDCE795F89C02022806D0032815D097
:10AC500031462846FFF769FBD1E754B1802C08D074
:10AC600021462846FFF78EFE80212846FFF78AFE00
:10AC7000C5E731462846FFF758FBC0E7708840B962
:10AC80003CB1802C05D0F08818B921462846FFF742
:10AC900079FE2846FFF76DFBB1E795F89C02022884
:10ACA00006D0032815D031462846FFF73EFBA6E71D
:10ACB00054B1802C08D021462846FFF763FE80213E
:10ACC0002846FFF75FFE9AE731462846FFF72DFB3F
:10ACD00095E77088002892D1600603D02146284667
:10ACE000FFF791FC2846FFF744FB21462846FFF773
:10ACF00008FBFF2883D0002881D1C5F8D402D5F8FD
:10AD0000B8028268002A90D031462846904707460C
:10AD100075E7FFE795F89C024FF00008022806D07F
:10AD2000032825D031462846FFF7FFFA67E734B1FC
:10AD3000802C04D031462846FFF7F7FA5FE720065B
:10AD400007D504F07F0000EB800005EB8001143193
:10AD500007E004F07F0000EB800005EB800101F5C7
:10AD6000AA71C1F8008002222846FFF7F5FA46E7EB
:10AD700020060CD504F00F0000EB800005EB8000EE
:10AD8000808C68B931462846FFF7CFFA37E704F0E0
:10AD90000F0000EB800005EB8000B0F8640148B1C3
:10ADA00020060CD504F07F0000EB800005EB800648
:10ADB00014360CE031462846FFF7B7FA1FE704F0D7
:10ADC0007F0000EB800005EB800606F5AA764CB10B
:10ADD000802C07D021462846FFF703FD28B101202B
:10ADE000306004E0C6F8008001E0C6F8008002226E
:10ADF00031462846FFF7B0FA01E770B505460E4622
:10AE00000024307810F0600009D0202807D04028B6
:10AE100005D031462846FFF788FA204670BD95F8E0
:10AE20009C02012808D0022806D0032804D031460D
:10AE30002846FFF77AFAF0E7B088C1B201291ED898
:10AE4000C1B22846FFF75FFAFF2800D048B10324BB
:10AE5000F0880028E1D1002CDFD12846FFF789FADD
:10AE6000DBE7D5F8B8128A683AB1C5F8D4022846AB
:10AE70008A68314690470446EAE70324E8E731460A
:10AE80002846FFF752FAC8E770B50A7801234E78D2
:10AE900002F00F041C4DA340012E19D0D0F81C481D
:10AEA00044EA0343C0F81C3800EB4210D0F8002BF2
:10AEB00012040BD4D0F8002B0B890979C3F30A03D1
:10AEC0001A4345EA81410A43C0F8002B002070BDB7
:10AED000D0F81C489BB21C43C0F81C4800EB421041
:10AEE000D0F800391B04F1D4D0F800390C89097965
:10AEF000C4F30A048904234341EA82510B432B43E0
:10AF0000C0F80039E2E7000000800010D0F8001916
:10AF10006FF30A01C0F80019D0F8041841F48071E9
:10AF2000C0F804180020704710B5036C124CA342FF
:10AF300005D9D0F8003B002B01DA002010BD00F548
:10AF4000316000230360036843F400230360036857
:10AF500043F018030360036843F0C0430360A0F5A7
:10AF60003160012906D100F530604261016841F08D
:10AF700080210160002010BD0A30544F0B784A78C0
:10AF8000012A00EB43100BD0D0F8002B22F4001262
:10AF9000C0F8002B0979032914D0022912D017E038
:10AFA000D0F8002922F40012C0F8002909790329F9
:10AFB00001D002290CD1D0F8001941F08051C0F81D
:10AFC000001905E0D0F8001B41F08051C0F8001BCB
:10AFD000002070470A784B780978012B00EB41106C
:10AFE00012D0D0F8001B002906DB2AB1D0F8001BD4
:10AFF00021F08041C0F8001BD0F8001B41F4001183
:10B00000C0F8001B00207047D0F80019002906DBAB
:10B010002AB1D0F8001921F08041C0F80019D0F809
:10B02000001941F40011C0F80019EBE7F8B50C78ED
:10B030006FF060460B784F78904D012F00EB431373
:10B0400029D0D3F8107B6FF31207C3F8107BD3F825
:10B05000107B2F40C3F8107B002C7DD00D69002D94
:10B060007BD08C6825446D1EB5FBF4F5ADB26C4306
:10B070000C62D3F8104B06EAC5452C43C3F8104BBD
:10B08000D3F8104B0D6AC5F312052C43C3F8104BCF
:10B09000012A6FD0D6E00F69EFB1D3F810796FF3C2
:10B0A0001207C3F81079D3F810792F40C3F810793C
:10B0B000FCB10F698D682F447F1EB7FBF5F5ADB26B
:10B0C000D3F8107906EAC5463743C3F810790E79EC
:10B0D000012E1AD028E003F511631E682E401E6071
:10B0E0001D6845F400251D601D686FF312051D6085
:10B0F00022E00E698D68AE4200D90D61D0F810597A
:10B1000045F40026C0F810690EE0D3F8106926F067
:10B11000C046C3F81069D3F810694FF0C04707EA7A
:10B1200045752E43C3F81069D3F810590E69C6F35C
:10B1300012063543C3F81059012A1CD000EB441302
:10B14000D3F8004944F00444C3F800490C79012CB9
:10B1500038D00A69002A01E04DE060E009D0D0F85B
:10B160003428097801F00F03012199400A43C0F8FF
:10B17000342881E062E0CA691AB100EB4413C3F8D5
:10B1800014290979012914D1D0F80818C90508D45F
:10B1900000EB4411D1F8002942F00052C1F8002917
:10B1A00007E000EB4411D1F8002942F08052C1F8C9
:10B1B000002900EB4410D0F8001941F00441C0F818
:10B1C000001959E0D0F80848E40506D4D3F800493E
:10B1D00044F00054C3F8004905E0D3F8004944F0B6
:10B1E0008054C3F8004900920A8A93B20A78C96869
:10B1F00000F0A2F940E00C690CB18C680C618C681D
:10B200000C62D0F8105BC4F312042543C0F8105B45
:10B21000D0F8104B44F40024C0F8104B38E7D3F8B2
:10B22000104B8D68C5F312052C43C3F8104BD3F8AF
:10B23000104B44F40024C3F8104B29E7CA680AB144
:10B24000C3F8142B0979012910D1D0F80808C005DA
:10B2500006D4D3F8000B40F00050C3F8000B05E013
:10B26000D3F8000B40F08050C3F8000BD3F8000B6C
:10B2700040F00440C3F8000B0020F8BDFFFF07E0DA
:10B2800038B5002200920B784D7800EB431442F25F
:10B290001073012D1AD0D4F8005B002D40DAD4F8D9
:10B2A000005B45F00065C4F8005B0C7800EB4414CB
:10B2B000D4F8005B45F08045C4F8005B009C641C3A
:10B2C0000094009C9C4224D9012229E0D4F8005922
:10B2D000002D25DAD4F8005945F00065C4F800596E
:10B2E0000C7800EB4414D4F8005945F08045C4F8BC
:10B2F0000059009C641C0094009C9C4201D90122CE
:10B300000EE00C7800EB4414D4F80049002CF0DB7C
:10B3100006E00C7800EB4414D4F8004B002CCDDB95
:10B32000104638BD18B5002400944FF07063009AA1
:10B33000521C0092009A9A4201D9032018BD02695A
:10B34000002AF4DA0094202242EA81110161009976
:10B35000491C00910099994201D9032018BD016947
:10B360008906F4D4002018BDD0F8080800F00600C3
:10B37000002805D0022805D0062803D00F207047EA
:10B380000020704702207047406900F001007047BC
:10B39000D0F81818D0F81C08084080B27047D0F8D0
:10B3A0001818D0F81C080840000C704710B5D0F8E9
:10B3B0001038D0F8342801F00F04E24002F0010206
:10B3C00043EAC21200EB4110D0F80809104010BD4A
:10B3D00000EB4111D1F8081BD0F814080840704761
:10B3E000416980690840704730B5034608469408B3
:10B3F00002F00301002203F5805303E01D6840F8CA
:10B40000045B521CA242F9D300290BD000221C6815
:10B41000D50024FA05F300F8013B521C491E89B2FD
:10B420000029F5D130BD00F50060026822F4FE620B
:10B43000026002684FF4FE6303EA01110A430260EE
:10B4400000207047022A0ED082B30921C26822F47C
:10B450007052C260C2684FF4705303EA81210A43FC
:10B46000C26000207047224A224B0A449A4201D20D
:10B470000F21EBE7204A214B0A449A4201D20E21C8
:10B48000E4E71F4A1F4B0A449A4201D20D21DDE72F
:10B490001D4A1E4B0A449A4201D20C21D6E71C4A8F
:10B4A0001C4B0A449A4202D20B21CFE71DE01A4AF4
:10B4B0001A4B0A449A4201D20A21C7E7184A194B8B
:10B4C0000A449A4201D20921C0E7174A174B0A449D
:10B4D0009A4201D20821B9E7154A1144154A91420E
:10B4E00001D20721B2E70621B0E70921AEE700004B
:10B4F000405327FF00350C00401E1BFF40420F0049
:10B5000000DC0BFF804F1200808CF9FE20D6130068
:10B5100060B6E5FE60E3160000D3CEFE40771B0068
:10B52000C05BB3FEC091210000CA91FE20753800B7
:10B53000E05459FEE09C410010B5029C002C0DD156
:10B54000DB1C9C08002300EB023000F5805003E078
:10B5500051F8042B02605B1CA342F9D3002010BDFC
:10B56000FEE703B401984100009850EAC12018BFDB
:10B5700004204A0D18BF40F0010040F2FF72B2EB08
:10B58000515F08BF40F00200012808BF052002B04B
:10B5900070470907090E002804DB00F1E02080F85D
:10B5A0000014704700F00F0000F1E02080F8141D37
:10B5B00070470000000000002DE9F04D2DED040B58
:10B5C0002DED0A8B9AB0DDE92550279CDDF890A07F
:10B5D00025F0004624F00048BAF1000F14BF012105
:10B5E000002101EB4502F84953184A1093422AD32F
:10B5F000002814BF0123002303EB44030B44F34949
:10B600008B4220D358EA00019FEDF19B72D0DFF806
:10B61000C8B35D4503D1BAF1000F05D184E0BAF19A
:10B62000000F08BF002100D0012101EB450111F5F9
:10B63000001F08D8002814BF0121002101EB44019C
:10B6400011F5001F0BD99DED261B9DED240B1AB0A3
:10B65000BDEC0A8B04B0BDE8F04D00F071BC0027D2
:10B66000002DBCBFDD49884521DADD498845A8BFEA
:10B6700002271CDAC3451ADCDA4901EB28511429E8
:10B6800008DDC1F1340220FA02F101FA02F282422D
:10B690000DD108E058B9C1F1140228FA02F101FAFB
:10B6A00002F2424503D101F00101C1F1020756EA5D
:10B6B0000A0120D1002C1EDA002D18BF022F01D064
:10B6C000012F0AD00220F5F71EF81AB0BDEC0A8B44
:10B6D00004B0BDE8F04D00F023BC0220F5F713F8EC
:10B6E00000F01EFCB1EE400B1AB0BDEC0A8B04B0AA
:10B6F000BDE8F08D18E09FEDBCAB9FEDBD8B002841
:10B700007DD1B64880451CD105F1804010F58010F0
:10B7100008BFBAF1000F07D0B34508DC002CA8BF62
:10B720009DED260BE0DA07E0B0EE490BDCE7002CDC
:10B73000B8BF9DED260BD5DBAF48784490ED000BEC
:10B74000D2E7D84548D1002C43DA2EB186423AD10F
:10B75000BAF1000F3DD126E0BAF1000F13D002205C
:10B76000F4F7D1FF00F0FCFB8DED020B9DED240BF7
:10B770008DED000B10EE900A039961F31E0003900B
:10B780009DED020BB0E78DED02AB9DED240B1AEEA3
:10B79000901A10EE900A8DED000B61F31E000390DD
:10B7A0009DED020BA0E78DED028B9DED240B18EEB5
:10B7B000901A10EE900A8DED000B61F31E000390BD
:10B7C0009DED020B90E704DA9DED241B89EE010B41
:10B7D0008AE79DED240B87E786421ADAB4F1804FA1
:10B7E00004BF9DED240B20EE000B3FF47DAFA4F1D0
:10B7F0000050B0F1FF500CD1002D0ADB00E008E052
:10B800009DED240B51EC100B01F026FA41EC100BCE
:10B810006AE79DED240B51EC100B00F0EDFBBAF143
:10B82000000FCDE90E0140D19FED750B46B3A6F197
:10B83000E040B0F17F600ED05E4536D1002D00DAD9
:10B8400097B3022F0CBF01204FF0FF3000EE100A1B
:10B85000B8EEC00B48E7002D01DD002C0DDA002DFD
:10B8600001DD002C1DDB002D14DA002C12DB012F72
:10B8700008BF9FED650B3FF437AFB0EE4A0B33E7DF
:10B88000022F18BF002D0CD0012F0AD1002DFFF67A
:10B890002BAF06E0002DB8BF002C06DA012F3FF4D5
:10B8A00023AFB0EE480B1FE719E0012000EBE57075
:10B8B00050EA070113D0791EB0EE498B084308BF48
:10B8C0009FED538B5448002580457ADD53495448F9
:10B8D000884514DDB0420DDB002C19DB2CE0012083
:10B8E000F4F711FF1AB0BDEC0A8B04B0BDE8F04DBF
:10B8F00000F02ABBB34502DC002C09DC1CE08642C8
:10B9000002DA002C18DA03E05E4528DD002C13DD96
:10B910000220F4F7F8FE00F023FB8DED020B28EE79
:10B920000A0B8DED000B10EE900A039961F31E00D7
:10B9300003909DED020BD7E60220F4F7E4FE00F041
:10B940001BFB10EE901A18EE900A8DED020B8DED98
:10B95000008B61F31E0003909DED020BC4E69DED8C
:10B960000E0B9FED313B30EE490B8DED040B20EEBD
:10B97000002B9DED041B9FED2E0B01EE430B9DED67
:10B98000043B9FED2D1B03EE401B9DED040B9FED33
:10B990002E3B22EE012B9FED2A1B20EE011B20EEF9
:10B9A000030B9FED2B3B02EE430B31EE002B8DED95
:10B9B000022B02959DED022B32EE411B30EE411B16
:10B9C00021E149E000000000FFFF1F00FFFF0F0022
:10B9D000000000000000F03F0000F03F0000F07F9A
:10B9E0000000404301FCFFFF000000000000F07F6A
:10B9F00000000000000000007230000000000000A5
:10BA00000000000000000080000000000000F0FFC7
:10BA1000000000000000F0BF0000E0410000F04323
:10BA2000FFFFEF3F00000000000000000000D03FDB
:10BA3000555555555555D53F000000000000E03FD5
:10BA4000000000604715F73F44DF5DF80BAE543E41
:10BA5000FE822B654715F73F0020B6F5801F0BDAF5
:10BA60009DED0E0B9FEDEC1B6FF0340020EE010BF3
:10BA700010EE906A8DED0E0BE94A00EB2650C6F3EE
:10BA80001301A0F2FF3741F07F6040F04050914237
:10BA9000D8BF002408DDE34A8A42C8BF012403DC82
:10BAA0000024A0F580107F1CDF49794401EBC4011C
:10BAB0000F9091ED001B9DED0E2B9DED0E0BDB49C4
:10BAC00031EE023B30EE410B89EE032B20EE02AB50
:10BAD0008DED02AB7944029591ED003B4FF00051A2
:10BAE00041EA600000EB84408DED043B00F500204E
:10BAF00005909DED043B9DED044B2AEE0ACB33EE01
:10BB0000411B9DED0E3BCA48062133EE411B9DEDC6
:10BB1000023B03EE440B03EE410B20EE02BBB0EE02
:10BB20004C0B784400F0C4F92CEE0C1B20EE010BFA
:10BB30009DED021B31EE0A1B0BEE010B9DED021B6E
:10BB400021EE011B9FEDBC2B31EE023B33EE003B9F
:10BB50008DED043B04959DED043B33EE422B32EE1C
:10BB6000411B30EE412B9DED020B9DED041B20EEA1
:10BB7000011B9DED040B2BEE000B02EE0A0B31EEC8
:10BB8000002B8DED022B02959DED022B32EE411B19
:10BB900030EE410B9DED021B9FEDA92B21EE021B08
:10BBA0009DED022B9FEDA83B22EE032B9FEDA83BC2
:10BBB000A94800EE032B784400EBC40090ED000B85
:10BBC000A64832EE000B02EE107AB8EEC22B8DEDD5
:10BBD000042B31EE003B784400EBC4009DED044B98
:10BBE00090ED002B33EE023B33EE043B8DED023B38
:10BBF00002959DED023B33EE443B33EE422B32EE99
:10BC0000411B30EE411B9DED260B954A8DED000B3F
:10BC100000959DED260B9DED002B30EE420B9DED2A
:10BC2000022B20EE020B9DED262B02EE010B9DED6B
:10BC3000001B9DED022B21EE021B8DED021B30EE51
:10BC4000011B11EE900A11EE101A8DED001B9042AF
:10BC500024DB821A11430ED19FED831B9DED002B37
:10BC60009DED023B30EE011B32EE432BB4EEC21BC6
:10BC7000F1EE10FA26DD0220F4F745FD00F070F930
:10BC800010EE901A18EE900A8DED020B8DED008BE0
:10BC900061F31E0003909DED020B25E5744B20F02F
:10BCA00000429A420ED3734A024411437FF444AED9
:10BCB0009DED022B31EE421BB4EEC01BF1EE10FAEB
:10BCC000BFF63AAE20F000416B4A6C4B002402EB09
:10BCD00021529942D8BF9DED021B27DD511C4FF424
:10BCE000801222FA01F10144654BC1F30A527B44F0
:10BCF000A2F2FF3293ED001B624B8DED041BD3408B
:10BD000021EA0303C1F3130141F48011C2F11402CB
:10BD100021FA02F405930028B8BF64429DED021B8E
:10BD20009DED042B31EE421B8DED021B30EE011B0D
:10BD30008DED041B04959DED041B9FED532B9DED94
:10BD4000023B21EE021B9DED042B32EE432B30EE25
:10BD5000420B9FED4F2B20EE020B9DED042B9FED30
:10BD60004E3B4F48052102EE030B31EE002B8DEDCB
:10BD7000002B32EE411B30EE41AB9DED000B20EE6F
:10BD8000000B8DED040B784400F092F89DED001B44
:10BD90009DED042B02EE401B8DED021B9DED000B73
:10BDA00020EE010B9FED402B31EE422B80EE021B6B
:10BDB0009DED002BB0EE4A0B02EE0A0B31EE400B6C
:10BDC0009DED001B30EE410B39EE400B10EE900A5A
:10BDD0008DED000B00EB045001150029C8BF019048
:10BDE00013DC224651EC100B02F063F9FFF7B9FBAC
:10BDF000042808BF00F0C0F822469DED000B51EC6E
:10BE0000100B02F056F9CDE900019DED000B28EE74
:10BE1000000B69E400000000000000000000404347
:10BE20008E9803007AB60B007A2C0000D82C000004
:10BE3000322C00000000000000000000000008405C
:10BE4000000000E009C7EE3FF5015B14E02F3EBEA5
:10BE5000FD033ADC09C7EE3F8E2B00005E2B00008D
:10BE60000000904000000000FE822B654715973CC3
:10BE700000CC904000346F3F01FCFFFF0000E03F2A
:10BE8000BE2A0000FFFF0F0000000000432EE63F27
:10BE9000EF39FAFE422EE63F396CA80C615C20BEF9
:10BEA000FE2900000000000000000000000000402B
:10BEB000491E00EBC102B0EE401B92ED000B31F0C9
:10BEC00006020DD0491E00EBC102B0EE403B92EDE0
:10BED000002B31F00602B0EE420B03EE010BF1D164
:10BEE000022914D004290AD0062918BF704790ED02
:10BEF0000A2B00EE012B90ED080B02EE010B90EDEA
:10BF0000062B00EE012B90ED040B02EE010B90EDE1
:10BF1000022B00EE012B90ED000B02EE010B70479F
:10BF20009FED031B9FED042B81EE020B7047000079
:10BF3000000000000000F03F0000000000000000D2
:10BF400030EE010B704700009FED031B81EE010BEB
:10BF5000704700000000000000000000000000002A
:10BF60009FED030B20EE000B704700000000000067
:10BF700000000000000000709FED030B20EE000B9E
:10BF800070470000000000000000000000000010EA
:10BF90009FED110B002208E030F8123001EE103A4C
:10BFA000B8EE411B31EE000B521C8A42F4DB01EE6D
:10BFB000101AB8EEC12B80EE021B9FED092B81EE0B
:10BFC000020B9FED091B20EE010B9FED091B20EEDC
:10BFD000010BB7EEC00B704700000000000000002E
:10BFE00000000000E0FFEF400000000000C8A94092
:10BFF00039B4C876BE9F064082B0CDE9000121F079
:10C00000004001909DED000B02B051EC100B704709
:10C01000F8F7B4FAFDF7AEF9FCF784FBFCF728FB60
:10C02000FCF744FBFCF76AFAFCF72EFDFCF790FCEA
:10C03000FCF722FCFCF7DAFC012208481102F8F7B1
:10C0400081FA00F021F8064A0021064800F004F9C0
:10C050000549886000F02CF8FEE700000000025857
:10C0600040E10008819100080800002410B5EFF3BA
:10C070000581002902D06FF0050403E0002408B117
:10C0800000F084FF204610BDEFF30580002802D0A9
:10C090006FF0050070470548016811B14FF0FF309F
:10C0A0007047012101600020704700004801002412
:10C0B00010B5EFF30580002802D06FF0050010BD29
:10C0C00007480168012902D04FF0FF3010BD054A32
:10C0D000002111700221016001F010F8002010BD54
:10C0E000480100241FED00E0F8B50D460024221F92
:10C0F000561C002805D0EFF30581C1B11DB11446CF
:10C100001FE014461DE0002100916A4601F0E8FBA3
:10C11000012801D0344614E0009890B10A494FF04C
:10C1200080500860BFF34F8FBFF36F8F09E029463F
:10C1300001F024FC012804D015B16FF0010400E0E7
:10C1400034462046F8BD000004ED00E0F8B50E4688
:10C1500014464FF00005EFF3058100294DD1B8B327
:10C1600086424AD84A1E5CB1A36823B1E1685029CF
:10C1700001D3012205E023B9E16811B9002200E0F2
:10C180000022511C39D0012809D0012A2BD0314678
:10C1900001F0C8F80546DDB15CB321682AE0012A48
:10C1A00017D003220021012001F0FBF80546002DE5
:10C1B000F1D0002EEFD0002328461A46194601F090
:10C1C0008FF90128E7D0284600F08EFE0025E2E72F
:10C1D00013E0032000900022A3680120114601F023
:10C1E00002F90546E3E7A268314601F0B9F80546D1
:10C1F000D1E70021284600F065FE2846F8BD000082
:10C2000038B50024E51E00280BD0EFF30581B1B14D
:10C2100000210091694601F075FA012804D02C46EE
:10C2200015E06FF0030412E0009880B109494FF067
:10C2300080500860BFF34F8FBFF36F8F07E000237C
:10C240001A46194601F04CF9012800D02C46204628
:10C2500038BD000004ED00E02DE9FF470B464FF02C
:10C260000008CDF80C80EFF30581A1BB98B34FF423
:10C27000807618240025691E72B3176807B13D4601
:10C28000976907B13C46671E382F02D21779FF071E
:10C2900003D0002004B0BDE8F087576907B1BE089D
:10C2A000D2F808C0BCF1000F0CD0D2F80C90B9F154
:10C2B0005C0F07D3D2F81090B9F1000F02D00FB184
:10C2C00001210BE0BCF1000F08D1D76837B917691D
:10C2D00027B9002102E01BE0FFE70021012901D07E
:10C2E00059B115E09168126902912946CDE90042E1
:10C2F000324601F071FC03900AE003A9B2B2CDE925
:10C300000041294601F036FC012801D0CDF80C800F
:10C310000398BFE72DE9F04104460F46134EF56838
:10C320003068001D00F0CDFC601C07D137B13168CA
:10C33000BDE8F0410E48091D00F014BD2C443068E2
:10C340004460AC4206D23168B06B091DBDE8F041D3
:10C3500000F0F0BC3168706B091D00F0EBFCB06AB6
:10C36000844200D2B462BDE8F0810000F8000024ED
:10C3700068F7002470B5044600F000FD1C4DA86865
:10C38000401CA860286810B1686938B10CE02C60C6
:10C39000A868012808D100F0A3F905E02868E16A3F
:10C3A000C06A884200D82C60686A401C6862606479
:10C3B000E06A2969884200D9286100EB80000D49B4
:10C3C00001EB8000211D00F0CDFC00F0F7FC686956
:10C3D00000280CD02868E16AC06A884207D2064962
:10C3E0004FF080500860BFF34F8FBFF36F8F70BD69
:10C3F000F8000024B8F2002404ED00E038B500F0A5
:10C40000BDFC104C2068C8B90F4800F085FC0E48F0
:10C41000143000F081FC0C48E060143020610A4BBD
:10C42000002010210090F03B0A2003F1500200F0A0
:10C43000DAFF206010B105A100F044FDBDE83840EE
:10C4400000F0BCBC340100246CF80024546D72511F
:10C450000000000070B50C4D0C4E11E000F08EFC99
:10C46000F068C468201D00F02CFCA868401EA8607D
:10C470006868401E686000F0A1FC204600F053F898
:10C4800068680028EAD170BDF800002454F7002441
:10C490000B4630B4026C002A0CD0C1681144C16054
:10C4A0008468A14201D30168C160C168184630BCEC
:10C4B000F4F759B830BC70472DE9F04104461746EF
:10C4C0000026A56B226C002A10D0C7B1E068F4F7F3
:10C4D0004AF8E168206C091AE1602268914202D2B0
:10C4E000A168081AE060022F16D017E02068A8B9EA
:10C4F000A06801F019FC06460020A0600EE060680C
:10C50000F4F731F8216C606808446060A1688842E3
:10C5100004D32068606001E005B16D1E6D1CA56349
:10C520003046BDE8F08110B5044694F85900002863
:10C530000BD0012811D0022814D0502080F311888C
:10C54000BFF34F8FBFF36F8FFEE7206B00F04CFC03
:10C550002046BDE8104000F047BC2046BDE8104032
:10C5600000F042BC10BD416A002904D0006B006895
:10C57000C0F1380070470020704700000749CA68C2
:10C580001168002904D00021016019B10020704712
:10C590000121F9E7D06800687047000034010024E9
:10C5A0004FF4A0410F48420706D0C01D20F00700FD
:10C5B0000C49411AC1F5A0410B4A10600023536099
:10C5C0000144083921F00701183A11604B600B60F3
:10C5D0000B1A436001604068906050604FF000406B
:10C5E000506170474C01012464010024074E4FF054
:10C5F0008054074DFFF72EFF30680128FAD92C60D0
:10C60000BFF34F8FBFF36F8FF4E70000B8F2002441
:10C6100004ED00E070B51D46049C002909D022609D
:10C62000E06321640121204600F014FF84F84C509F
:10C6300070BD2460F4E72DE9F05F82460E46174690
:10C640009B46DDE90A590C9CB900A522206BF4F742
:10C6500001F8206B7F1E00EB870020F007077807AA
:10C6600007D0502080F31188BFF34F8FBFF36F8F37
:10C67000FEE74FF0000866B100202218315C82F816
:10C680003410315C11B1401C1028F6D384F843807B
:10C6900001E084F83480382D00D33725E562E56465
:10C6A000C4F85080201D00F042FB04F1180000F097
:10C6B0003EFB2461C5F13800A0616462C4F8548077
:10C6C00084F858805A465146384600F0B3FA206044
:10C6D000B9F1000F01D0C9F80040BDE8F09F00009B
:10C6E00070B50024114D04EB840005EB800000F0D0
:10C6F00013FB641C382CF6D30D4800F00DFB0C48DE
:10C70000143000F009FB0A48283000F005FB084807
:10C710003C3000F001FB0648503000F0FDFA0548BF
:10C72000034941631431816370BD0000B8F20024F5
:10C7300018F70024F800002430B5134900E0114632
:10C740000A688242FBD34B685C18844203D140687C
:10C750001844486008460D6844682318AB420DD160
:10C76000094B183B1B689A4206D05268224442602B
:10C770000A681268026002E0036000E00260814221
:10C7800000D0086030BD00006401002470B50024B2
:10C790004160006191420C4D0AD8D11A82699142E0
:10C7A00001D301240EE0011D286900F0C3FA09E05D
:10C7B0009A4203D2994201D3012403E0011DE868A3
:10C7C00000F0B8FA204670BD3401002410B50446CC
:10C7D00000F0D4FAA06B20B1002400F0EFFA20465C
:10C7E00010BD0124F9E710B5044600F0C7FAA06BAC
:10C7F000E16B884201D1012400E0002400F0DEFA60
:10C80000204610BDF8B505460E461748C068C068FA
:10C81000C468201D00F055FA94F82800410718D587
:10C82000A0692B46324641192046FFF7AFFFA0B161
:10C8300000202A46034601460090204601F0C4FB32
:10C8400058B9502080F31188BFF34F8FBFF36F8F1B
:10C85000FEE720F0010084F82800216A01B020469C
:10C86000BDE8F040084700003401002430B587B02F
:10C870003C4D6EE00398002803DADDE904200699B8
:10C8800090470398002864DB059C606910B1201D67
:10C8900000F017FA02A800F0AFF8024603980A2841
:10C8A00057D2DFE800F00505052D334A05052D3385
:10C8B00094F8280040F0010084F828000498A16949
:10C8C000034601442046FFF761FF68B3216A204612
:10C8D000884794F8280040073BD500200090049832
:10C8E0000023A16942181946204601F06DFBD8B912
:10C8F000502080F31188BFF34F8FBFF36F8FFEE797
:10C9000014F8280F20F00100207022E094F828008D
:10C9100040F0010084F828000498A06128B1811833
:10C9200013462046FFF732FF13E0502080F31188B2
:10C93000BFF34F8FBFF36F8FFEE794F82800810796
:10C9400003D4204600F050FA03E020F0010084F800
:10C9500028002868002203A900F024FF002889D1BC
:10C9600007B030BD34010024F8B506460D4600F08E
:10C970000DFC684600F040F80446009810B101F044
:10C980008BFAF8BD45B9A64206D801F085FA2146D2
:10C990003046FFF737FFF8BD0C481DB10169096843
:10C9A00091B100250068311B2A4600F0CBFA01F056
:10C9B00073FA0028EFD106494FF080500860BFF3AA
:10C9C0004F8FBFF36F8FF8BD0125EBE734010024D3
:10C9D00004ED00E00748416B0968002905D0416B70
:10C9E000C968C9684968816270474FF0FF31816248
:10C9F00070470000F800002470B5054601F028F9E2
:10CA00000446074EB068844204D200F00BF80120BF
:10CA1000286001E000202860B460204670BD00005E
:10CA200034010024F8B51A4E20E0C0680568C468D7
:10CA3000201D00F046F9216A2046884794F8280016
:10CA4000400713D5A0692844A84206D96060246134
:10CA5000211DF06800F06EF908E000202A46034628
:10CA600001460090204601F0AFFA40B1F06801683D
:10CA70000029DAD1F0683169F1603061F8BD5020E9
:10CA800080F31188BFF34F8FBFF36F8FFEE7000075
:10CA90003401002409484068401C07D0502080F32E
:10CAA0001188BFF34F8FBFF36F8FFEE7502080F3E5
:10CAB0001188BFF34F8FBFF36F8FFEE76C01002427
:10CAC00008B56846FFF75AFD0099FFF74DFFFFF7DD
:10CAD000CDFEF6E72DE9F041044600F04FF994F958
:10CAE000455004F1240609E0606A48B1304601F07F
:10CAF00097F908B100F07AFA6D1E6DB2002DF3DCE3
:10CB00004FF0FF3684F8456000F058F900F036F930
:10CB100094F9445004F1100709E0206948B13846FF
:10CB200001F07EF908B100F061FA6D1E6DB2002DC2
:10CB3000F3DC84F84460BDE8F04100F03FB9000048
:10CB40002DE9F0410546002600F020FB324F386801
:10CB500008B9FFF725FD786905424DD18DB108353B
:10CB600068070ED005F00700C0F10800054468070B
:10CB700007D0502080F31188BFF34F8FBFF36F8F22
:10CB8000FEE7CDB37868854236D823491831084688
:10CB9000046801E0214604466068A84202D2206889
:10CBA0000028F7D13868844226D00E6808362068FD
:10CBB00008606068411B10290ED96019420707D030
:10CBC000502080F31188BFF34F8FBFF36F8FFEE7C4
:10CBD00041606560FFF7B0FD61687868401A786071
:10CBE000BA68904200D2B860786901436160002061
:10CBF0002060F868401CF86001F04EF9700707D01B
:10CC0000502080F31188BFF34F8FBFF36F8FFEE783
:10CC10003046BDE8F08100004C010024044908685A
:10CC2000002803D00868026D521C0265086870472E
:10CC3000F800002424384FF08073036221F00101D2
:10CC4000C1610449816142606FF0020140F820191E
:10CC50007047000095CA000800B541EC100B2DED9F
:10CC6000028B83B0B1EEC08B18EE100A18EE901A4A
:10CC70008DED008B002818BF0120084320F00040F4
:10CC8000C0F17F6000F1E040C00F14D010EE101A28
:10CC900010EE900A8DED000B002918BF012108430A
:10CCA00020F00040C0F17F6000F1E040C00F04BF01
:10CCB0000120F3F728FD51EC180B03B0BDEC028BFB
:10CCC00000BD0169D0E901329A60D0E901235A60C0
:10CCD0004A68824201D182684A6000220261086883
:10CCE000401E086008687047044B036003F15C0055
:10CCF00008604FF4807010607047000094F80024C2
:10CD0000044B036003F15C0008604FF48070106016
:10CD100070470000F0FC002400F1080141604FF072
:10CD2000FF328260C1600161002101607047002113
:10CD30000161704730B50C68621C02D000F1080236
:10CD400002E0026904E01A4653681D68A542FAD958
:10CD500053684B6099608A60516008610168491CA2
:10CD6000016030BD42684A6093688B609368596087
:10CD7000916008610168491C01607047502080F390
:10CD80001188BFF34F8FBFF36F8F0A494868401C6B
:10CD9000486001280CD10848006810F0FF0F07D048
:10CDA000502080F31188BFF34F8FBFF36F8FFEE7E2
:10CDB000704700006C01002404ED00E00949486858
:10CDC000002806D0401E4860002801D180F3118859
:10CDD0007047502080F31188BFF34F8FBFF36F8FE0
:10CDE000FEE700006C01002470B500282AD0083846
:10CDF0000446154D60686969084207D1502080F3E8
:10CE00001188BFF34F8FBFF36F8FFEE722683AB1EF
:10CE1000502080F31188BFF34F8FBFF36F8FFEE771
:10CE20008843606000F0B2F960686968084468602F
:10CE30002046FFF781FC2869401C2861BDE870404E
:10CE400001F02AB870BD00004C0100244FF0E02032
:10CE50000021016181614FF47A7204490968B1FBD4
:10CE6000F2F1491E4161072101617047E40000248D
:10CE700010B5F3F7DDFA114910280ED300F1E020C8
:10CE800090F8F0030A78904207D2502080F311887E
:10CE9000BFF34F8FBFF36F8FFEE7094800688968C3
:10CEA00000F4E060884207D9502080F31188BFF376
:10CEB0004F8FBFF36F8FFEE710BD00006C010024A1
:10CEC0000CED00E010B50022064B53F832401CB1C7
:10CED000521C082AF9D310BD43F8321003EBC201EB
:10CEE000486010BD78F2002410B50446002C0BD029
:10CEF000204600F013F894F8460000280CD1204694
:10CF0000BDE81040FFF770BF502080F31188BFF3D9
:10CF10004F8FBFF36F8FFEE710BD00000021084A5E
:10CF200002EBC1035B68834206D1002042F8310066
:10CF300002EBC10148607047491C0829F0D37047D3
:10CF400078F2002470B504460D461646FFF716FF2A
:10CF500094F944304FF000005B1C01D184F8440088
:10CF600094F94510491C01D184F84500FFF726FFCC
:10CF7000A06B28B904F124003246294600F056F887
:10CF80002046BDE87040FFF7A5BD0000024610B581
:10CF90000020002A12D00F48006B38B1502080F3D7
:10CFA0001188BFF34F8FBFF36F8FFEE700F0EEF8ED
:10CFB00000211046FFF7AEF900F06EFF002807D100
:10CFC00005494FF080500860BFF34F8FBFF36F8F5C
:10CFD00010BD0000F800002404ED00E002490A6AD8
:10CFE0000260C96841607047F800002401490120CF
:10CFF000C8617047F800002410B50C4600280AD01C
:10D00000094909681831FFF795FE2046BDE8104030
:10D010000121FFF77FB9502080F31188BFF34F8FB4
:10D02000BFF36F8FFEE70000F800002470B50D46D7
:10D03000144600280DD00B4909681831FFF792FEFD
:10D040000CB14FF0FF3521462846BDE87040FFF790
:10D0500061B9502080F31188BFF34F8FBFF36F8FFA
:10D06000FEE70000F800002470B50B4604460028D7
:10D070003ED0226DA2B1E16C994200D21946E06A1D
:10D08000884235D0012A33D11A4D2A6894420FD1F3
:10D09000502080F31188BFF34F8FBFF36F8FFEE7EF
:10D0A000502080F31188BFF34F8FBFF36F8FFEE7DF
:10D0B000E162A269002A02DBC1F13801A1610E4ED2
:10D0C00000EB8000616906EB8000814210D1201DD9
:10D0D000FFF7F7FDE06A2969884200D9286100EB73
:10D0E0008000211D06EB8000BDE87040FFF73ABECE
:10D0F00070BD0000F8000024B8F2002430B587B0FD
:10D1000000250695059504AA05A906A8FFF7ECFDDC
:10D11000DDE90510049A002302901A48CDE9005178
:10D1200016A100F059FD184CE06208B1012000E0A2
:10D130000020012801D100F013FF012809D0401C74
:10D1400019D1502080F31188BFF34F8FBFF36F8F39
:10D15000FEE7502080F31188BFF34F8FBFF36F8F2E
:10D160004FF0FF30A06201206061E56007B0BDE8CC
:10D17000304000F047B807B030BD000049444C458E
:10D1800000000000EDC50008F80000240248016B13
:10D19000491C016370470000F800002410B5174BCC
:10D1A000186B002802D00120D86110BD0020D86182
:10D1B0001869134901E0C0B1401E00EB800251F82C
:10D1C0002220002AF7D000EB800201EB82014A689E
:10D1D00052684A6001F10804A24201D152684A60D3
:10D1E0004968C9681960186110BD502080F3118822
:10D1F000BFF34F8FBFF36F8FFEE70000F8000024EE
:10D20000B8F200241CB537480168374A914207D16B
:10D21000502080F31188BFF34F8FBFF36F8FFEE76D
:10D2200000683149491E884207D1502080F3118897
:10D23000BFF34F8FBFF36F8FFEE72C490878019043
:10D24000FF200870087800909DF800009DF80020ED
:10D2500000F0F000904207D0502080F31188BFF317
:10D260004F8FBFF36F8FFEE79DF80000204C00F05A
:10D27000500020700720A06006E0A068401EA0605B
:10D280009DF80000400000909DF800000006F4D4D6
:10D29000A068032807D0502080F31188BFF34F8F78
:10D2A000BFF36F8FFEE74FF44070A06001980870E5
:10D2B0000C482030016841F470010160016841F0C0
:10D2C00070410160FFF7C2FD00206060F3F778F85D
:10D2D0000848016841F040410160F3F75DF8002023
:10D2E0001CBD000000ED00E071C20F4100E400E051
:10D2F0006C01002434EF00E010B5502080F3118859
:10D30000BFF34F8FBFF36F8F00F0A8FC18B1044933
:10D310004FF080500860002080F3118810BD00009D
:10D3200004ED00E010B50C46002809D084420FD966
:10D33000502080F31188BFF34F8FBFF36F8FFEE74C
:10D34000502080F31188BFF34F8FBFF36F8FFEE73C
:10D350000222002100F025F8002800D0846310BDCF
:10D3600038B50C46002809D084420FD9502080F3EC
:10D370001188BFF34F8FBFF36F8FFEE7502080F30C
:10D380001188BFF34F8FBFF36F8FFEE70221134663
:10D3900000220091114600F026F8002800D0846396
:10D3A00038BDF8B505460E461746002D13D005FBCF
:10D3B00006F05030FFF7C4FB044654B12246503209
:10D3C000002084F846003B46314628460094FFF78B
:10D3D00021F92046F8BD502080F31188BFF34F8F0C
:10D3E000BFF36F8FFEE738B5049D002804D05BB112
:10D3F00002B189B1C2B120E0502080F31188BFF39F
:10D400004F8FBFF36F8FFEE7502080F31188BFF37B
:10D410004F8FBFF36F8FFEE7502080F31188BFF36B
:10D420004F8FBFF36F8FFEE739B1502080F3118823
:10D43000BFF34F8FBFF36F8FFEE7502400941C465D
:10D44000012384F846302B460094FFF7E3F820468A
:10D4500038BD000070B504460D46002C25D0FFF7FE
:10D460008DFCD4E90F20216802FB0011A16000218E
:10D47000A16321686160E06B216C401E226800FBA3
:10D480000121E1604FF0FF3084F8440084F845004A
:10D4900004F110008DB1FFF73FFC04F12400FFF709
:10D4A0003BFCFFF78BFC012070BD502080F31188FE
:10D4B000BFF34F8FBFF36F8FFEE721690029F0D0D4
:10D4C00000F0AEFC0028ECD004494FF0805008601A
:10D4D000BFF34F8FBFF36F8FE3E7000004ED00E071
:10D4E0002DE9FF4782B004468A461E460025002CDF
:10D4F00003D0BAF1000F08D011E0502080F311885A
:10D50000BFF34F8FBFF36F8FFEE7206C38B1502011
:10D5100080F31188BFF34F8FBFF36F8FFEE7022EAA
:10D520000AD1E06B012807D0502080F31188BFF3A7
:10D530004F8FBFF36F8FFEE700F07CFB48B9049874
:10D5400038B1502080F31188BFF34F8FBFF36F8F36
:10D55000FEE7DFF8EC804FF080574FF00009FFF74F
:10D560000DFCA06BE16B884205D3022E03D004981A
:10D5700008B325B327E0324651462046FEF79CFF0C
:10D58000616A59B104F1240000F04AFC68B1C8F89E
:10D590000070BFF34F8FBFF36F8F06E028B1C8F85C
:10D5A0000070BFF34F8FBFF36F8FFFF707FC0120B1
:10D5B00006B0BDE8F087FFF701FC0020F8E76846F9
:10D5C000FFF70CFD0125FFF7F9FBFFF7DFFDFFF784
:10D5D000D5FB94F94400401C01D184F8449094F99F
:10D5E0004500401C01D184F84590FFF7E7FB04A9F2
:10D5F000684600F081FA30B12046FFF76BFA00F080
:10D600004BFC0020D4E72046FFF7EDF890B10499D9
:10D6100004F11000FFF7F0FC2046FFF75BFA00F082
:10D620003BFC00289BD1C8F80070BFF34F8FBFF3BD
:10D630006F8F94E72046FFF74DFA00F02DFC8EE740
:10D6400004ED00E02DE9F0470446894690461F4668
:10D65000002C03D0B9F1000F08D011E0502080F366
:10D660001188BFF34F8FBFF36F8FFEE7206C38B187
:10D67000502080F31188BFF34F8FBFF36F8FFEE709
:10D68000022F0AD1E06B012807D0502080F31188C7
:10D69000BFF34F8FBFF36F8FFEE7FFF7E9FB50201B
:10D6A000EFF3118680F31188BFF34F8FBFF36F8FB5
:10D6B000A06BE16B884206D3022F04D0002086F3D2
:10D6C0001188BDE8F08794F94550A06B3A46494669
:10D6D0002046FEF7F1FE681C04D06D1C84F845500E
:10D6E0000120ECE7606A0028FAD004F1240000F081
:10D6F00097FB0028F4D0B8F1000FF1D00120C8F852
:10D700000000EDE770B504460E46002C09D0206CF1
:10D7100078B1502080F31188BFF34F8FBFF36F8F24
:10D72000FEE7502080F31188BFF34F8FBFF36F8F58
:10D73000FEE7206848B9A06838B1502080F311880E
:10D74000BFF34F8FBFF36F8FFEE7FFF791FB5020C2
:10D75000EFF3118580F31188BFF34F8FBFF36F8F05
:10D76000A26BE06B904218D994F94500521CA26359
:10D77000411C04D0401C84F8450001200EE0606A82
:10D780000028FAD004F1240000F04AFB0028F4D06D
:10D79000002EF2D001203060EFE7002085F31188E1
:10D7A00070BD00002DE9F74783B004468A46002685
:10D7B000002C03D0BAF1000F08D011E0502080F304
:10D7C0001188BFF34F8FBFF36F8FFEE7206C38B126
:10D7D000502080F31188BFF34F8FBFF36F8FFEE7A8
:10D7E00000F028FA48B9059838B1502080F3118824
:10D7F000BFF34F8FBFF36F8FFEE7DFF8E090002796
:10D800004FF08058FFF7BAFAA56BC5B151462046D4
:10D81000FEF73EFE6D1EA563206950B104F11000B5
:10D8200000F0FEFA28B1C9F80080BFF34F8FBFF3B4
:10D830006F8FFFF7C3FA012006B0BDE8F0870598A7
:10D8400008B126B107E0FFF7B9FA0020F4E701A814
:10D85000FFF7C4FB0126FFF7B1FAFFF797FCFFF7CC
:10D860008DFA94F94400401C01D184F8447094F975
:10D870004500401C01D184F84570FFF79FFA05A9C7
:10D8800001A800F039F958B12046FFF723F900F05C
:10D8900003FB2046FEF79AFF0028B3D00020CBE719
:10D8A0002046FEF793FF90B1059904F12400FFF79D
:10D8B000A3FB2046FFF70EF900F0EEFA0028A1D1F5
:10D8C000C9F80080BFF34F8FBFF36F8F9AE72046F0
:10D8D000FFF700F900F0E0FA94E7000004ED00E043
:10D8E0002DE9F047044689469046002C03D0B9F153
:10D8F000000F08D011E0502080F31188BFF34F8F44
:10D90000BFF36F8FFEE7206C38B1502080F3118891
:10D91000BFF34F8FBFF36F8FFEE7FFF7A9FA5020D9
:10D92000EFF3118780F31188BFF34F8FBFF36F8F31
:10D93000A66BF6B194F9445049462046FEF7A8FD7F
:10D94000761EA663681C04D06D1C84F84450012028
:10D9500010E020690028FAD004F1100000F060FA0D
:10D960000028F4D0B8F1000FF1D00120C8F8000071
:10D97000EDE7002087F31188BDE8F0872DE9F34338
:10D9800083B004460025A946002C09D0206C78B14C
:10D99000502080F31188BFF34F8FBFF36F8FFEE7E6
:10D9A000502080F31188BFF34F8FBFF36F8FFEE7D6
:10D9B00000F040F948B9049838B1502080F311883C
:10D9C000BFF34F8FBFF36F8FFEE7DFF8288100268C
:10D9D0004FF08057FFF7D2F9A06BC8B1401EA0638B
:10D9E000206810B9FFF71AF9A060206950B104F15E
:10D9F000100000F015FA28B1C8F80070BFF34F8F7F
:10DA0000BFF36F8FFFF7DAF9012005B0BDE8F083AF
:10DA1000049808B17DB112E0B9F1000F07D0502091
:10DA200080F31188BFF34F8FBFF36F8FFEE7FFF7CF
:10DA3000C5F90020E9E701A8FFF7D0FA0125FFF7B3
:10DA4000BDF9FFF7A3FBFFF799F994F94400401CD7
:10DA500001D184F8446094F94500401C01D184F858
:10DA60004560FFF7ABF904A901A800F045F8C8B17B
:10DA70002046FFF72FF800F00FFA2046FEF7A6FE2B
:10DA80000028A7D0B9F1000F0AD0FFF777F9204698
:10DA9000FEF769FD0146A068FFF7E6FAFFF78EF989
:10DAA0000020B2E72046FEF791FEE8B1206838B9C1
:10DAB000FFF764F9A06800F075F98146FFF77EF979
:10DAC000049904F12400FFF797FA2046FFF702F8C3
:10DAD00000F0E2F900287FF47DAFC8F80070BFF3D2
:10DAE0004F8FBFF36F8F75E72046FEF7F3FF00F00F
:10DAF000D3F96FE704ED00E02DE9F04105460C464F
:10DB0000002D11D0C4B1FFF739F9194EF0686B68D8
:10DB1000C11A2268571C17D02F68366AB74215D031
:10DB2000834213D801241DE0502080F31188BFF3F5
:10DB30004F8FBFF36F8FFEE7502080F31188BFF344
:10DB40004F8FBFF36F8FFEE700240BE08A4206D9A8
:10DB5000501A20602846FFF741FA002402E0002016
:10DB600020600124FFF72AF92046BDE8F08100007B
:10DB7000F80000242DE9FF5F81468A4616469B4641
:10DB8000DDE90E78B000FEF7DBFF054628000AD07D
:10DB90005C20FEF7D5FF04460CB1256304E028465F
:10DBA000FFF722F900E000249CB1002084F859001E
:10DBB000CDE900785B463246CDE902405146484601
:10DBC000FEF739FD2046FEF7D5FB012004B0BDE885
:10DBD000F09F4FF0FF30F9E7F0B585B00746DDE97B
:10DBE0000A600C9C002815D0E4B15C2503952063E5
:10DBF000022084F85900002004ADCDE90240CDE9AF
:10DC000000653846FEF717FD2046FEF7B3FB049883
:10DC100005B0F0BD502080F31188BFF34F8FBFF3E4
:10DC20006F8FFEE7502080F31188BFF34F8FBFF353
:10DC30006F8FFEE705484169002903D0006B18B1DA
:10DC4000002070470120704702207047F800002430
:10DC50000148C06870470000F80000242DE9F04139
:10DC600000262F4F386B002805D0B869401CB861DA
:10DC70003046BDE8F081FD686D1CFD609DB9786B94
:10DC8000006838B1502080F31188BFF34F8FBFF385
:10DC90006F8FFEE7786BB96B7963B863386A401CA5
:10DCA0003862FEF797FEB86ADFF8788085420DD3B8
:10DCB000786B006838B1786BC068C468606885426A
:10DCC00012D2B86202E04FF0FF30B8623868C06A22
:10DCD00000EB800058F82000012800D90126F869DF
:10DCE0000028C5D00126C3E7201DFEF7EAFFA06A81
:10DCF00018B104F11800FEF7E4FFE06A39698842C0
:10DD000000D9386100EB8000211D08EB8000FFF78F
:10DD100029F8E06A3968C96A8842C9D30126C7E789
:10DD2000F8000024B8F2002470B504460020002C4E
:10DD30002BD01A4D29688C4207D0502080F31188CF
:10DD4000BFF34F8FBFF36F8FFEE7216DF1B1491E17
:10DD50002165E36CE26A9A4217D0002915D1201D93
:10DD6000FEF7AFFFE06CE062C0F13800A061E06A4E
:10DD70002969884200D9286100EB8000084901EB3D
:10DD80008000211DFEF7EEFF012070BD502080F3C2
:10DD90001188BFF34F8FBFF36F8FFEE7F8000024A9
:10DDA000B8F2002470B504460020002C2CD01A4D87
:10DDB000E16A2A68D26A914227D2A069002804DB6E
:10DDC0002868C06AC0F13800A061E06A134E61693A
:10DDD00000EB800006EB8000814211D1201DFEF790
:10DDE00070FF2868C06AE0622969884200D928610A
:10DDF00000EB8000211D06EB8000FEF7B3FF02E080
:10DE00002868C06AE062012070BDE16C2A68D26AAD
:10DE10009142F9D2012070BDF8000024B8F200242C
:10DE200070B5C068C468002C14D004F11800064610
:10DE3000FEF747FF154D2A6BA2B115483146FEF794
:10DE400091FFE06A2968C96A88421CD90120012132
:10DE5000E96170BD502080F31188BFF34F8FBFF38D
:10DE60006F8FFEE7201DFEF72CFFE06A29698842CC
:10DE700000D9286100EB8000064901EB8000211DDC
:10DE8000FEF770FFDDE7002070BD0000F800002401
:10DE900040F70024B8F200242DE9F04100240027C7
:10DEA0002B4D286B002807D0FEF768FF286B401E1B
:10DEB0002863286B40B146E0502080F31188BFF3FF
:10DEC0004F8FBFF36F8FFEE7A868E0B3DFF8848061
:10DED00001261CE0D8F80C00C46804F11800FEF715
:10DEE000F0FE201DFEF7EDFEE06A2969884200D9A8
:10DEF000286100EB8000184901EB8000211DFEF72E
:10DF000031FFE06A2968C96A884200D3EE61D8F817
:10DF100000000028DED10CB1FEF75CFDAC6944B115
:10DF2000FFF79CFE00B1EE61641E002CF8D10020CA
:10DF3000A861E86938B10127084938070860BFF3CC
:10DF40004F8FBFF36F8FFEF739FF3846BDE8F08182
:10DF5000F800002440F70024B8F2002404ED00E0AB
:10DF600030B587B00024FEF749FA134D2868B0B1E8
:10DF700000200690059004AA05A906A8FEF7C0FE99
:10DF8000DDE905100222029000230E48CDE90021B0
:10DF9000049A0AA1FFF720FE686000B1012414B1C1
:10DFA00007B0204630BD502080F31188BFF34F8F5B
:10DFB000BFF36F8FFEE7000034010024546D722020
:10DFC00053766300C1CA00082DE9FF4106469C460E
:10DFD0000A9F0020002E15D0154D2C68002C0ED065
:10DFE00000910192029606291BDAFFF723FE022810
:10DFF00010D0002328681A466946FFF771FA04B06A
:10E00000BDE8F081502080F31188BFF34F8FBFF33C
:10E010006F8FFEE7286800233A466946FFF760FAEB
:10E02000EDE70023624669462046FFF70BFBE6E773
:10E030003401002402494FF0000000F008B800BF8E
:10E040000000F87F4FF04070E1EE100A70470CF0CE
:10E050000F03092B08BF082000F059800A2B0BD0B2
:10E06000082B18BF704708BF1CF0400F0AD04FF0B4
:10E0700000004FF0000170471CF0400F18BF4FF038
:10E08000004070471CF0100F08D020F0704300F0E3
:10E090007F4242EAD3014FEA4370704700F060408C
:10E0A00021F07F4242EA000201F07F4040EA7270B4
:10E0B00070474FF0FF0C4CF4E06C1CEA11531CBF8E
:10E0C0009CEA030C9445C2BFDA4201EB025170474F
:10E0D000002B0DD0BCF1000F0FD0002A01F0004141
:10E0E000A4BF41F0E04141F07F614FF00000704774
:10E0F00001F000414FF00000704750EA01334FF04B
:10E100009B0C18BF4CF0806C7FF494AF70471CF4EC
:10E11000801F11D01CF4E02F03D06FEACC314900EE
:10E1200070474FF04050EFF3008222F0704242EA15
:10E13000000282F3008870474FF000007047000033
:10E14000D4E700080000000000000000000000000C
:10E150000000000000100000180000000000000097
:10E1600000000000B8E70008000000000000000008
:10E170000000000000000000001000001800000077
:10E18000000000000000000088139411A00FAC0DE7
:10E19000B80BC4099808D00708074006780514058D
:10E1A000B0044C04E803B603840352032003EE02D8
:10E1B000BC028A0258022602F401CC0190015E01E1
:10E1C00040012C010401E600D200BE00B400AA0008
:10E1D000000000000000000000000000000000003F
:10E1E000000000000000000000000000000000002F
:10E1F000000000000000000000000000000000001F
:10E20000000000000000000000000000000000000E
:10E2100000000000000000000000000000000000FE
:10E2200000000000000000000000000000000000EE
:10E2300000000000000000000000000000000000DE
:10E240000000000000000000000000008813A00F84
:10E25000B80BC409D007DC051405B0044C04E8036E
:10E2600084032003BC020802CC0190015E012C0152
:10E270000401E600D200BE00AA00A0008C008200CB
:10E2800078006E0069005A00550050004D004B00A8
:10E29000480047004600450044004300420041005A
:10E2A00040003F003E003D003C003B003A0039008A
:10E2B0003800370036002D002C002B002A002900E2
:10E2C00028002700000000000000000000000000FF
:10E2D000000000000000000000000000000000003E
:10E2E000000000000000000000000000000000002E
:10E2F000000000000000000000000000000000001E
:10E30000000000000000000000000000000000000D
:10E310008813A00FB80BC409D007DC051405B0049E
:10E320004C04E80384032003BC020802CC019001E2
:10E330005E012C010401E600D200BE00AA00A0008C
:10E340008C00820078006E0069005A005500500071
:10E350004D004B0048004700460045004400430084
:10E360004200410040003F003E003D003C003B00B9
:10E370003A0039003800370036002D002C002B0001
:10E380002A00290028002700260025002400230059
:10E39000000000000000000000000000000000007D
:10E3A000000000000000000000000000000000006D
:10E3B000000000000000000000000000000000005D
:10E3C000000000000000000000000000000000004D
:10E3D000000000008813A00FB80BC409D007DC05AB
:10E3E0001405B0044C04E80384032003BC020802B3
:10E3F000CC0190015E012C010401E600D200BE00B8
:10E40000AA00A0008C00820078006E0069005A000B
:10E41000550050004D004B004800470046004500A5
:10E42000440043004200410040003F003E003D00E8
:10E430003C003B003A0039003800370036002D0020
:10E440002C002B002A002900280027002600250088
:10E45000240023002200210020001F0000000000F3
:10E4600000000000000000000000000000000000AC
:10E47000000000000000000000000000000000009C
:10E48000000000000000000000000000000000008C
:10E4900000000000000000008813A00FB80BC409A2
:10E4A000D007DC051405B0044C04E8038403200302
:10E4B000BC020802CC0190015E012C010401E600BF
:10E4C000D200BE00AA00A0008C00820078006E007E
:10E4D00069005A00550050004D004B0048004700AD
:10E4E00046004500440043004200410040003F0018
:10E4F0003E003D003C003B003A0039003800370048
:10E5000036002D002C002B002A00290028002700AF
:10E5100026002500240023002200210020001F00E7
:10E520001E001D001C001B001A0019001800170017
:10E5300016001500000000000000000000000000B0
:10E5400000000000000000000000000000000000CB
:10E550000000000000000000000000008813A00F71
:10E56000B80BC409D007DC051405B0044C04E8035B
:10E5700084032003BC020802CC0190015E012C013F
:10E580000401E600D200BE00AA00A0008C008200B8
:10E5900078006E0069005A00550050004D004B0095
:10E5A0004800470046004500440043004200410047
:10E5B00040003F003E003D003C003B003A00390077
:10E5C0003800370036002D002C002B002A002900CF
:10E5D0002800270026002500240023002200210017
:10E5E00020001F001E001D001C001B001A00190047
:10E5F0001800170016001500140013001200110077
:10E6000010000F000E000D000C000B0000000000B9
:10E6100000000000000000000000000000000000FA
:10E620008813A00FB80BC409D007DC051405B0048B
:10E630004C04E80384032003BC020802CC019001CF
:10E640005E012C010401E600D200BE00AA00A00079
:10E650008C00820078006E0069005A00550050005E
:10E660004D004B0048004700460045004400430071
:10E670004200410040003F003E003D003C003B00A6
:10E680003A0039003800370036002D002C002B00EE
:10E690002A00290028002700260025002400230046
:10E6A0002200210020001F001E001D001C001B0076
:10E6B0001A001900180017001600150014001300A6
:10E6C0001200110010000F000E000D000C000B00D6
:10E6D0000A00090008000700060005000400030006
:10E6E0000200010000000000010203040102030413
:10E6F00006070809000610160006101601000200A1
:10E700000400060008000A000C0010002000400071
:10E710008000000101010103070100000804020458
:10E720000801010100000000000000000000F03FAF
:10E73000000000000000F83F0000000000000000A2
:10E740000000004003B8E23F0000000000000000AD
:10E7500006D0CF43EBFD4C3E033333333333E33F3B
:10E76000FFAB6FDBB66DDB3F4D268F515555D53F67
:10E7700001411DA96074D13F65DBC9934A86CD3F35
:10E78000EF4E454A287ECA3F3E5555555555C53F23
:10E7900093BDBE166CC166BF2CDE25AF6A56113F15
:10E7A000F16BD2C541BDBBBED0A4BE726937663E17
:10E7B0000000000000000000436F6D6D756E69631E
:10E7C0006174696F6E526573706F6E655461736BBF
:10E7D0000000000064656661756C745461736B00C1
:10E7E00000E80008000000247C010000D4020008BA
:10E7F000DCE800087C0100243456010030030008E6
:10E8000021520A420102126210288813A00FB80B8D
:10E81000C409D007DC051405B0044C04E8038403E4
:10E820002003BC020802CC0190015E012C0104010E
:10E83000E612D212BE12AA12A0128C128212781202
:10E840006E1269125A12551250124D124B12481282
:10E85000471246124512441243124212411240120C
:10E860003F123E123D123C123B123A12391238123C
:10E87000371236122D122C122B122A12291228129C
:10E8800027122612251224122312221221122012DC
:10E890001F121E121D121C121B121A12191218120C
:10E8A000171216121512141213121212111210123C
:10E8B0000F120E120D120C1A0BCE120912081207AB
:10E8C00012061205120412032A02DA14389C1C2CB8
:0CE8D00090D003E4027F101AAA0181001E
:040000050800029954
:00000001FF
